:020000040000FA
:040000006FD00400B9
:101000006F00907E00000000000000009020002093
:10101000AA220020A9BDF9F56C23002000000000E1
:10102000000000006C230020902000200000000041
:101030000000000090200020000000009020002010
:101040000000000090200020902000209020002030
:101050009020002090200020582F00209424002071
:101060000000000090200020902000201E2400207E
:1010700090200020D22300209020002090200020EB
:101080009020002090200020902000209020002020
:101090009020002001A04111B7170040985F3AC688
:1010A000945F3247E39CE6FE3245410182800111A4
:1010B00013078008F337078093F787083EC20100C3
:1010C0000100B7170040930570052380B70413068D
:1010D00080FA2380C7040100010083C6B70493F699
:1010E000F60DA385D704238007049246F3A6068055
:1010F0000100010093760502D5CEF336078093F602
:10110000860836C4010001002380B7042380C70489
:1011100001000100B70614007D89558D88C70100C4
:1011200001000100010023800704A246F3A6068007
:101130000100010073370780137787083AC6010062
:1011400001002380B7042380C704010001000100CF
:1011500001003727004093061005A303D7802380A2
:101160000704B247F3A70780010001009307800836
:10117000F3B7078093F787083ECE01000100B71749
:101180000040130770052380E704130780FA2380CB
:10119000E7040100010003C7B70413670708A3852C
:1011A000E70423800704F247F3A70780010001004A
:1011B0000561828093760504BDC6F336078093F6F9
:1011C000860836C8010001002380B7042380C704C5
:1011D00001000100B7061400938606047D89558D31
:1011E00088C7010001000100010023800704C246F6
:1011F000F3A6068001000100733707801377870884
:101200003ACA010001002380B7042380C70401000B
:1012100001003727004093062005A303D7802380D1
:101220000704D24781B773370780137787083ACC12
:10123000010001002380B7042380C70401000100DE
:1012400098471367070C98C723800704E24719BF24
:101250000111814601468145114506CE97000000E7
:10126000E780605893078008F3B7078093F78708F3
:101270003EC601000100B717004013077005238028
:10128000E704130780FA2380E7040100010003C785
:101290006704136717002383E70423800704B2471A
:1012A000F3A7078001000100F2400561828041112F
:1012B000814601468145114597000000E780A05214
:1012C00013078008F337078093F787083EC40100AF
:1012D0000100B7170040130670052380C70493066A
:1012E00080FA2380D70401000100FD552396B70240
:1012F00023800704A245F3A5058001000100733790
:101300000780137787083AC6010001002380C704CD
:101310002380D7040100010003C767041367170087
:101320002383E70423800704B247F3A70780010063
:10133000010001A0BD473305F50201007D1575FDD3
:101340008280411122C426C206C6AA8401446317C2
:101350009400B24022449244410182800504130566
:10136000803E420497000000E78000FD4180C5B741
:101370009305000273A04580824573901534924016
:101380002242B2424243D2436244F2440255925551
:101390002256B2564257D2576258F25806499649D9
:1013A000264AB64A464BD64B664CF64C065D965DD1
:1013B000265EB65E465FD65F09617300203041113C
:1013C000B7170040985F3AC6945F3247E39CE6FE49
:1013D000324541018280B71700401307000323887C
:1013E000E702854717170000232EF74673002030C9
:1013F000411122C42D6426C24AC006C637190040D6
:101400001304A4AAB704002023208900976000E0F9
:10141000E780E0369C408297976000E0E7802036C6
:10142000E5B737370040834747009146BD8B639E41
:10143000D702B73600401306F00F973500009385AA
:10144000651F9737000083D7E72E03C7A6001377E1
:10145000F70F1DE3B7E70400BC4F09468945171590
:1014600000000345A5F7829731A099466394D70001
:10147000834757007300203003C786001377F70FA8
:10148000E365F6FC13851700AE97173800002313A9
:10149000A82A2380E70075B7B787004003C7670015
:1014A000098B6309071003C77700930600031377BE
:1014B0000703630DD70817380000034878771736FD
:1014C00000001306E6730547B30606012380E60015
:1014D00083C577001737000013078774429793F589
:1014E000F50F2300B70003C58700973500009385EB
:1014F0002572C2951375F50F2380A50003470700D9
:1015000089451377F703630CB70C63E7E50A6306B5
:10151000071A8545630CB7129737000083C75771C8
:101520003307F600034707001377F70F19CB85073A
:1015300093F7F70F3D476363F71A17370000A309C6
:10154000F76EB787004009472383E700B78700405D
:1015500083C77700E207E18763DE0704973700005F
:1015600083C7176D17370000130787693E978546B5
:101570002300D700173700001307876A3E979306AA
:1015800000032300D70017370000130767683E9752
:10159000A14685072300D70093F7F70F3D47636403
:1015A000F71417370000A305F768B787004009470D
:1015B0002383E70073002030930610026300D70EE8
:1015C000930620026305D70693060002E316D7F4BC
:1015D00003C727021377C70F13672700D5A803C7D0
:1015E00067001377070465CB03C7A702173800000D
:1015F00013088842173500001305C539134707083B
:101600002385E70203C7A7021377370F1367870005
:101610002385E702814713070004B305F5008C41D9
:10162000B306F80091078CC2E399E7FEF5B503C74E
:10163000A702134707042385E70203C7A70213770E
:10164000C70F136727002385E702F9B503C76700B3
:101650001377070449C303C767021738000013084C
:10166000682F173500001305A526134707082383A5
:10167000E70203C767021377370F136787002383D7
:10168000E702814713070004B305F5008C41B30658
:10169000F80091078CC2E399E7FEBDBD03C767025E
:1016A000134707042383E70203C767021377C70FB3
:1016B000136727002383E70285B503C76700137705
:1016C000070411CB03C727021377370F136787006F
:1016D0002381E70291B5238006003DBD97370000C6
:1016E000A3880754B9BD97370000A383075475BD7D
:1016F0002303048015472303E48001002302A48010
:10170000828083076480E3CE07FE23030480828007
:1017100083076480E3CE07FE03454480828083070D
:101720006480E3CE07FE2302A4808280411126C498
:101730004AC24EC006C61377F50BAD47AA892E895B
:101740009544630CF700194597000000E78080FA84
:1017500097000000E78020FB8D444E859700000035
:10176000E78040F9FD59FD1463983401B240A2446A
:101770001249824941018280135509011375F50F01
:1017800097000000E780E0F92209F1BF011126CCA3
:1017900006CEB704080097000000E780C0F61545A4
:1017A00097000000E78000F597000000E78080F6D2
:1017B00097000000E78000F62AC697000000E78047
:1017C00080F432459377150089EB13651500137586
:1017D000F50FF240E24405618280FD14E9F0014515
:1017E000CDBF397126DC4ADA4ED852D656D45AD2F9
:1017F0005ED006DE62CE66CCB7E700E07D5783AAF6
:10180000070022C603AA470023A0E71823A2E7186F
:10181000B7170040130770052380E704130780FA09
:101820002380E70483C74704930B75FFB684E20760
:1018300093FBFB0F8546AA892E8B32893724004003
:10184000E187015763FA76016308D50089461307DB
:1018500000026313D5000157D98F93F7F70FB71C18
:1018600000402382FC0411472303E4801305F00F9A
:1018700097000000E78000E8094C97000000E7802F
:1018800080E863657C15B7050700DA9537870700A0
:10189000795563FEE504B3879500636AF704370B57
:1018A0000800A94733EB65016395F90881E8814495
:1018B00097000000E78020E5268515A8DA85094510
:1018C00097000000E780C0E605090345F9FFFD1415
:1018D000050B97000000E780C0E481C49377FB0FFD
:1018E000E5F797000000E780A0EA69F17D55B7179A
:1018F0000040130770052380E704130780FA238054
:10190000E70403C74704418B2382E704F250B7E79B
:1019100000E023A0571123A24711E2543244525948
:10192000C259325AA25A125B825B724CE24C21615C
:101930008280A547639BF90685691309F00FB306FA
:101940009900B3742B01B6941349F9FFB37499004D
:10195000856B33796901416B9387F9FFB3F72701F1
:1019600099E363FC340193D94900C147E3E637FFAB
:101970003DBF0569C1697D19D9B71305800D63881D
:101980006901130500026384790113051008CA85F3
:1019900097000000E780C0D997000000E78040DF93
:1019A00031D54E99B38434416DBFDA852D4597000A
:1019B0000000E780E0D7CA94E30B99EE0509970091
:1019C0000000E78020D5A30FA9FEFDB79387F9FF9C
:1019D00093F7F70F636DFC0C83C71C0413073008E3
:1019E0006315F706370708006361EB06B3079B0032
:1019F000B706100063FBD704334BEB0089476399AC
:101A0000F9068980D549E38404EADA850945970017
:101A10000000E780E0D111090327C9FF9147232087
:101A2000E48003076480E34E07FE23033481FD173F
:101A3000EDFBFD14110B81C49377FB0FE9FF9700B9
:101A40000000E780E0D461F155B5B717004003C747
:101A50005704B70708001377070219E3B787070091
:101A60007955E376FBE833079B00E3F9E7F841B5E6
:101A70008547E380F9F0DA852D4597000000E7807F
:101A800020CB9389F4FFE38404E297000000E78011
:101A900060C893F7390091EB83260480032709007F
:101AA00093074900E396E6E03E89CE84D9BFB54767
:101AB0006399F9001305900B97000000E78080C33D
:101AC000FDB3B1471305B00AE388F9FE9947639760
:101AD000F904B7050800B365BB002D459700000069
:101AE000E78000C581448D4BA14997000000E78045
:101AF00060C263967401832704802320F900850463
:101B0000E39534FF8327048013172B0163550700E7
:101B10002312F90069BB2322F90051BB9D47639F43
:101B2000F90281451305B00497000000E78040C02A
:101B3000BD442320090023220900FD59970000001D
:101B4000E78040BD93F77400CA9703C70700FD14F0
:101B5000398D2380A700E39334FF91BBA14763979E
:101B6000F90697000000E780A0C28144630D0B00D6
:101B70008D479304C0036308FB00930400056304CE
:101B80008B01930440041375C507E30295D21945F0
:101B900097000000E78000B697000000E780A0B63D
:101BA000054597000000E780E0B426859700000017
:101BB000E78020B7094597000000E78080B69700CE
:101BC0000000E780E0BCE31405CE0DB39147639FAE
:101BD000F9001305600697000000E780A0B19700A8
:101BE0000000E78040B213059009F9B5E38109CC04
:101BF000F1547DB9BD660147173600001306C620B3
:101C0000938606A685458347060093F7F70F91C391
:101C100082800507E3F9E6FE973700002386B71EAA
:101C2000DDB77D166206618693178601E18763D46E
:101C3000070001458280931726003307F500AE9711
:101C400018439C4363E7E7007D16E37FF7FC7D556F
:101C5000828005458280FD15E205E18513978501A7
:101C6000618793F7F50F63480700FD15139725006B
:101C70002A97584365D713851700620561858280CE
:101C80003308B5021C4283A80600B335B502C297DB
:101C900033B50701AE98469585486367B5006394F0
:101CA000A50063E3070181480C43C6950CC388C2B5
:101CB0001CC2828081471397870161876343B70005
:101CC0008280139727002A97232007008507E5B70E
:101CD0008147014793968701E18663C5B6001335B6
:101CE0001700828093962700AA9694428507558F05
:101CF000D5B793D755408A07AA979C430545331516
:101D0000B5007D8D828017F3FFDFE702833D2A84D3
:101D100097000000E78060F405C5931725003E9406
:101D20000327C4FF814711EB7D1516053E9542053B
:101D3000418517F3FFDF6700033D05838507E5B79E
:101D40000145C5BF81471397870161876343C7007A
:101D5000828013972700B386E50094422A9785076F
:101D600014C3D5B77D1662066186014793178601B5
:101D7000E18763D50700133517008280931726008B
:101D8000B306F500AE9794429C437D16B58F5D8FE8
:101D9000F1BF8A05AA9501476363B500828083A6D7
:101DA000C5FFF11593D71600D98F9CC11397F60183
:101DB000E5B72A830148014701456343D700828084
:101DC000B387050183A80700B30706019C43C697A4
:101DD000AA976384F80033B517010507B308030118
:101DE000620723A0F80061871108C1BF2A83014759
:101DF0008147014563C3D70082803388E50083288B
:101E00000800330EE600032E0E003388A840330886
:101E1000C8416384080133B508018507B308E300AE
:101E2000E20723A00801E1871107E9B717F3FFDFF5
:101E3000E702232B0111B286B2842E86AA850A8579
:101E400097000000E780C0FA2A84A6850A859700DB
:101E50000000E78020E833348000060413351500C5
:101E6000018D056117F3FFDF6700E32917F3FFDF3B
:101E7000E702A3244111AA89AE8A328BB68402C23A
:101E800002C402C60144131C8401135C8C416349E3
:101E90009C02939B1400FD1B0549138CF4FFF15C1D
:101EA00033048901620461846340740792478E049D
:101EB000CE9423AEF4FE410117F3FFDF67006323E6
:101EC00013192400B30B2B01014A93172A00D6974C
:101ED00083A50B0088437800340050009700000071
:101EE000E78040DA050A93178A01E187F11BE35E78
:101EF000FCFC92474E9905042320F900A2473EC2FC
:101F0000B24702C63EC441B7131A8901135A8A4127
:101F1000131D240093178A01E18763CF970092472E
:101F20000A044E941CC0A24705091379F90F3EC25A
:101F3000B24702C63EC4ADB7B3079A0313152A00D1
:101F400056950841780034005000050AEA97DA9760
:101F50008C4397000000E780E0D26DBF197106C284
:101F600012C416C61AC81ECA22CC26CE2AD02ED219
:101F700032D436D63AD83EDA42DC46DECAC0CEC2C9
:101F8000D2C4D6C6DAC8DECAE2CCE6CEEAD0EED2F9
:101F9000F2D4F6D6FAD8FEDA971500009385058CB0
:101FA0008841E700050092402242B2424243D243B8
:101FB0006244F244025592552256B2564257D257C5
:101FC0006258F25806499649264AB64A464BD64BBD
:101FD000664CF64C065D965D265EB65E465FD65F45
:101FE0000961730020300000972100209381810156
:101FF000175100201301018117F5FFFF1305C500DC
:102000009705002093850500171600201306C6FDCE
:1020100063FAC5008322050023A055001105910530
:10202000E3EAC5FE17050200130545F197150020E8
:102030009385C5FB171600201306C66563FAC50015
:102040008322050023A0550011059105E3EAC5FE92
:1020500017150020130505649745002093858526F4
:102060006377B500232005001105E36DB5FEFD4241
:10207000739002BC8D4273904280B722000093821D
:10208000828873900230970200209382A2F793E235
:10209000320073905230975200009382828873907E
:1020A00012346FB0F47573002030397101436EC67D
:1020B00019A0397141536AC866CA62CC5ECE19A0B4
:1020C000397101535AD056D252D44ED64AD826DA54
:1020D00022DC06DE33016140828241114AC026C201
:1020E00022C406C68282B24D4101024D924C224C5E
:1020F000B24B4101024B924A224AB2494101024984
:1021000092442244B240410182803D432A87637356
:10211000C3029377F700BDEFADE5937606FF3D8AE6
:10212000BA960CC34CC30CC74CC74107E36BD7FE30
:1021300011E28280B306C3408A0697020000969699
:102140006780A6002307B700A306B7002306B700E1
:10215000A305B7002305B700A304B7002304B70005
:10216000A303B7002303B700A302B7002302B700FD
:10217000A301B7002301B700A300B7002300B700F5
:10218000828093F5F50F93968500D58D9396050182
:10219000D58D61B7939627009702000096968682A8
:1021A000E78086FA9680C1171D8F3E96E374C3F8C8
:1021B000A5B73367B500FD530D8B79E7B7877F7FF0
:1021C0009387F7F710419441B372F6003363F6003A
:1021D000BE92B3E262006397720C6318D606504158
:1021E000D441B372F6003363F600BE92B3E26200EC
:1021F0006398720A631BD60410459445B372F600C7
:102200003363F600BE92B3E262006391720A631E0A
:10221000D6025045D445B372F6003363F600BE9241
:10222000B3E26200639A72086311D60210499449BE
:10223000B372F6003363F600BE92B3E262006393BA
:1022400072085105D105E30FD6F6131706019397CF
:102250000601631CF7001357060193D706013305E7
:10226000F7409375F50F91E982804183C18333056F
:10227000F7409375F50F91E182801377F70F93F78D
:10228000F70F3305F74082800346050083C605003B
:10229000050585056313D60065FA3305D6408280AF
:1022A00011059105E312D6FE014582802105A105A5
:1022B000E31CD6FC014582803105B105E316D6FC4E
:1022C000014582804105C105E310D6FC01458280AD
:1022D000B717004003C777051377E70FA38BE70411
:1022E000130700F8A38DE7043D47238CE704130789
:1022F0005003A38CE70403C7A7051377D70F238DDB
:10230000E7048280B717004003C7E7020D89411137
:102310001377C70F498F93068008F3B6068093F6AC
:10232000860836C601000100930670052380D70495
:10233000930680FA2380D704010001002387E70277
:1023400023800704B247F3A7078001000100410181
:10235000828041112A83014E930E407E130F001993
:10236000930F400663E56E129308001913034006AD
:10237000B3781503854E0D4FA14F337365020D8958
:102380001335150063EFBE121308F6FF79467298F5
:102390004208135808013307C70213D61700BE07B7
:1023A00032976146B3F6C60213068070B386C60242
:1023B0003697A166F58F42075D8FB716004083C739
:1023C000F60293F70708A303F1000346710083C7E1
:1023D000F60293F70708E394C7FE83477100B71628
:1023E000004093F7F70F6388071293078008F3B74D
:1023F000078093F787083EC401000100B71700402B
:10240000930670052380D704930680FA2380D704AF
:102410000100010023AA070383C6170393E60608F9
:10242000A388D70223800704A247F3A707800100EF
:1024300001001166B71700407D16D45BC85F938515
:102440004703A98EF18EF5FA93068008F3B606804D
:1024500093F6860836C601000100930670052380B6
:10246000D704930680FA2380D7040100010098C1A5
:1024700003C7170313670704A388E7022380070431
:10248000B247F3A7078001000100410182807D135C
:102490003368E3039308E016630E08003368F30320
:1024A0009308D016630808009378330093B8180097
:1024B0009388D81633081E01131E0801135E0E01FF
:1024C00055B56393E5030548638608000148630337
:1024D00003002A8871087298FD15131E0801C205B1
:1024E000135E0E01C18179BD13F8150063F4BF00BE
:1024F0007908D5B713381800E5BF83C7F60293F7FC
:102500000708A303F1000346710083C7F60293F79F
:102510000708E394C7FE8347710093F7F70FF1DFD5
:10252000E9B531714AD966CB06DF22DD26DB4ED70D
:1025300052D556D35AD15ECF62CD6AC96EC7AA8C26
:1025400002D897100000E78020B12A8993078008FD
:10255000F3B7078093F787083EDA01000100B71749
:102560000040130770052380E704130780FA2380D7
:10257000E7040100010003C7F7021377770FA38771
:10258000E70203C7F70213678700A387E7022380E8
:102590000704D257F3A70780010001000545970003
:1025A0000000E78060D6130780C13347E902116A53
:1025B00093070AE893065002BD69930BA004814A71
:1025C000014B13048008930470057D1AB347F90288
:1025D0003307D7023EC0FD873ECC938709A69309F7
:1025E000803E3347F7023AC27D873AC43347390306
:1025F0008549B399990193D93940B306D702B30BF2
:102600007703B3C6F602B3CBFB0236C6FD8636C8E7
:1026100093D6FB4136CEB7460F0093860624334946
:10262000D9028566938606FAB3969601B389E902C4
:10263000130760553309D90293060010B389E902E4
:102640003349D902B3C9F9029316390036CA37198A
:102650000040FD8636D0930D090493D7F9413ED250
:10266000F336048093F6860836DC010001009307F8
:1026700070052380FD00930680FA2380DD000100B1
:1026800001008346390593F6860FA309D9048346D2
:10269000390593E61600A309D90423800D00E256FC
:1026A000F3A6068001000100130C80FA116DF336C9
:1026B000048093F6860836DE01000100930770055A
:1026C0002380FD0023808D01010001008346390530
:1026D000216693E60602A309D90483560905B3E6E9
:1026E000A6012318D90483560905D18E2318D904CD
:1026F00023800D00F256F3A60680010001008346F8
:10270000390593F606026381061A03463905218AC4
:102710006DDE081897100000E7800098733604807B
:1027200013768608B2C20100010023809D00238039
:102730008D0101000100B717004003C6370513766D
:10274000F60DA389C70403C6370513660602A389DD
:10275000C704835609052166B3E6A6012318D904E8
:1027600083560905D18E2318D90423800D0096467F
:10277000F3A60680010001008346390593F60602A0
:10278000638B061483463905A18AEDFE970000206D
:10279000E7806090AA8636D497000020E780A08F5B
:1027A000A256E30AD5FE835609054255B3E6A601B3
:1027B0002318D90497100000E780C08F834639059D
:1027C000A18AEDDE03560905834629058247337643
:1027D000CA00B306DA0293D5F641B296B388F64042
:1027E000E24733B8C6002E983308F840A247B3B684
:1027F00016013308D84063C70701631DF8009247EC
:1028000063FA1701C247634FF80E63950701B24799
:1028100063EAF80E894663E9660FF24693151800DD
:1028200013D3F8015E8613951800B365B30042D642
:1028300046D497C00100E78060DD3258050B137B5A
:10284000FB0F63470001631A0838A25863870838F2
:1028500013081500B336A800B69513D6F5013298C3
:10286000B336C800AE9613581800FE06B3E606014C
:102870007336048013768608B2C6010001002380F7
:102880009D0023808D01010001000356C902B2960C
:10289000C206C1822316D90223800D00B646F3A6D4
:1028A00006800100010021B5F336048093F6860806
:1028B000B6C00100010023809D0023808D0101002E
:1028C00001008346390593E60602A309D904238053
:1028D0000D0086460DB5F336048093F68608B6C41F
:1028E0000100010023809D0023808D010100010073
:1028F0008346390593E60602A309D90423800D0017
:10290000A646BDB5E30B0BF0F336048093F68608BC
:10291000B6C801000100930680FA23809D00238041
:10292000DD00010001008346390593F5FC0F93F6A5
:10293000860FA309D90483463905CD8EA309D9048E
:1029400023800D00C646F3A6068001000100130592
:1029500080FA03463905930639051D8A631C9629BA
:102960007336048013768608B2CC0100010013068A
:1029700080FA23809D002380CD000100010003C662
:1029800006001376F60D2380C60003C60600136604
:1029900006022380C600835609051166D18E2318CE
:1029A000D904835609052166D18E2318D9042380C2
:1029B0000D00E646F3A6068001000100130680FA2A
:1029C0008346390593F60602638006268346390559
:1029D000130C3905A18AFDDA081897000000E7807A
:1029E000A06BF336048093F68608B6D00100010090
:1029F000930680FA23809D002380DD000100010002
:102A000083460C00116693F6F60D2300DC00834626
:102A10000C0093E606022300DC0083560905D18EE4
:102A20002318D904835609052166D18E2318D904A9
:102A300023800D008656F3A60680010001001306D0
:102A400080FA8346390593F60602638A0620834698
:102A50003905A18AEDFE97F0FF1FE780C0632A8C3D
:102A600097F0FF1FE7802063E30C85FF835609057D
:102A700011664255D18E2318D90497000000E780D3
:102A800060638346390513063905A18AFDDAF336FA
:102A9000048093F68608B6D401000100930680FAFC
:102AA00023809D002380DD00010001008346060095
:102AB00093F6F60D2300D60023800D00A656F3A64C
:102AC0000680010001008356090503462905D24707
:102AD000B376DA003306CA021305800C9355F6412B
:102AE0003696330DF6408257333CD6002E9C333653
:102AF000A601330CFC40330CCC40330885039256BE
:102B00004E86B335A5033305A503C29597C00100D2
:102B1000E780C0AF63468001631E0C16630C0D1680
:102B2000130615003335A6002E959356F5013696FB
:102B3000B335D600AA959396F50105828585D18E89
:102B40006346B000639D051A638B061A0356C902DB
:102B500015823305D6003336C500B2956348B00000
:102B6000639105241306F00F637DA622894663F363
:102B7000561593078008F3B7078093F78708BED6EA
:102B80000100010037170040930770052300F70488
:102B9000930780FA2300F704010001008356C7025F
:102BA00089678117D58FC207C1832316F7022300D7
:102BB0000704B657F3A7078001000100FA506A54D2
:102BC000DA544A59BA592A5A9A5A0A5BFA4B6A4C49
:102BD000DA4C4A4DBA4D296182801308F5FF33352E
:102BE000A800FD152E951356F5013298B336C8008E
:102BF000AA9695B9F336048093F68608B6CA010002
:102C0000010023809D002380AD0001000100834668
:102C10003905CD8EA309D90423800D00D646F3A62D
:102C200006800100010035B3F336048093F6860870
:102C3000B6CE0100010023809D002380CD0001005D
:102C400001008346390593E60602A309D9042380CF
:102C50000D00F646F3A606800100010095B3F33699
:102C6000048093F68608B6D20100010023809D00FF
:102C70002380CD00010001008346390593E606025A
:102C8000A309D90423800D009656F3A606800100FF
:102C9000010045BB9306F5FF33B5A600FD152E9543
:102CA0009355F501AE96B3B5B600AA951396F50106
:102CB000858269B5F336048093F68608B6D801009C
:102CC0000100930680FA23809D002380DD0001002F
:102CD00001008356C9020566011693F6F60FD18EE0
:102CE000C206C1822316D90223800D00C656F3A660
:102CF000068001000100850A93FAFA0F95B233E6C7
:102D0000B60045C20356C9023305D0403338A0008F
:102D1000B305B040B385054115826345B000D1E1EC
:102D20006371A608894663F0560593078008F3B7D8
:102D3000078093F78708BEDA01000100B71700404B
:102D4000130770052380E704130780FA2380E70444
:102D50000100010003D7C7027D8B2396E702238081
:102D60000704D65781BDF336048093F68608B6DC97
:102D700001000100930680FA23809D002380DD007E
:102D8000010001008356C9020566011693F6F60F8D
:102D9000D18EC206C1822316D90223800D00E656C9
:102DA000B9B793078008F3B7078093F78708BEDEAB
:102DB0000100010037170040930770052300F70456
:102DC000930780FA2300F704010001000356C702AD
:102DD00093975600B297C207C1832316F7022300C8
:102DE0000704F657C1BB914763EEB70217D701003E
:102DF0001307071F8A05BA959C41BA978287B717B0
:102E0000004003A7470B1345F5FF698F23AAE70A84
:102E100003A7070B698F23A8E70A03A7070A798D81
:102E200023A0A70A8280B717004083A6470B134749
:102E3000F5FFF98E23AAD70A83A6070B558D23A881
:102E4000A70A83A6070A758F23A0E70A8280B7170F
:102E5000004003A7470B498F23AAE70A03A7070BE4
:102E60001345F5FF45BFB717004083A6470B13472F
:102E7000F5FF758F23AAE70A03A7070A598D4DB7F7
:102E8000B717004003A7470B498FEDB7914763EE93
:102E9000B70217D701001307E7158A05BA959C41B9
:102EA000BA978287B717004003A7470D1345F5FF70
:102EB000698F23AAE70C03A7070D698F23A8E70CE6
:102EC00003A7070C798D23A0A70C8280B7170040B9
:102ED00083A6470D1347F5FFF98E23AAD70C83A6C7
:102EE000070D558D23A8A70C83A6070C758F23A06B
:102EF000E70C8280B717004003A7470D498F23AA2C
:102F0000E70C03A7070D1345F5FF45BFB7170040B2
:102F100083A6470D1347F5FF758F23AAE70C03A778
:102F2000070C598D4DB7B717004003A7470D498FC0
:102F3000EDB7797122D43714004026D24AD0035914
:102F400024028354040206D64209C2044ECE52CC57
:102F500056CA13590901C1802DE11379F9F793F489
:102F6000F49F4209C20413590901C18093078008E4
:102F7000F3B7078093F787083EC401000100930769
:102F800070052300F404930780FA2300F404010081
:102F90000100231124032310940223000404A247F8
:102FA000F3A7078001000100B25022549254025945
:102FB000F249624AD24A45618280B7F507008146EC
:102FC0003000B105194597000020E7808081A247B5
:102FD00013972701E34A07FC1369090893E40440A7
:102FE00093098008F3B7098093F787083EC0010072
:102FF0000100930A700523005405130A80FA230088
:10300000440501000100231124032310940223002E
:1030100004048247F3A7078001000100294597F0C7
:10302000FF1FE7802031F3B9098093F989084EC268
:1030300001000100230054052300440501000100A4
:103040008357040293E707202310F40223000404AB
:103050009247B9B7B7170040884742054181937737
:10306000050491EB9377F5013755E80113050580C9
:103070003345F50282809377050C130700046397AC
:10308000E7009377F50137459C1CCDB72165130503
:1030900005D0828037E700E01C435443A183E20659
:1030A000D58F1CC1FD572320F7182322F7188280E3
:1030B00013178500B7E700E023A0E710618123A282
:1030C000A7108280B7F700E08847CC47828081470D
:1030D00037370040A14663C4C7003285828003456C
:1030E000B740E38EA6FE3385F5000345050085074E
:1030F0002304A740CDB797070020938727EF9C4371
:10310000173700201307071C3E95636EE50017373D
:1031100000201307274F6368A70017070020232705
:10312000A7EC3E858280FD57EDBF8280411122C40D
:1031300006C62A8497000000E78000F22947B307FB
:10314000E502B2408D83B3D7870222449507B3D7F7
:10315000E70237370040C207C1832316F700410159
:103160008280411137150E0006C697000000E780E7
:1031700020FCB7370040130770F82381E7000D47A4
:10318000A381E70013070004A380E7000547238716
:10319000E700B24041018280373700408347270073
:1031A0001A0593F7F703C98F93F7F70F2301F70079
:1031B0008280B737004003C7170019C9D98DA38093
:1031C000B70003C70700136787002380E7008280EA
:1031D00093C5F5FFF98DA380B7008280AE872A875B
:1031E000B736004021463738004089E71703000012
:1031F0006700E3F383C8B600E30916FF05078348B9
:10320000F7FFFD17C20723041801C183F9BF41115D
:1032100022C406C62A8497000000E780E0E329471D
:10322000B307E502B2408D83B3D7870222449507E6
:10323000B3D7E70237370040C207C1832316F740F0
:1032400041018280716541111305052006C6970072
:103250000000E78000FCB7370040130770F82381B7
:10326000E7400D47A381E74013070004A380E74030
:1032700005472387E740B24041018280CC4141119C
:1032800006C6328503C6150083C5050022064D8E8D
:1032900042068D654186138875A2630C0611634B47
:1032A000C804138845A26300060D634AC8009385CD
:1032B00035A26301B6082390060029464DA0138865
:1032C00055A26305060D938565A2E316B6FE8D45EE
:1032D0001D4663E6E5081146198E63F3C7003E8676
:1032E000B7E704002390C600FC4797D501009385FB
:1032F000A5D29DA0138895A263030611634E060D07
:103300001388A5A263000613938505A5E315B6FAF5
:1033100099451D4663E5E504198E63F3C7003E86B3
:10332000B7E704002390C600FC479705002093856B
:1033300025D61DA09D451D4663E3E5022146198E55
:1033400063F3C7003E86B7E70400FC472390C6003E
:103350009705002093858534BA9582970146B2403F
:10336000328541018280AD451D46E3EAE5FE3146E6
:10337000198E63F3C7003E86B7E704002390C600AA
:10338000FC4797D501009385A5CBF9B7B1451D46FC
:10339000E3E7E5FC3546198E63F3C7003E86B7E7E1
:1033A00004002390C600FC4797D50100938545CAC9
:1033B00065B78D451D46E3E4E5FA1146198E63F3C2
:1033C000C7003E86B7E704002390C600FC4797D5A8
:1033D0000100938525C549B78D451D46E3E1E5F814
:1033E0001146198E63F3C7003E86B7E704002390A9
:1033F000C600FC4797D50100938545C7B1BFA545D9
:103400001D46E3EEE5F42946198E63F3C7003E86B8
:10341000B7E704002390C600FC4797D501009385C9
:1034200025C11DBFB5451D46E3EBE5F23946198EB2
:1034300063F3C7003E86B7E704002390C600FC474D
:1034400097D50100938545BC01BFB7E7040003A3EE
:103450000713970600209386A6C24146A545170587
:1034600000201305E5B802832D455DE703C505007F
:103470000947631FE50803A84500411106C6034735
:10348000180032850346080022074168518F9308CF
:1034900028FE6307170563E9E800051863030703BF
:1034A00023900600294591A8130648FE630AC70425
:1034B0001518E31707FF15463E87637BF60015478F
:1034C00001A8130600023E876374F600130700028A
:1034D000B7E704002390E600FC471316070111A884
:1034E0003E8691C30546B7E70400FC472390C6001B
:1034F0004206CC45418282970145B240410182801B
:10350000130600083E87E375F6FC13070008C9B7E9
:103510002390060005458280828041677917630405
:10352000E504411122C406C685472A84639FF5003D
:10353000B7E7040022852244B24003A3871397050E
:1035400000209385E52F4101028389476399F500A7
:10355000B7E7040083A7070B8545829771D9B2406E
:103560002244410182808280797126D252CCAE847D
:103570002A8A97D50100938565B117D501001305F7
:1035800065B306D63AC622D44AD0368432894ECEA6
:1035900097B00100E780C052A28517D5010013053E
:1035A00065B297B00100E780A051294597B00100AE
:1035B000E780E05583C7840093F70702F9E383C9E6
:1035C00004008947054532476396F908D44083C70C
:1035D000160083C60600A207D58FC166138616FEA5
:1035E000638CC7028D16638FD7068D6693862690EF
:1035F00029456391D706B7E70400A286225403A3A6
:103600004714B250F2494A86A6850259925452850F
:10361000624A8547456102832D450DEF93070002FD
:10362000354563E98702B7E70400FC47C844130641
:103630000002CA8582978149970700209387072156
:103640009C43014581CB9C4391C74E852286CA8508
:1036500082970145B250225492540259F249624A6B
:10366000456182802D457DF79307700F3545E3E373
:1036700087FEB7E70400FC47C8442286CA858297C4
:1036800065BF2145C1BF411122C437E4040083272F
:10369000841326C2AA84416506C697050020938537
:1036A000251A7D1582978327C40A17050000130584
:1036B00005E78588829795C0032304132244B2400E
:1036C000924497060020938626AE4146C5451705CD
:1036D00000201305659C41010283B24022449244BC
:1036E00001454101828019C59707002023A0A71634
:1036F00001458280454582801147636AA70A97D6B3
:103700000100938666970A0536951841411106C651
:103710003697AE87B2850287130700026145639D25
:10372000E700B7E70400FC47130600021705002076
:10373000130545F782970145B24041018280054754
:103740006145E39BE7FEB7E70400FC470546170524
:103750000020130525F7F9BF1307700F6145E39D9E
:10376000E7FCB7E70400FC471306700F17050020BD
:10377000130585F5C1B7130700086145E39EE7FA15
:10378000B7E70400FC4713060008170500201305DF
:1037900025034DB715476145E390E7FAB7E7040005
:1037A000FC471546170500201305C50961B70945F3
:1037B0008280411126C2B7E4040083A7C41322C447
:1037C0004AC006C62E8497050020938565072A897E
:1037D0008297058905C5970700209387E78B83D7D4
:1037E000A70BA28503A3440D2310F4002244B2408A
:1037F00092444A850249014641010283B240224473
:103800009244024949454101828097070020238163
:1038100007049707002023AF0702B717004003A74C
:10382000070CB706C0FFFD16758F23A0E70C03A792
:10383000070DB7064000558F23A8E70C03A7070C18
:103840003D9B23A0E70C03A7070D1367070123A8DF
:10385000E70C8280B717004003A5470C83A7470CED
:10386000598113451500C18B058999E3136525001E
:103870009707002083C7C7FD6380A7029707002032
:103880002388A7FC11C9970700209387A7FC03A3EF
:1038900007006303030002838280114517F3FFFFD3
:1038A000670063C8011122CC06CE3714004026CA37
:1038B0004AC84EC652C483447405034AB4058349BA
:1038C00084050349940597F0FFFFE780A0A0834794
:1038D000A40593F4F40F137AFA0F93E71700230D5E
:1038E000F40493F9F90F1379F90FB717004003C7E0
:1038F000A705058B6DFF03D5C705A38D4705238C51
:103900003705A38C2705A38B9704F2406244D24469
:103910004249B249224A05618280411193970501CB
:1039200022C406C626C2C1872E8463DC0700B7E422
:103930000400FC54829719C1BC5482972165218DE3
:1039400015A893F7150013C515008DE793F725000B
:103950009DC797000000E78020F0B7E70400BC4F48
:103960001306000A894517050020034525EF8297B5
:1039700013452400B240224492444101828093972F
:10398000250163D80702B7E4040083A7C41E829709
:1039900097000000E780A0F0BC4C375607001306E4
:1039A0000630896517050020034545EB82970965B8
:1039B00079B7939715010145E3DE07FA17C50100B2
:1039C0001305457897B00100E7806027B7E704004A
:1039D000BC4F13060064916517050020034505E8F8
:1039E00082971165A9BF1D71A2CC37E404005C5C0D
:1039F000485886CE494697C5010093852570829721
:103A000011E917C501001305A57097B00100E78003
:103A1000002301A0B7F600E0795798CAFD57DCCA29
:103A20000567B7E700E023A0E7101306F00290C295
:103A300023A0E718010001003707002018471306EC
:103A4000000481459706002023A8E6E04157A38A99
:103A5000E7403C4408088297970700209387077D3A
:103A60003EC8856713870740938757D1231AE10023
:103A70002312F1021307B00F97F7FFFF9387C76474
:103A80002310E1023ED81547970700009387C7E14E
:103A9000B7F50700A30FE1003EDC054797070000DC
:103AA0009387E7DF81463000E10519452301E102F4
:103AB0003EDE97F0FF1FE780C0D218088147994685
:103AC00030003E960346060085070507A30BC70096
:103AD000E398D7FEC24791C70357410185676373D7
:103AE000F70001A0B7E7040083A7470A08088297F8
:103AF000AA8511C917C501001305C56297B0010059
:103B0000E78000FC01A0F6406644256182804111F7
:103B100026C2B7E4040083A7040806C622C417051A
:103B200000001305C5DF829717040020130404D397
:103B30002300A40097000000E780800297000000A7
:103B4000E780E0CC03450400224403A38405B2408F
:103B5000924413060032896541010283797106D6C9
:103B600022D413078008F337078093F787083EC2F3
:103B700001000100B7170040930570052380B704CA
:103B8000130680FA2380C7040100010083C6F702F0
:103B900093F6A60FA387D702238007049246F3A6C5
:103BA00006800100010073370780137787083AC445
:103BB000010001002380B7042380C7040100010035
:103BC00003C7F70213672700A387E70223800704D0
:103BD000A247F3A7078001000100054597E0FFFF1A
:103BE000E780807297000000E78060CB0147814644
:103BF0008147054685451305407E97E0FFFFE78036
:103C0000807537E404003C44680051468145829742
:103C1000B707C0A83EC8B787E803938707D03ECA56
:103C200097E7FF1F9387A7793EC67C586800829765
:103C3000B250225445618280411197D5010093858D
:103C4000A5B217C501001305E54606C697B00100E9
:103C5000E78000E717D501001305C5C997B001003B
:103C6000E78000E6B2402945410117B30100670033
:103C700003EA411197D50100938545B017C50100AE
:103C80001305454306C697B00100E78060E317D5EA
:103C900001001305E5C497B00100E78060E2B2407F
:103CA0002945410117B30100670063E6411122C4B1
:103CB00006C6834705002A849DC797D501009385D2
:103CC000A5B117C501001305E53E97B00100E780D7
:103CD00020DF4C4017D50100130505D497B0010033
:103CE000E78000DE3DA058410DEF97D50100938598
:103CF000A5AE17C501001305E53B97B00100E780AD
:103D000020DC17D501001305A5D297B00100E7808C
:103D100020DB2244B2402945410117B3010067006E
:103D200003DFA1679386D7036313D70297D50100FA
:103D3000938585AA17C501001305C53797B0010003
:103D4000E78000D817D50100130585CF7DBFED07AB
:103D500097D50100938545A817C501001305853542
:103D6000631BF70097B00100E78080D517D50100ED
:103D7000130545CE59BF97B00100E78060D44C4091
:103D800017D50100130505CF91BF411197D501004B
:103D9000938505A017C501001305C53106C697B068
:103DA0000100E780E0D1B2402945410117B301008D
:103DB0006700E3D5797122D426D24AD02E842A898D
:103DC0008145B2844800714606D697E0FFFFE78040
:103DD000003497F7FF1F9387275EDC4783D70700E0
:103DE000231421012313F10097500000E780E0E63F
:103DF0008547A305F1009307401F3EC6FD572305E5
:103E0000A100230AF10097500000E78040F92686C0
:103E1000A285480097500000E78000E7B250225486
:103E2000925402594561828097270020239307907E
:103E300097170020238C077EB7E70400BC47411189
:103E400006C641468145170500201305A52C82971B
:103E5000170700200347072E9307F00A6315F702A0
:103E60009307F0F88945170500201305A52C1707BF
:103E700000202301F72C97070020A38D072A9760C5
:103E80000000E780A0A097600000E78000CC97606A
:103E90000000E78080CE81453705040097070020A9
:103EA00023A80726970700202392072697070020BC
:103EB000238F072497070020239E071C97070020C5
:103EC000239C071A970700202391072497070020B7
:103ED000239A072497300000E780602B0145976004
:103EE0000000E780A0A397D501009385E58C17C556
:103EF00001001305251C97B00100E78060BC17D5B1
:103F00000100130565BD97B00100E78060BBB240BA
:103F10002945410117B30100670063BF4111814684
:103F200017F6FF1F13068646854517050020035523
:103F3000651406C697C00000E780402A15C997D5CA
:103F400001009385258817C501001305A51697B0B4
:103F50000100E780E0B617D501001305E5A797B08B
:103F60000100E780E0B5294597B00100E78020BA5D
:103F700097D501009385058517C5010013058513A5
:103F800097B00100E780C0B317D50100130505A65F
:103F900097B00100E780C0B2294597B00100E780E3
:103FA00000B797F7FF1F93872741DC47054797D551
:103FB0000100938525812390E70017C501001305B3
:103FC000650F97B00100E780A0AF17D5010013057A
:103FD00025A397B00100E780A0AEB240294541017A
:103FE00017B301006700A3B2011122CC06CE26CA86
:103FF0004AC84EC693F715002E84B5CB9700000033
:10400000E78000F2930710F8170700202304F71247
:104010009707002083D7C70517070020A30CF710C8
:104020009145A183170500201305C510170700202F
:104030002303F71097070020A38F070E9760000057
:10404000E780C084B7E70400BC4F13060014930553
:104050000010170500200345E580829713451400E2
:10406000F2406244D2444249B2490561828093F7EA
:104070000510B1C3054597600000E780208A171539
:1040800000200355056B97500000E780A05597204E
:104090000000E780602D9707002083C7F71889E7A5
:1040A00097600000E78060AA97600000E780E0ACBE
:1040B0001345041075B793F72500E9CF17070020C3
:1040C0000357C70469C7AD64B71900409384A4AA15
:1040D00023A099009706002093868603944297D7E1
:1040E0000100938767A11706002003464602814519
:1040F000170500201305050297700000E780C0290E
:1041000023A0990097F7FF1F239CA71A2A8941C172
:1041100097C501009385C57117C50100130585F981
:1041200097B00100E780C099CA8517C50100130543
:10413000251097B00100E780A098294597B00100AD
:10414000E780E09C97070020239207FC930710F874
:10415000170700202300F7FE9707002083D747F1B9
:1041600017070020A308F7FCA183170700202304EA
:10417000F7FC91458D47170500201305A5FB170790
:104180000020A30AF7FA97500000E780207013453B
:104190002400F9B593F74500D1C397C50100938575
:1041A000256917C501001305E5F097B00100E78008
:1041B000209117C501001305650997B00100E7803C
:1041C0002090294597B00100E7806094930720F87C
:1041D000170700202300F7F69707002083D787EB07
:1041E00017070020A308F7F4A18317070020230472
:1041F000F7F4854717070020A30FF7F29750000048
:10420000E780E0B9170500201305C5F291459750E6
:104210000000E780A0671345440099B593F7850037
:10422000A9C797C501009385A56017C501001305AF
:1042300065E897B00100E780A08817C50100130565
:10424000250297B00100E780A087294597B00100BB
:10425000E780E08B97070020239A07EA9770000019
:10426000E780602313458400E5BB93F70501D1C3C4
:104270008545170500200355E5E197600100E780BB
:1042800020D997C501009385A55A17C501001305CC
:1042900065E297B00100E780A08217C50100130511
:1042A00065FD97B00100E780A081294597B0010026
:1042B000E780E085930730F817070020230CF7E626
:1042C0009707002083D707DD17070020A304F7E630
:1042D00017050020130505E6A1838D45170700206B
:1042E000230BF7E497500000E780405A1345040180
:1042F00085BB93F70502D1C797C501009385455348
:1043000017C50100130505DB97A00100E780407B7E
:1043100017C50100130545F897A00100E780407A12
:10432000294597A00100E780807E930740F8170792
:1043300000202301F7E09707002083D7E7D3170772
:104340000020A309F7DEA183170700202305F7DE6D
:10435000854717070020A300F7DE97070020239D5D
:1043600007D097500000E78080A3170500201305B1
:1043700065DC914597500000E780405113450402E9
:10438000C5B193F70504FDC397C501009385454A60
:1043900017C50100130505D297A00100E780407200
:1043A00017C501001305C5F097A00100E780407113
:1043B000294597A00100E78080759707002083C7F3
:1043C00067D71307700A6386E7061307800A638CB2
:1043D000E7081307600A6393E704930760F8170779
:1043E00000202309F7D49707002083D707D21707A7
:1043F0000020A301F7D4A18317070020230DF7D2D3
:10440000854717070020A30CF7D2B14517050020F8
:10441000130545D297500000E780404797500000B1
:10442000E780E0971345040497070020239F07CCFB
:1044300005B9930770F817070020230DF7CE9707EB
:10444000002083D787CC17070020A305F7CEA183D0
:10445000170700202301F7CE854717070020A30D7B
:10446000F7CC994565B7930780F8F1B793F705083E
:104470000145E38707BE97C501009385653B17C5D6
:104480000100130525C397A00100E780606317C5ED
:104490000100130565E397A00100E78060622945EC
:1044A00097A00100E780A0669307A0F817070020F7
:1044B0002302F7C89707002083D7C7C61707002035
:1044C000A30AF7C6A183170700202306F7C685476E
:1044D00017070020A301F7C697070020239407C4FD
:1044E00097500000E780A08B17050020130585C4B6
:1044F000914597500000E7806039134504088DB658
:10450000411122C497C501009385452E2A8417C501
:104510000100130525BA06C697A00100E780405A9E
:104520004C4017C501001305A54897A00100E7807E
:104530002059294597A00100E780605D03470400EA
:104540009307F00F631FF70297C501009385052AB3
:1045500017C50100130505B697A00100E780405676
:104560004C4017C501001305A54597A00100E78041
:1045700020552244B2402945410117A3010067009C
:104580000359B240224441018280411122C426C213
:104590002A84AE8417C501001305C5B197C5010073
:1045A0009385852006C697A00100E780605117C556
:1045B00001001305E55097A00100E78060502945F0
:1045C00097A00100E780A05497C501009385C51D01
:1045D00097070020239087AA17C50100130585AD12
:1045E000054497070020239597A89707002023925A
:1045F00087A897170020239E971297A00100E780B5
:10460000204C9715002083D5C51217C5010013054E
:10461000A54B97A00100E780A04A294597A001007B
:10462000E780E04E971700202382870097F7FF1F4F
:10463000938787D8DC4717F5FF1F0345A52203D7CB
:104640000700C167FD17631EF700B7E7040003A367
:1046500087051306000A85452244B2409244410171
:104660000283B7E7040003A387051306001493052C
:104670000010DDB7B1C1411122C417C501001305F7
:1046800065A32E8497C501009385451106C697A0A2
:104690000100E780E042A28517C5010013058541AE
:1046A00097A00100E780C0412244B2402945410162
:1046B00017A301006700A3458280011122CC37E4D3
:1046C00004005C5C06CE354697C501009385C52382
:1046D00017D50100130545EC829711E917C50100B4
:1046E000130505A397A00100E780605501A097F787
:1046F000FF1F9387E7173EC4B7F5070085679387C9
:104700000780814617F6FF1F13060616E1051945B7
:104710003EC697E0FF1FE780C00C7C44194697F522
:10472000FF1F93856514170500201305E5968297F2
:10473000340017F6FF1F1306261397C50100938553
:10474000256817C501001305256997700000E780EB
:10475000A0992A841DCD97C501009385650C17C5C6
:1047600001001305259597A00100E7806035A2851B
:1047700017C501001305451A97A00100E7804034D2
:10478000294597A00100E7808038F2406244056126
:10479000828097E00000E780A0FF17C501001305A5
:1047A000A50E97600000E780E08D97A00000E780ED
:1047B000E05397600100E78060B817F5FF1F13050D
:1047C00025BC97600100E78000A117C50100130513
:1047D000A50C97600100E780E0B82A84976000008C
:1047E000E78020F497100100E78040909780010057
:1047F000E780602997700000E78000509760000014
:10480000E780206A97300100E780A05197C501003A
:104810009385050117C501001305C58919C897A01F
:104820000100E780E029A28517C5010013050511E5
:10483000A1B797A00100E780A02817C501001305C4
:10484000251297A00100E780A027294597A0010025
:10485000E780E02B97300100E780802D97F0000083
:10486000E780404C7DC18545370504009730000046
:10487000E780E09197C50100938585FA17C501008F
:104880001305458397A00100E780802317C5010029
:104890001305850E97A00100E7808022294597A087
:1048A0000100E780C02697F7FF1F938767A083D793
:1048B000070017170020231EF7E68547171700206B
:1048C0002306F7D697F7FF1F938707AFDC4703D779
:1048D0000700C167FD176316F70097F0FFFFE78039
:1048E000206497700000E78040CB1305C5149770D3
:1048F0000000E78040CB97200000E780E0A6171576
:104900000020035505E397500000E780A0CD054542
:1049100097500000E780800097500000E780E02576
:1049200097C501009385C5EF17B50100130585787C
:1049300097A00100E780C01817C501001305050600
:1049400097A00100E780C01725BD97C5010093859A
:1049500025ED17B501001305E57597A00100E78067
:10496000201617C501001305251797A00100E78041
:104970002015294597A00100E7806019014597504F
:104980000000E780A0F969BF411122C437E40400A8
:104990008327041A06C6829797500000E78040C814
:1049A0008327040817F5FFFF13054564829797F7DF
:1049B000FF1F2389A7EA17F5FF1F1305E59F9740FF
:1049C0000000E78060702244B240410117030000FC
:1049D0006700E3CEB7E70400FC471171A2DDCAD936
:1049E00086DFA6DBCED72E8432892E86AA8517F5E0
:1049F000FF1F13052574829717F7FF1F130787738F
:104A000083470700930680029387E70793F7F70F22
:104A1000E3ECF610BA898A0717B701001307C772CB
:104A2000BA979C43BA9782878D4797C501009385B3
:104A300065E117B501001305E567630FF40097A062
:104A40000100E780E00717C501001305659E97A0E8
:104A50000100E780E006BDA497A00100E7804006C2
:104A600017C501001305459E97A00100E78040058A
:104A7000294597A00100E7808009930720F8114697
:104A800097F5FF1F9385056B4A8517F7FF1F2303D3
:104A9000F76A97F7FF1FA380076A97F0FFFFE78089
:104AA000A0312A841DC997C501009385A5D917B5E2
:104AB00001001305256097A00100E7806000A28532
:104AC00017C501001305059C97A00100E78040FF72
:104AD000294597A00100E780800397C501009385D1
:104AE00065D617B501001305E55C97A00100E780C6
:104AF00020FD17C501001305259A97A00100E78046
:104B000020FC294597A00100E780600041659307DC
:104B100030FA054697F5FF1F9385C5617D1517F798
:104B2000FF1F2309F76097F0FFFFE780E0282A8442
:104B30001DC997C501009385E5D017B50100130580
:104B4000655797A00100E780A0F7A28517C501006F
:104B50001305459397A00100E78080F6294597A0AB
:104B60000100E780C0FAB7E70400BC4F05661306F2
:104B700006C8A14517F5FF1F0345C5CE8297FE5015
:104B80006E54DE544E59BE591161828091476303C1
:104B9000F40297C501009385E5CA17B50100130516
:104BA000655197A00100E780A0F117C5010013052A
:104BB000E59171BDB7E70400FC4F914517F5FF1F64
:104BC000034545CA829797C501009385A5C717B5C8
:104BD00001001305254E97A00100E78060EE17C580
:104BE00001001305659097A00100E78060ED29455D
:104BF00097A00100E780A0F197400000E780201A0D
:104C0000914535A485476303F40297C50100938558
:104C100065C317B501001305E54997A00100E780BA
:104C200020EA17C501001305A58D15B597F7FF1FDD
:104C300023922747B7E704000566BC4F130606C852
:104C4000C1450DBF8D476303F40297C501009385ED
:104C500065BF17B501001305E54597A00100E78082
:104C600020E617C501001305658BD5B3930740F8FF
:104C7000114697F5FF1F9385E54B4A8517F7FF1FF0
:104C8000230AF74A97F7FF1FA387074A97F0FFFF0A
:104C9000E78080122A84E30405EE97C5010093851E
:104CA00065BA17B501001305E54097A00100E7803C
:104CB00020E1A28517B501001305C57C97A001006E
:104CC000E78000E0294597A00100E78040E445BD6A
:104CD0009147E31CF4F6B7E70400FC4F930500028C
:104CE00017F5FF1F034505B8829797C50100938507
:104CF00065B517B501001305E53B97A00100E780F6
:104D000020DC17C501001305E582F1BD894763E387
:104D1000870297C501009385E5B217B50100130519
:104D2000653997A00100E780A0D917C501001305D8
:104D3000A58131BB97F4FF1F83C4E43F97F7FF1FA2
:104D400083C7573F97C501009385C5AFA20417B528
:104D5000010013052536DD8C97A00100E78040D6C1
:104D6000A28517B501001305657F97A00100E780B4
:104D700020D5C204294597A00100E78040D9C1840D
:104D80009305D4FF93960401C1824A8693F5F50FEB
:104D900017F5FF1F1305353A97200000E780E04222
:104DA000E35F90DC930750F817F7FF1F2304F738F1
:104DB00083C73900228697F5FF1F9385A53785079E
:104DC0004A8517F7FF1FA308F73697F0FFFFE78024
:104DD000A0FE2A84E30505DA97C50100938585A620
:104DE00017B501001305052D97A00100E78040CD00
:104DF000A28517C501001305E5CAC9B5894763E354
:104E0000870297C501009385E5A317B50100130537
:104E1000652A97A00100E780A0CA17B50100130515
:104E2000A57535B197400000E78060F7A28517F5BA
:104E3000FF1F1305253097500000E78020A581B3A0
:104E40008D476303F40297C501009385A59F17B5AD
:104E500001001305252697A00100E78060C617B55D
:104E6000010013052573E5B6B76602000146B77564
:104E70000200054597E0FF1FE780A096930760F8C2
:104E800017F7FF1F2308F72A97F7FF1FA385072AA5
:104E90009307000617F7FF1F2300F72A894717F724
:104EA000FF1FA30BF72897F7FF1F2388072897F703
:104EB000FF1FA3840728C14717F7FF1F2300F72808
:104EC000930720F917F7FF1FA30AF726314697F734
:104ED000FF1FA386A72697F5FF1F9385A5254A8563
:104EE00097F7FF1F238D072497F0FFFFE780C0ECA3
:104EF0002A84E30605C897C501009385A59417B5D4
:104F000001001305251B97A00100E78060BBA28567
:104F100017B501001305856955B3B1476303F40262
:104F200097C501009385059217B5010013058518F3
:104F300097A00100E780C0B817B501001305C56848
:104F400039B6B7E70400FC4F9305000417F5FF1FBF
:104F500003454591829797400000E78040E4B145C2
:104F6000F9B5914763E3870297C501009385858D65
:104F700017B501001305051497A00100E78040B4A0
:104F800017B5010013050566D9B497F4FF1F83C454
:104F9000A41A97F7FF1F83C7171AA204DD8C8E048B
:104FA000B77702006D14BE942286A68517B501005E
:104FB0001305856497A00100E78080B0B7E704007F
:104FC000FC47228697F5FF1F9385151728008297C7
:104FD00093160401C1823000A685094597E0FF1FA2
:104FE000E78020802A8409C917B50100130585626E
:104FF00097A00100E780A0C4930770F8194697F5C1
:10500000FF1F938525134A8517F7FF1F2304F71207
:1050100097F7FF1FA382871297F0FFFFE780C0D9A1
:105020002A84E30E05B497C501009385A58117B5C1
:1050300001001305250897A00100E78060A8A2855C
:1050400017B501001305055E95B99947630BF41276
:1050500097B501009385057F17B5010013058505F8
:1050600097A00100E780C0A517B501001305055DF5
:10507000F9BA914763E3870297B501009385857C70
:1050800017B501001305050397A00100E78040A3B1
:1050900017B501001305055C5DBA97F4FF1F83C4C3
:1050A000A40997F7FF1F83C71709A204DD8C8E049C
:1050B000B77702006D14BE942286A68517B501004D
:1050C0001305855A97A00100E780809FB7E7040089
:1050D000FC47228697F5FF1F9385150628008297C7
:1050E00093160401C1823000A6850D4597D0FF1F9D
:1050F000E780206F2A8409C917B501001305855878
:1051000097A00100E780A0B3930780F8194697F5B0
:10511000FF1F938525024A8517F7FF1F230CF70011
:1051200097F7FF1FA38A870097F0FFFFE780C0C8AB
:105130002A84E30605A497B501009385A57017B5E9
:105140000100130525F797A00100E7806097A2856D
:1051500017B501001305455495B699476303F4024A
:1051600097B501009385056E17B50100130585F409
:1051700097A00100E780C09417B5010013054553BF
:10518000F9B0B7E70400FC4F9305000417E5FF1FD3
:105190000345456D829797400000E78040C09945E0
:1051A00079B18D476303F40297B501009385856952
:1051B00017B50100130505F097A00100E7804090A6
:1051C00017B501001305455059B017B50100130577
:1051D000A55097A00100E78080A61305C01297D0C4
:1051E000FF1FE7800016014597E0FFFFE780C0EA58
:1051F0000D4597100000E780C0A6294597D0FF1FF6
:10520000E780201497D0FF1FE78080048DBA99476C
:105210006303F40297B501009385C56217B50100D9
:10522000130545E997A00100E780808917B50100C3
:105230001305454B29B817F7FF1F0347F7EF97F7FB
:10524000FF1F83C767EF22075D8F9166BA96C2067C
:105250001166C1821306F6EF8D476365D60297E7A4
:10526000FF1F938767159C4B17F6FF1F0346B6EC8D
:105270009386C7002DC203D6070069CA8907E39C3D
:10528000D7FE89471307A0F8114697F5FF1F9385AE
:1052900065EA4A8597F6FF1F238EE6E817F7FF1F9A
:1052A000A30BF7E897F0FFFFE78000B12A84E3083B
:1052B000058C97B501009385E55817B501001305D6
:1052C00065DF97900100E780A07FA28517B50100F8
:1052D00013058542E5B203D60700630EE60A890787
:1052E000E39BF6FE8D4779BF91476304F40297B5BF
:1052F00001009385255517B501001305A5DB97908F
:105300000100E780E07B17B50100130565406FF0F1
:105310000FF4B7E70400FC4F9305000817E5FF1FE3
:10532000034545548297C9B897B5010093858551C7
:1053300017B50100130505D897900100E780407864
:1053400017B501001305453E6FF06FF02390E7009D
:1053500017E5FF1F1305450697300100E780C0A23F
:1053600097B501009385054E17B50100130585D447
:1053700097900100E780C07417B501001305C53B85
:1053800097900100E780C073294597900100E7805E
:1053900000788147C5BD2390070017E5FF1F13055F
:1053A000A50197300100E780209E97B50100938505
:1053B000654917B501001305E5CF97900100E78017
:1053C000207017B501001305A5385DBF411122C437
:1053D00006C6834705002A849DC797B501009385BB
:1053E000254217B501001305E5CC97900100E78031
:1053F000206D4C4017B50100130505719790010011
:10540000E780006CE1A05841B707CF009387777D14
:10541000631DF70697B501009385853E17B501001A
:10542000130545C997900100E78080691C448356A5
:10543000E4008355C40003C6070017B50100130537
:10544000256E97900100E780A0672945979001009D
:10545000E780E06B0357E4009707002083D7672DB0
:105460006309F7008355C400084497E0FFFFE78015
:1054700020D70356E4008355C40008442244B240B8
:10548000410117F3FFFF67002355B707CC0093874F
:10549000777D6315F70497B501009385653617B5D9
:1054A0000100130525C197900100E78060611C444D
:1054B0008356E4008355C40003C6070017B50100F6
:1054C0001305056697900100E780805F2244B24093
:1054D000294541011793010067006363B707CE00B8
:1054E0009387777D6304F70297B501009385453173
:1054F00017B50100130505BC97900100E780405CDB
:105500004C4017B501001305E556CDBDB24022440D
:1055100041018280B7E70400FC4741112E8606C690
:1055200022C426C24AC02E842A89AA8517F5FF1FE5
:10553000130545C0829797B501009385653217B56D
:105540000100130525B797900100E780605797F594
:10555000FF1F83C525BE17B50100130565D89790B9
:105560000100E780E055294597900100E780205A27
:1055700097F4FF1F938404BC83C7040041479387BB
:10558000070693F7F70F636EF75A17B70100130773
:10559000E7C58A07BA979C43BA9782879D476307F6
:1055A000F40297B501009385A52B17B501001305EB
:1055B00065B097900100E780A05017B50100130572
:1055C000A5D297900100E780A04F8DA497F7FF1F09
:1055D00083C757B6DDCB17F7FF1F0347D7B597F73C
:1055E000FF1F83C747B522075D8F97F7FF1F83C74C
:1055F000A7B4C2075D8F97F7FF1F83C7F7B3E20712
:10560000D98F17F7FF1F2325F7B083C7640097B51D
:1056100001009385E52417B501001305A5A917F727
:10562000FF1F2306F7AE97900100E780604997F7C8
:10563000FF1F9387E7AD8C4317F6FF1F034626AD88
:1056400017B50100130505CC97900100E78040478E
:10565000294597900100E780804B97F7FF1FA38BA8
:1056600007AC2244B24092440249930700F817F76E
:10567000FF1F2301F7AC9D4517F5FF1F130585ABF1
:105680004101174300006700632097600000E78036
:1056900000F097F7FF1F2380A7AA9357850017F7FD
:1056A000FF1FA30AF7A8935705012A8417F7FF1FC6
:1056B0002304F7A893578501014517F7FF1FA30D92
:1056C000F7A697600000E780E0F097F7FF1F2386BA
:1056D000A7A697B501009385A51817B50100130576
:1056E000659D97900100E780A03D17F6FF1F0346D8
:1056F000C6A4A28517B50100130545C2B1B7CD47B1
:105700006303F40297B501009385851517B5010071
:105710001305459A97900100E780803A17B501007C
:10572000130545C179BD37E404007C44414697F533
:10573000FF1F938535A017F5FF1F1305A59D8297C1
:1057400097F7FF1F83C727A017F7FF1F0347979FF0
:10575000A20703238405D98F17F7FF1F2318F79A91
:105760001306000A89452244B2409244024917E5D3
:10577000FF1F0345250F410102838D476303F40298
:1057800097B501009385C50D17B5010013058592E6
:1057900097900100E780C03217B50100130545C995
:1057A0000DB517F4FF1F0344049997F7FF1F83C734
:1057B000779897B501009385A50A220417B50100D3
:1057C0001305458F5D8C97900100E780602FA285BF
:1057D00017B50100130585B797900100E780402EAB
:1057E000294597900100E78080320D4697F5FF1F0D
:1057F00093854594228597E0FFFFE780E05BAA84CC
:1058000021C197B501009385A50517B501001305C2
:10581000658A97900100E780A02AA68517B5010048
:10582000130505B497900100E78080292244B24017
:105830009244024929454101179301006700232D35
:1058400097F7FF1F23988784B7E70400116603A327
:105850008705130606E8914539B78D476303F402BF
:1058600097B501009385C5FF17B501001305858421
:1058700097900100E780C02417B50100130505CA01
:1058800089B317F4FF1F0344048B97F7FF1F83C7E7
:10589000778A97B501009385A5FC220417B501000E
:1058A000130545815D8C97900100E7806021A285FA
:1058B00017B50100130505AC97900100E780402063
:1058C000294597900100E78080240D4697F5FF1F3A
:1058D00093854586228597E0FFFFE780E04DAA8407
:1058E0001DC197B501009385A5F717A50100130504
:1058F000657C97900100E780A01CA68517B5010084
:10590000130585A805B797E7FF1F23978776B7E7A5
:105910000400116603A38705130606E89305000239
:1059200099B5894763E3870297B50100938545F3ED
:1059300017A501001305057897900100E78040182E
:1059400017B50100130545C0ADB997E4FF1F83C427
:10595000847E97E7FF1F83C7F77D97B50100938586
:1059600025F0A20417A501001305C574DD8C9790DE
:105970000100E780E014A68517B50100130545A2D4
:1059800097900100E780C013294597900100E780B8
:105990000018228697E5FF1F9385C579268597E035
:1059A000FFFFE78060412A84630E051A97B5010066
:1059B000938505EB17A501001305C56F97900100AE
:1059C000E7800010A28517B501001305A59E99BDBB
:1059D000854763F98718834519002244B2409244F1
:1059E0000249B335B00097E7FF1F238FB76A17B599
:1059F00001001305659D4101179301006700430CE9
:105A0000A2852244B24092444A85024941011703CB
:105A100000006700432B99476303F40297B5010028
:105A2000938505E417A501001305C568979001004B
:105A3000E780000917B501001305C5CA59B617E478
:105A4000FF1F0344446F97E7FF1F83C7B76E97B5E7
:105A500001009385E5E0220417A501001305856583
:105A60005D8C97900100E780A005A28517B5010025
:105A70001305059797900100E780800429459790CA
:105A80000100E780C008194697E5FF1F9385856AE6
:105A9000228597E0FFFFE7802032AA841DC197B5D9
:105AA00001009385E5DB17A501001305A56097901C
:105AB0000100E780E000A68517B5010013054593B6
:105AC00095B397E7FF1F239F8764B7E7040011662C
:105AD00003A38705130606E89305000869B1854707
:105AE00097B501009385C5D717A501001305855CFF
:105AF000630BF40097900100E78080FC17B501006C
:105B0000130545907DBC97900100E78060FB17B5B9
:105B100001001305A59097900100E78060FA2945E0
:105B200097900100E780A0FE2244B24092440249CF
:105B300097E7FF1F239C075C410117630000670084
:105B4000839597B501009385A5D117A5010013058D
:105B5000655697900100E780A0F617B50100130580
:105B6000A5BC85B4B24022449244024941018280DE
:105B7000411106C622C426C239C12A8497E000001A
:105B8000E780401AAA8411EDB7E70400BC474146FC
:105B9000814522858297B240224426859244410164
:105BA000828041657D1597E00000E7808018B7E7A7
:105BB000040001E9BC474146814522858297814422
:105BC000D9BF0347E501FC479305900819E3930506
:105BD0000003AA9541462285829785446DBF4111F5
:105BE00006C622C497E0FFFFE780001D21CD97E79E
:105BF000FF1F83D7874B85072A8417E7FF1F2316CC
:105C0000F74A97B50100938525C797E7FF1F239FA4
:105C1000A74817A501001305E54997900100E78003
:105C200020EAA28517B501001305C5E7979001008A
:105C3000E78000E92244B240294541011793010061
:105C40006700E3EC97E7FF1F83D76746B240224423
:105C5000850717E7FF1F231CF7444101828041118C
:105C600022C491462A8417E6FF1F1306A65A9D6593
:105C70002D4506C697D0FF1FE780A0B6B7F70700EF
:105C800003C70701A5476313F70001A0930600109F
:105C900001469D65254597D0FF1FE78080B497E7B3
:105CA000FF1F238987562244B240914617E6FF1F03
:105CB000130646569D652945410117D3FF1F67000E
:105CC00043B21171CED7B7E9040083A7C904CAD97A
:105CD00017E9FF1F13090946A2DD2E8686DFA6DB22
:105CE0002E84AA854A85829797E7FF1F83C787443A
:105CF0001307700A6385E710636DF7001307600AE6
:105D00006385E704FE506E54DE544E59BE5911614E
:105D100082801307800A6385E7161307900AE393CE
:105D2000E7FE8D476306F41C97B501009385C5EA2D
:105D300017A501001305053897900100E78040D8AA
:105D400017B50100130585E625A08D47630CF40205
:105D500097B50100938545E817A501001305853522
:105D600097900100E780C0D517B50100130545DD08
:105D700097900100E780C0D4294597900100E78003
:105D800000D949B7854717B50100130525DD17E789
:105D9000FF1F230BF73097900100E78040EAB775AB
:105DA0000200B76602000146054597D0FF1FE78055
:105DB00040A3930760F817E7FF1F230DF73697E717
:105DC000FF1FA38A07369307002617E7FF1F232527
:105DD000F736E5779387072117E7FF1F2310F7367C
:105DE000B14597E7FF1F238C073497E7FF1FA38870
:105DF000A7344A8597000000E780E01621B7914755
:105E000063E3870297B50100938505DD17A50100BF
:105E10001305452A97900100E78080CA17B5010055
:105E20001305C5D5B1B797E4FF1F83C4E43097E7E6
:105E3000FF1F83C75730A204DD8C83A7C9046D14EC
:105E4000228697E5FF1F9385352F280082978E04C1
:105E500093160401B7750200C1823000A69509456A
:105E600097D0FF1FE780E097930770F817E7FF1FB1
:105E70002302F72C994597E7FF1FA38FA72A95BF09
:105E8000914763E3870297B501009385E5D417A591
:105E900001001305252297900100E78060C217B525
:105EA0000100130525CFE9B597E4FF1F83C4C4287B
:105EB00097E7FF1F83C73728A204DD8C83A7C90497
:105EC0006D14228697E5FF1F93851527280082977A
:105ED0008E0493160401B7750200C1823000A695A6
:105EE0000D4597D0FF1FE780C08F930780F8BDBF97
:105EF00017B501001305C5CC97900100E78020D4A9
:105F0000930790F82304F100834719008D4528007A
:105F1000A304F100834729002305F1009700000046
:105F2000E78060041305C01297C0FF1FE78060413F
:105F3000014597D0FFFFE78020160D459700000030
:105F4000E78020D2294597C0FF1FE780803F97C098
:105F5000FF1FE780E02F7DB397E7FF1F23A4A72C47
:105F6000828097E7FF1F9387E72B03A30700630354
:105F700003000283174300006700439141114AC0A8
:105F800097F6FF1F83D6E67A328917D6FF1F03568E
:105F9000C64422C426C206C62A84AE8497000000E6
:105FA000E780405435C12DC0994763FF970483476C
:105FB000140003470400A207D98F13978700A18319
:105FC000D98FC2073167C1831307C755639EE702A4
:105FD00097D7FF1F83D76740A301F400A183230253
:105FE000F40097F7FF1F83D7C77491C7A302F4008B
:105FF000A1832303F400A68517B501001305C5C1CD
:1060000097900100E780C0AB97F7FF1F83C7076237
:10601000A5C797D5FF1F83D5453C17B501001305CC
:1060200065C197900100E780A0A92686A28517D5B3
:10603000FF1F0355853A97000000E78080BA63068A
:10604000090497F7FF1F83C7675EA1E397E7FF1F68
:1060500083C7871D9DCB95C897E7FF1F83C7C704DC
:106060008DE722852244B2400249A685924441012F
:10607000174300006700838117B50100130585BC35
:1060800097900100E780A0BB5DBFB24022449244DC
:10609000024941018280834755008345450017B579
:1060A0000100130525B6A207DD8D179301006700D7
:1060B00023A117B501001305E5B31793010067008D
:1060C00003B88D4763F6B708011126CA06CE22CC65
:1060D0000344350097E4FF1F83C4141597B50100EE
:1060E000938505B7B337800017E7FF1FA30EF7129C
:1060F00009C497B50100938565B617B5010013056E
:1061000065B697900100E780A09B97E7FF1F83C7C4
:10611000B7116386970097000000E780A02C974096
:106120000000E78080A59967938757EE2316F1005A
:10613000680085479145A30781002307F100970078
:106140000000E78040E2F2406244D2440561828070
:106150008280894763F7B708011122CC06CE26CA90
:106160008344250085472A84639DF404914763F5A1
:10617000B704034545008347340022055D8D97D75A
:10618000FF1F239CA72497000000E780803E9967AB
:10619000938767EE2314F1008347340023059100B1
:1061A000A305F10083474400954528002306F1002C
:1061B00097000000E78020DBF2406244D244056192
:1061C0008280FDF89967938767EE2314F10097D7D3
:1061D000FF1F83D78720A305F10023050100A183BA
:1061E000E1B782800111996722CCD51717F4FF1F00
:1061F0001304C4432314F1008347040026CA97F410
:10620000FF1F938404532305F10083D70400280063
:106210009545A305F100A18306CE2306F100970062
:106220000000E78040D403D604008345040017B57E
:106230000100130525A497900100E7806088F240D3
:106240006244D244056182809D677971D917231613
:10625000F10097F7FF1F9387673D83C7070013057A
:10626000F10006D62307F10097000000E780809038
:1062700009E9B7E70400BC47414681451305F10031
:1062800082976800CD4597000000E780C0CD97F564
:10629000FF1F83C5A53917B501001305A5A0979069
:1062A0000100E780E081B250456182805DC9411103
:1062B00022C426C206C6930750FA2300F5009307AE
:1062C000A005A300F50089472301F5009147A3012C
:1062D000F5009307C003A302F50097F7FF1F93870C
:1062E000E73483C707009304C5002A842303F5001D
:1062F00097E7FF1F938757F383C707002302050023
:10630000A303F50097F7FF1F83D7A7422304F500E7
:10631000A183A304F50097D7FF1F83D7070C23059C
:10632000F500A183A305F500268597000000E7800E
:10633000608401E9B7E70400BC47414681452685F2
:1063400082972285F14597000000E780A015230E73
:10635000A4002181A30EA400B24022449244410132
:10636000828082805D710A8586C6A2C49700000083
:10637000E78000F437E404007C448A8508107946FD
:1063800082973C441305E10309468145829710102A
:1063900093050002014597D0FFFFE7802036B64005
:1063A000264461618280411122C426C24AC02A84E7
:1063B000AE843289AA8585660146254506C697C002
:1063C000FF1FE7800042A2852244B240CA8626868B
:1063D000024992442945410117C3FF1F67006340EA
:1063E0000111B7C7A55A22CC9387C73317E4FF1F03
:1063F000130494E33EC4834704002C00214619652E
:1064000006CE3EC697000000E78020FA83450400D0
:1064100017B501001305859397800100E780406A56
:10642000F2406244056182800111A1463000996505
:106430002D4522CC06CE97C0FF1FE780803AA247A9
:1064400037C4A55A1304C43363958702B24517B500
:10645000010013056587B335B00097E7FF1FA385DB
:10646000B7DC97800100E780A065F24062440561D7
:1064700082809165A1463000938505F02D4597C037
:10648000FF1FE7800036A247E38287FC97E7FF1FE4
:10649000A38C07D8814517B5010013052585D1B711
:1064A000C16769768146FD1705061397060141838A
:1064B0006364B7003E8582803307D5000347070039
:1064C000B98F214713F81700858363050800B18F42
:1064D000C207C1837D171377F70F6DF78506F1B7F4
:1064E00041C5A547054763F2B70883471500034731
:1064F00005003168A207D98F13978700A183D98F30
:10650000C207C1831308C8550547639007074111A7
:1065100006C622C426C203442500914763F08704BF
:106520009307540063ECF502A301C5002182230206
:10653000C5009304340091C6A302D500A1822303B1
:10654000D5002A84A68597000000E780A0F5269450
:106550002300A4002181A300A4000147B2402244EB
:1065600092443A854101828005473A858280011133
:10657000B7C7A55A22CC9387E7342A842AC6214676
:106580002C00156506CE3EC497000000E780E0E1D0
:10659000A28517A501001305657D97800100E7809E
:1065A000205297000000E78020DCF2406244056141
:1065B00082800111A146300095652D4522CC06CE82
:1065C00097C0FF1FE780E021A24737C4A55A1304F4
:1065D000E43463958702B24517A5010013050573DE
:1065E00097D7FF1F239BB7DEC205C18197800100AB
:1065F000E780004DF2406244056182809165A146CA
:106600003000938505EE2D4597C0FF1FE780601D84
:10661000A247E38287FCD14717D7FF1F231FF7DA72
:10662000D14517A5010013056570C9B721C14111F6
:1066300026C206C622C4AE848DC52A8497000000F7
:10664000E780806697E7FF1F83C707BE99CB228547
:106650002244B240A68592444101173300006700EE
:10666000E322B2402244924441018280828001119F
:106670004AC806CE22CC26CA4EC693F715002E89EC
:106680009DCBAD67371700409387A7AA1CC3B7E718
:106690000400BC4F13060019854517D5FF1F03459D
:1066A000A5D3829713451900F2406244D24442496F
:1066B000B2490561828093F72500638A071C17F7AA
:1066C000FF1F0357E706954763F9E70C014417F6E8
:1066D000FF1F1306E6F59306300513055004130853
:1066E00010049308B00413039005930764006374C7
:1066F000F7043A84FD5997F4FF1F83C464F397F7B6
:10670000FF1F83C7F7F2A204DD8CAD679387B755EF
:10671000638BF41463E3970AA9679387A755638E85
:10672000F414A28517F5FF1F130585F097000000EC
:10673000E78000F031A2B307860083C50700639AA3
:10674000D50483C517006396A50483C5270063920B
:10675000050583C53700639ED50283C54700639A4C
:10676000150383C7570063966702A2890DE897F562
:10677000FF1F83D5E5FBB3853541C20517F5FF1F24
:10678000130505EBC1814E9597000000E78040EAB4
:10679000E1A005044204418089BF3A84FD59854740
:1067A000E3EB87F45DC4854517F5FF1F130545E846
:1067B00097000000E780C0E769A8B1679387C755D5
:1067C0006380F404B5679387D755E39CF4F4A285FE
:1067D00017F5FF1F1305C5E597300000E780000B94
:1067E0008947630FF4049305E4FFC205C18117F5DF
:1067F000FF1F130505E497000000E780E04A89A029
:1068000097200000E78060F797000000E7802049AC
:1068100011C9A28517F5FF1F130585E19700000038
:10682000E78080480546A28517F5FF1F130545E060
:1068300097F0FFFFE780C07497200000E780E0F347
:10684000A68517A501001305255497800100E78050
:106850002027FD57E39DF9F097F7FF1F239A07ECD8
:106860001345290091B5A28517F5FF1F130545DCD7
:1068700097000000E7806082E1B7A28517F5FF1F4F
:10688000130505DB97000000E780E08255BF93F712
:1068900045000145E38A07E017A5010013050550EF
:1068A00097800100E780A03997300000E780A02B97
:1068B00013454900D5BB411122C437E404005C5C98
:1068C00006C6354697A501009385050417B5010056
:1068D000130585CC829711E917A501001305C54C56
:1068E00097800100E780A03501A08327041C8297D0
:1068F0002A84054597C00000E780E0E89760010022
:10690000E780006E97600100E780004397B00000C9
:10691000E78060FA2285B240224441018280411121
:10692000054506C622C426C297C0FFFFE780A060C7
:106930001305A00497B0FF1FE78060777575854544
:106940007D1597C0FFFFE780404A7D75854513059B
:10695000F53697C0FFFFE780A05337140040832728
:10696000840A8D451305002093E707202324F40AA9
:1069700097C0FFFFE7806047B7E4040097D0FFFFB0
:10698000E780808CC85897800100E780402B17B5BE
:106990000100130565C097800100E780402A832726
:1069A000840C8545414593E707082324F40C97C0E0
:1069B000FFFFE780E04D8D451305000897C0FFFFFE
:1069C000E780004D97C0FFFFE780E07937A507001B
:1069D0001305051297C0FFFFE7808075014597C03A
:1069E000FFFFE780A07B95450545894717F7FF1F07
:1069F0002302F7D497C0FFFFE780E07BB7E700E012
:106A000013070006238DE7403707000423A0E71093
:106A100097D0FFFFE78060FD97D0FFFFE780600F12
:106A200097000000E78060E997000000E78000A081
:106A300097000000E78020B897E0FFFFE78000F5AF
:106A400097000000E780802797000000E780801013
:106A500083A70408170500001305A5C1829797D7DF
:106A6000FF1F238BA796BC4C1306006485458297B5
:106A700097C0FF1FE780C09701458280AD67371739
:106A800000409387A7AA1CC3B7E700E03707400080
:106A900023A0E71801000100B7F7070003C70701AB
:106AA000A5476316F7009397450191C301A04111D3
:106AB000AE860146AA85254506C697C0FF1FE7801A
:106AC00040D2B240B7E700E03707400023A0E7100C
:106AD000410182804111B2862E86AA852D4506C6C7
:106AE00097C0FF1FE780E0CFB2400145410182809F
:106AF0009307000463ECC7041D71A2CC2A84080824
:106B0000A6CACAC886CE32C697800100E780E0EFE9
:106B1000AD67371700409387A7AA1CC3B7E400E00E
:106B20003709400023A0241901000100B2461008D3
:106B3000A285294597C0FF1FE780A0CAF64066449A
:106B400023A02411D644464925618280395582808C
:106B500041110D658D4506C697C0FFFFE780E0280F
:106B6000B71700408D6623A6D70A17F5FF1F130538
:106B7000A5BC1387C70A9387870A1CC15CC58566B5
:106B800089675CC958C114C518C9B7E70400B24089
:106B900003A3871E410102838145B307B5008387A4
:106BA000070089E7172300006700C3C38505C205F6
:106BB000C181E5B797A70100938707391357C5002F
:106BC0003E9703470700011106CE2304E100135747
:106BD00085003D8B3E970347070023060100A30471
:106BE000E100135745003D8B3D893E97AA97034727
:106BF000070083C7070028002305E100A305F10073
:106C000097000000E78080F9F24005618280411121
:106C100026C2E97797F4FF1F938484C222C4938726
:106C2000A7552E842381B4002E86AA8517F5FF1F51
:106C3000130545C106C62390F400A3810400978084
:106C40000100E78080DC93052400C205C18117F5AF
:106C5000FF1F130505BF97000000E780A084B387DE
:106C600084002382A7002181A382A70093056400EA
:106C70002244B24026859244C205C18141011723B6
:106C80000000670023B609C99307800263E6B700D6
:106C9000170300006700E3F7828017F5FF1F034525
:106CA00025AB828097F7FF1F83C747B989E7172372
:106CB0000000670023B3828097F7FF1F83C727BBBD
:106CC00099EF411106C697200000E78080A9B240E5
:106CD000854717F7FF1F230CF7B841018280828098
:106CE0006304054A6382054A5D71CAC04EDE86C6EA
:106CF000A2C4A6C252DC56DA5AD85ED662D466D294
:106D00006AD0B9472A89AE8963F9B706394697A58B
:106D100001009385251197800100E780A0CC31ED1B
:106D20008347E900130710036394E702854717F7C9
:106D3000FF1F2305F7B017A501001305A50F97F74F
:106D4000FF1F239C07AE97000000E78020E571A09D
:106D50001307000317A501001305C510E395E7FE0F
:106D600097F7FF1F238C07AC97F7FF1F239707ACFC
:106D700017A501001305850DF9B797F7FF1F83C706
:106D8000E7AB63870722BD6AB96B938CFA55014A5A
:106D900017FBFF1F130B0B9C138CEB65938AFA6692
:106DA00005A8B307490183C6070097F7FF1F83D7DC
:106DB000C7A8B1E39307A005639BF600854717F7C3
:106DC000FF1F231CF7A697F7FF1F2385D798050AF7
:106DD00093170A01C183E3E637FDB6402644964483
:106DE0000649F259625AD25A425BB25B225C925C0B
:106DF000025D61618280054D639BA7039307500A82
:106E0000639EF600894717F7FF1F2318F7A2930721
:106E100050FA17F7FF1FA30FF79255BF9307A0056E
:106E2000E387F6FA97F7FF1F239907A04DB713875B
:106E300017004207DA9741832380D70017F6FF1F18
:106E4000231DE69E8D47E3F4E7F817F4FF1F034484
:106E5000949097F7FF1F83C7079022045D8C9307D8
:106E6000F4FFC207C1839306F00DE3EDF6FA930732
:106E70006400C207C183E31CF7F493052400C20534
:106E8000C18117F5FF1F1305058D97F0FFFFE78000
:106E9000606133078B008347570003474700A20711
:106EA000D98F17F7FF1F231A07986318F50E81442F
:106EB000630CA40197F4FF1F83C4048AA20497F70C
:106EC000FF1F83C77789DD8C170500001305E5DBFD
:106ED00097F0FFFFE780800863878407636D9C025B
:106EE0009387EB556382F40497F7FF1F83C7C78628
:106EF00005476389E70681CB1387A7051377F70F4B
:106F00008D4663F2E6081307F0072300E100A300B3
:106F1000F10089459DA063829405E39754FD97F0A5
:106F2000FFFFE780A03211A8A28517F5FF1F130508
:106F3000A58297F0FFFFE7800019014597F0FFFF5A
:106F4000E780C00169B5A28517F5FF1F1305C5804D
:106F500097F0FFFFE7802020CDB797F0FFFFE78095
:106F6000A028E1BF930710F8130511002300F100DA
:106F700097F0FFFFE780C033FD450A8597000000CA
:106F8000E78020C95DBFA28517E5FF1F1305C57CFB
:106F900097F0FFFFE78020D34DB79307F0078945AF
:106FA0000A852310F10097000000E78080C605B530
:106FB000BD4763F53717414697A501009385C5EC9A
:106FC0004A8597800100E780E0A16319051417A5A1
:106FD00001001305A5EC97000000E78020BC17E531
:106FE000FF1F0355057597000000E780E0BC97E799
:106FF000FF1F83C7A76317A501001305A5E189E754
:1070000017A50100130585E197000000E78000B98E
:1070100017A50100130505EA97000000E78000B8F6
:1070200017C5FF1F0355053997000000E780C0B85A
:1070300017A50100130545E897000000E78000B69A
:1070400017C5FF1F0355653997000000E780C0B6DC
:1070500017A501001305C5E697000000E78000B4FE
:1070600017D5FF1F0355A50497000000E780C0B4A3
:1070700017A50100130545E597000000E78000B261
:1070800017D5FF1F0355650297000000E780C0B2C7
:1070900017A501001305C5E397000000E78000B0C5
:1070A00017D5FF1F0355850097000000E780C0B08B
:1070B00017A50100130505E297000000E78000AE68
:1070C00017C5FF1F0355C51F97000000E780C0AE1E
:1070D00017A50100130585E097000000E78000ACCC
:1070E0000A8597F0FFFFE780E0A88347010003458A
:1070F0001100A2075D8D97000000E780E0AB834799
:10710000210003453100A2075D8D97000000E78054
:10711000A0AA179501001305A55635B1C14763FE16
:107120003705414697A50100938585DB4A85978001
:107130000100E780208B31E1834709011307100329
:10714000639CE700854717E7FF1F2303F76017A538
:107150000100130525DAC5BE1307000317A50100BA
:10716000130545DCE391E7BE97E7FF1F2382075E27
:1071700017A50100130585D9F9B6CE854A8597C0B4
:10718000FFFFE780E00591B98280411126C2AE84FD
:107190008D4522C406C62A8497C0FFFFE78040CFF2
:1071A000B717004099C803A5C70C418D23A6A70CAB
:1071B000B240224492444101828003A5870C418D54
:1071C00023A4A70CF5B78347050003471500A207C2
:1071D000D98FC2076177C18713072720639AE70019
:1071E000834525003705040017030000670023FAD4
:1071F000828017E6FF1F1306E6678147B2861303F6
:10720000F00FA9483308F6000348080013F7F70FFA
:107210006307A80C630668008507E39517FF2947F5
:10722000B387E6002380A70097E7FF1F9387476592
:107230005DA8411113D765001347170006C693F6E2
:107240003500058B954791CA054699476387C60067
:1072500009469D476383C600A14713F645003336B0
:10726000C00093F68503050685C2A145638BB6046D
:10727000E145638AB604930580026388B6049305EA
:1072800080036393B600914697F5FF1F238FF58423
:1072900097F5FF1F238AC58497F5FF1FA386D58422
:1072A000BE8517A50100130525CE97800100E78054
:1072B0002081B240854717F7FF1FA308F7824101DD
:1072C00082808546D1B78946C1B78D4675BF17A55F
:1072D00001001305E5CD177301006700637E17E712
:1072E000FF1F1307E759BA972380B700E147E3026E
:1072F000F5F493077002E30CF5FC82802A87238063
:107300000500814717E5FF1F1305C5561308F00F49
:107310002946B306F50083C606006396E60297E6A3
:10732000FF1F9386E655B69783C707000545238060
:10733000F5009947636EF7029D4763FDE700E1475B
:10734000630DF7008280638506018507E393C7FC20
:107350000145C5B7238005008280B737004003C7C9
:10736000370083C7050093F70704D98F2380F50002
:1073700082805D7152DC56DA5ED6716A97FBFF1F20
:10738000938BCB878D6AA6C24EDE62D486C6A2C41A
:10739000CAC05AD866D26AD06ECEC1495E8C97E414
:1073A000FF1F9384A44E130A0A20938A7ADC17F9EC
:1073B000FF1F0349A987B3872B0183C7070093F7F2
:1073C000F70FC9EFB787004003C76700058BE310CD
:1073D000077C03C76700118BE30D077E83C7570047
:1073E000918B99E36F10200317F7FF1F0347278442
:1073F00085476304F7006F10400197E7FF1FA386DE
:10740000E76E97E7FF1F2383075497E7FF1F23814A
:10741000076097E7FF1F238F076A97E7FF1F238CFB
:10742000076A97E7FF1FA383075297E7FF1FA38110
:10743000075E97E7FF1FA38F076897E7FF1FA38CDF
:10744000076897E7FF1FA383076A97E7FF1FA380DB
:10745000077EB787004011476F00707793071900C8
:1074600093F7F70F3D476364F70617E7FF1F230FF6
:10747000F77A97E7FF1F9387677ACA9783C7070052
:107480001307100293F7F703638EE71E6366F70492
:1074900005446385871CE38C07620947638EE71008
:1074A00013070002E384E74EB7E700E03707400028
:1074B00023A0E71801000100629923000900FD19CB
:1074C00023A0E71093F9F90FE39309EEE5BD97E7E1
:1074D000FF1F238D077471BF130730026388E70C09
:1074E00063E8E71613074002638CE70A13070003FB
:1074F000E39CE7FA97E7FF1F93874771CA9703C793
:107500000700A1471377F70FE31BF71483C7640045
:1075100097E6FF1F2382F65C97E7FF1F83C7773745
:1075200091C7FD5797E6FF1F2388F65A97E5FF1F7F
:1075300083C5D53597E7FF1FA380B75A97E7FF1F8D
:1075400083C7C73413FB07089306000493F70706A5
:10755000639FD74C9307A009638DF51663EAB712B2
:107560009307F0056386F54A930750096384F52A6B
:10757000014497E7FF1F83C737561547E392E73665
:10758000B7E700E03707400023A0E718010001003B
:10759000B786004023808602130680FC6F00500EE1
:1075A000FD5717E7FF1F2308F752FDBDFD5717E7EB
:1075B000FF1F2301F752CDBD17A501001305C5B06C
:1075C00097700100E780A06797E7FF1F9387076424
:1075D000CA9703C40700014B97ECFF1F938C8C43A1
:1075E0001374F40F17AD0100130D8DAE63478B04B8
:1075F000294597700100E7808051854717E7FF1FF5
:10760000A308F74017E7FF1F2305874017E7FF1F71
:10761000230EF74C37E700E0B70640002320D718C9
:1076200001000100378600408347A60293F7370F19
:107630002305F6022320D71085BDB3876C0183C5CF
:1076400007006A85050B97700100E780604779BFE6
:10765000854717E7FF1F230DF73AB9B517E7FF1F57
:107660001307C75A4A970347070097E6FF1FA38FE0
:10767000F62C97E6FF1F238CE62C17E7FF1F230746
:10768000F7461DB5854717E7FF1F2301F72C29BDD6
:107690009307400A6389F5349307200B6384F5361A
:1076A0009307100AE396F5EC838724000144E3D2A4
:1076B00007EC97E7FF1F83C7971D93F63700638A90
:1076C000061A0546638AC62209466395C61A1D47EF
:1076D00055A217E5FF1F0345851BC94797ECFF1F00
:1076E00083CCFC1A97E5FF1F83C5851A17E4FF1F9B
:1076F0000344141A6315F510CD476392FC109307E9
:107700007008639CF5021307300FB7170E0063086B
:10771000E4001307900DB7B704006314E40817E7FB
:10772000FF1F2321F73CBE8517A501001305C59A4D
:1077300097700100E780C03825BD93078008639DDE
:10774000F500B307804013F4F70FB777460093872F
:1077500087CDB3D78702E1B793079008639AF50006
:10776000B307804013F4F70F91679387C766D5B7C7
:107770009307A008639BF500B307804013F4F70F4D
:10778000B7173D0093870790E9B79307B008639A4E
:10779000F500B307804013F4F70F9167938797D0F4
:1077A0004DBF93F5F5078D47639BF500B307804008
:1077B00013F4F70FB7975B00938707D859BF894732
:1077C000639BF500B307804013F4F70FB7770B0006
:1077D0009387071BBDBF8547639AF500B3078040B9
:1077E00013F4F70FDD67938767E3A5B7D28785F9B1
:1077F000B307804093F7F70FB3D7FA020DB797009E
:107800000000E780409FA285668597000000E78022
:10781000809EB9BB9305610017E5FF1F034525074F
:1078200017E4FF1F0344B40697000000E78040AD53
:1078300093057100228597000000E78060AC3C0052
:1078400017E7FF1F232AF73A834761002304F1005B
:1078500083477100A304F100894717E7FF1F230D39
:10786000F7268357810017E7FF1F2311F70209440A
:1078700009B3154793F64700B336D00093F7870353
:10788000850685C32146638BC7066146638AC706A2
:10789000130680026388C706130680036393C7003C
:1078A000914717E6FF1F2301D62497E6FF1FA38DFC
:1078B000F62297E7FF1F238AE72217E7FF1F0347F8
:1078C00027FD9376070497E7FF1F83C777FC8DEEAC
:1078D0001377770C93067008630CD7021377F707BA
:1078E0008D466312D70CB307F040B7955B0093F752
:1078F000F70F938505D849A81947ADBF854755B7F8
:10790000894745B78D4771BF930670086311D70249
:107910001307300FB7150E006389E7021307900DA8
:10792000B7B504006383E7021307700845BF9306E9
:10793000800C6311D702B307F040B775460013F708
:10794000F70F938785CDB3D5E70297E7FF1F23ABEA
:10795000B718D9BB9306900C631CD700B307F0404F
:1079600093F5F70F91679387C766B3D5B702F1BF59
:107970009306A00C631DD700B307F040B7153D0078
:1079800093F7F70F93850590B3D5F5027DBF930666
:10799000B00CE315D7F4B307F04093F5F70F9167F8
:1079A000938797D0D9B78946631BD700B307F040B8
:1079B000B7750B0093F7F70F9385051BF1B7854655
:1079C000631AD700B307F040DD6593F7F70F93858F
:1079D00065E35DBFD28535FBB305F04093F5F50F48
:1079E000B3D5BA029DB783C72400C18B99C7854719
:1079F00017E7FF1F2305F70EA5BE97E7FF1F23809C
:107A0000070EBDB6854717E7FF1FA300F70E8DB61B
:107A10003C0017E7FF1F2321F71E094793070003C8
:107A20002314F10097E6FF1F2388E60A2DBD639417
:107A30000756A94763E5B742179701001307075296
:107A40008A05BA959C41BA97828717E4FF1F0344C1
:107A500014E4894C6306940D63E68C068547630342
:107A6000F4089307F00F17E7FF1F0347E70663F6D5
:107A7000E70017E7FF1F2301F70697ECFF1F83CCF2
:107A8000AC059307000413F4FC0F63F4970113048F
:107A9000000497E7FF1F9387271603AD0700228690
:107AA0002685EA85B38C8C40229D97700100E78083
:107AB000C0F597E7FF1F2381970397E7FF1F23ADCB
:107AC000A71345BC8D47630CF40A9947E31BF4F8F0
:107AD000979701009387074F17E7FF1F232EF71093
:107AE000A94751B717E7FF1F0347671497E7FF1F21
:107AF000938787004946979501009385A5556306AE
:107B00008700979501009385E5503E8597700100A9
:107B1000E780A0EF17E7FF1F2320A70EC947A1B7F3
:107B200097E6FF1F83C6A610054797E7FF1F9387B9
:107B3000A7FC6394E6023E85130670029795010048
:107B40009385C54E97700100E78020EC17E7FF1F73
:107B50002324A70A9307700239B73E851306300421
:107B6000979501009385C54697700100E780E0E98D
:107B700017E7FF1F2322A70893073004EDB597E509
:107B8000FF1F83C5C5D017950100130525569770B3
:107B90000100E780E0F2054D97EDFF1F83CD2D0931
:107BA00097E5FF1F83C5A5CE179501001305055462
:107BB0006398AD0B97700100E78080F097E7FF1F97
:107BC00083C7E7CCB5CBE36EF4E817940100130448
:107BD000A44C638CB701179401001304644C6386B2
:107BE0009701179401001304244D2285977001001A
:107BF000E78020061375F50F93071500860717E732
:107C0000FF1F230BF7EE8D4717E7FF1FA306F7EEC5
:107C100097E7FF1F938747EE0147BE861376F70F5E
:107C200089076365A60297E7FF1F23A7D7FC97E79D
:107C3000FF1F83C767EC05BD979701009387C73E79
:107C400017E7FF1F232AF7FA914731BD3306E400F7
:107C500003460600A380070005072380C7007DBFF9
:107C600097700100E780C0E597E7FF1F83C727C231
:107C7000E1D7E368F4DE179401001304E43E638C5B
:107C8000A701179401001304A43E6386970117947B
:107C900001001304643F228597700100E78060FBB8
:107CA0001375F50F93071500860717E7FF1F2305C8
:107CB000F7E48D4717E7FF1FA300F7E497E7FF1FDF
:107CC000938787E30147BE861376F70F8907E37C26
:107CD000A6F43306E40003460600A3800700050768
:107CE0002380C700D5B797E5FF1F83C545BA179511
:107CF00001001305654097700100E78060DC97E79D
:107D0000FF1F83C737DF93E7470017E7FF1FA30372
:107D1000F7DE83C7240017E7FF1FA30BF7DC89B842
:107D2000179501001305853E97700100E78020F14B
:107D300097E7FF1F9387C7DB83C7070017E7FF1F7E
:107D40002306F7B417E4FF1F034404D9333480003B
:107D50000DB0179501001305A53C97700100E78051
:107D600000EE97E7FF1F83C7F7D893E7070117E7F0
:107D7000FF1FA301F7D883C7240017E7FF1F2309BC
:107D8000F7D66FF0EFFE179501001305A53A97702F
:107D90000100E780C0EA03C704007D8B51EFB7877D
:107DA000004003C767021377C70B136727002383BD
:107DB000E70203C7A7021377C70B136727002385C2
:107DC000E70203C7E7021377C70B13672700238770
:107DD000E70203C727031377C70B1367270023891D
:107DE000E702854717E7FF1F2302F7B617E7FF1FD4
:107DF0002300F7C217E7FF1F230EF7CC17E7FF1F7B
:107E0000230BF7CC97E7FF1FA38207B497E7FF1F69
:107E1000A38007C097E7FF1FA38E07CA97E7FF1F3E
:107E2000A38B07CA97E7FF1FA38207CC97E7FF1F23
:107E3000A38F07DE6FF0CFF389476312F70297E74E
:107E4000FF1F83C7E7A49146638CD70863E0F6045D
:107E5000638EE70C6369F70A05476380E70EFD57F9
:107E600017E7FF1FA30AF7C637074000B7E700E090
:107E700023A0E71801000100B78600401306F0FCBC
:107E80002381C60223A0E7106FF00FE2130720083A
:107E90006382E7086362F70213071008E391E7FCC7
:107EA000378700408347670293F7C70B93E72700A4
:107EB0002303F7026FF0CFEB130730086389E70263
:107EC00013074008E39DE7F83787004083472703FF
:107ED00093F7C70B93E727002309F7026FF04FE9E9
:107EE000378700408347270393F73707F5B737876E
:107EF00000408347E70293F7C70B93E72700230768
:107F0000F7026FF0EFE6378700408347E70293F709
:107F10003707F5B7378700408347A70293F7C70BAA
:107F200093E727002305F7026FF08FE437870040BF
:107F30008347A70293F73707F5B737870040834792
:107F4000670293F73707ADB7179501001305851F33
:107F500097700100E780A0CE97E7FF1F2388079264
:107F6000D5B3179501001305E51E97700100E78052
:107F700000CD97E7FF1F239B079097E7FF1F93878D
:107F8000A7B503C40700894763F387000944137446
:107F9000F40F6FF00FDE13070002E392E7EC631BB0
:107FA0000B0A638FF500930720026383F50817958A
:107FB00001001305A51D97700100E78060B045B56D
:107FC000179501001305C51997700100E78020C7B8
:107FD0000144179D0100130DED19A14CB3878400D6
:107FE00083C507006A85050497700100E78040ADEE
:107FF000E31694FF178501001305856E9770010045
:10800000E780E0C317E4FF1F0344848801E897E793
:10801000FF1F238F0784014B6FF0AFD58947E31013
:10802000F4E4854717E7FF1F2304F7846FF04FD46C
:1080300017E6FF1F0346B68597E5FF1F83C5258515
:10804000179501001305851397700100E78040A77D
:108050006FF00FD26380F50693071002E399F5F4F1
:1080600097E5FF1F83C5C58217950100130505130A
:1080700097700100E780C0A497E7FF1F23AE97B673
:1080800097E7FF1F938707A6944383D7470017E717
:10809000FF1F034787A517D6FF1F2329D67E1D4440
:1080A00097D6FF1F2396F67E97D7FF1F2383E77E81
:1080B0006FF02FCC97D5FF1F83C5857D17950100E5
:1080C0001305450F97700100E780809F97D7FF1F2A
:1080D0002380077A97D7FF1F239A077A6FF02FF92B
:1080E0002547638FE7C89946378700406394D702D6
:1080F00023008702B7E700E0B706400023A0D718A7
:1081000001000100130600FC2301C70223A0D710C1
:108110006FF08FB99306100A639FD7002300870280
:10812000B7E700E0B706400023A0D7180100010020
:10813000130680FCD1BF9306A009E381D7FE930606
:10814000400AE38DD7FC93062002639DD700B7E772
:1081500000E0B706400023A0D7180100010023006B
:108160008702F9B78546E384D7FE93070008E3004A
:10817000FBFEB7E700E0B706400023A0D7180100D8
:108180000100130620FC23008702BDBF17E7FF1F75
:10819000034797946302F71E63E7E702954763007E
:1081A000F7109947630AF704B78600402380060258
:1081B000B7E700E03707400023A0E71801000100FF
:1081C0001306A0FC75B99307F005630AF70093073F
:1081D00050096306F70093071002E317F7FCB7E7AF
:1081E00000E03707400023A0E71801000100B78630
:1081F0000040130620FC69B117EBFF1F034BCB8D2A
:10820000930700045A8D63F46701130D000497E788
:10821000FF1F9387679E83AC07001374FD0F2286B0
:10822000E685268597600100E780207EB3078B40B6
:10823000669417E7FF1F2301F78A97E7FF1F23AD17
:10824000879AB7870040630C0B022380A703B7E629
:1082500000E03706400023A0C6180100010003C754
:108260002702134707042381E70203C72702137776
:10827000C70F2381E70223A0C6106FF0EFA223806F
:10828000070237E700E0B70640002320D7180100B7
:108290000100130620FC2381C7026FF0AFB93787B6
:1082A00000408347370097E6FF1F83C6768493F725
:1082B0000708D58FA301F700B7064000B7E700E035
:1082C00023A0D718010001001306A0FC35BD97E7D5
:1082D000FF1F9387A793CA9783C7070093F7F70FEA
:1082E000C1CF97E7FF1F83C78794D9E717D7FF1F31
:1082F0000347977E930700026310F70883AD0400DD
:1083000017DDFF1F034DCD5897DCFF1F83CC5C5852
:1083100017DBFF1F034BEB57E6876A87DA866E860B
:1083200097D5FF1F83C5C55417950100130505EAAE
:1083300097600100E780C07897D7FF1F23A4B77B21
:1083400097D7FF1F2382A77B97D7FF1FA38E97790D
:1083500097D7FF1F238B677997D7FF1FA389875074
:10836000B7E700E03707400023A0E718010001004D
:10837000B78600406FF04FA2B7E700E03707400034
:1083800023A0E71801000100B786004015BD97E65D
:10839000FF1F83C6C6890547639CE60429472381DE
:1083A000E70209472383E7022385E70297D7FF1FE8
:1083B000A38E077297E7FF1FA38B0786B78700403E
:1083C000A381070017D7FF1FA30407720547238364
:1083D000E700B640264496440649F259625AD25AFA
:1083E000425BB25B225C925C025DF24D6161828015
:1083F00029472381E70209472383E7022385E70210
:108400002387E7022389E70255B717D7FF1FA30089
:10841000F7466FE01FFF854717D7FF1F2308F75266
:1084200017D7FF1F2306F75E17D7FF1F2304F76A2E
:1084300017D7FF1F2301F76A6FE0BFFE854717D7E5
:10844000FF1F2305F75017D7FF1F2303F75C17D72C
:10845000FF1F2301F76817D7FF1F230EF76617D7F3
:10846000FF1FA305074E17D7FF1FA303075A17D7F0
:10847000FF1FA301076697D7FF1FA38E07648280A3
:10848000411106C697000000E78080FBB7870040D7
:1084900023800700130740FC2386E7001307C0046E
:1084A000A386E70017D7FF1F1307473E2398E7006F
:1084B00017D7FF1F13078741239AE70017D7FF1F1E
:1084C0001307074D239CE70017D7FF1F1307875893
:1084D000239EE70029472381E70209472383E70218
:1084E0002385E7022387E7022389E702A3810700A8
:1084F000930600F8A380D700930690022380D7004C
:10850000FD562383D7002381E7009306000537E754
:1085100000E0230BD740B70640002320D71003C745
:10852000170013671700A380E700B24097D7FF1F1B
:108530002390075C41018280411106C6970000002C
:10854000E78000F0B787004023800700130700FC96
:108550002386E7003147A386E70017D7FF1F1307DD
:10856000E7322398E70017D7FF1F13072736239A10
:10857000E70017D7FF1F1307A741239CE7002947F0
:108580002381E70209472383E7022385E702A381CA
:108590000700930600F8A380D7009306900223807B
:1085A000D700FD562383D7002381E70093060005FB
:1085B00037E700E0230BD740B70640002320D71051
:1085C00003C7170013671700A380E700B24097D7CF
:1085D000FF1F239F075041018280F1679387072087
:1085E00017D7FF1F2320F750854717D7FF1F231DDD
:1085F000F74EA14717D7FF1F2309F74E97D7FF1F45
:10860000A385074E97D7FF1F2382074E97D7FF1FDB
:108610002380072697D7FF1FA38B0724814717D5F1
:10862000FF1F13052525FD5517D6FF1F13064625E9
:108630002947B306F5002380B600B306F600238071
:1086400006008507E397E7FE97D7FF1FA387074834
:1086500097D7FF1FA385074897D7FF1F2380074899
:1086600097D7FF1F238B074697D7FF1F238A0746FD
:1086700097D7FF1FA384074697D7FF1F238107467D
:10868000814717D6FF1F130666574147B306F6000A
:10869000238006008507E39BE7FE828017D7FF1F34
:1086A0000347E75885476316F70017030000670084
:1086B000E3E8170300006700E3DC411122C406C6AB
:1086C00017D7FF1F0347A75685472E8613F4F50FCC
:1086D000AA856317F70417D5FF1F1305652F976049
:1086E0000100E780803297D7FF1F23830732B787C7
:1086F000004023848702B7E600E03706400023A04D
:10870000C6180100010003C7A7021377C70F23850E
:10871000E702B240224423A0C610014541018280F5
:1087200017D5FF1F1305851E97600100E780E02D18
:1087300097D7FF1F238C0720B7870040238287022B
:10874000B7E600E03706400023A0C618010001008C
:1087500003C767021377C70F2383E7025DBF411189
:1087600006C697000000E78080E7B240410117038A
:1087700000006700E3F2411106C697F0FFFFE780B3
:1087800080BF97D7FF1F83C7771CA1CB97D5FF1F4B
:1087900083C5E51B89C917D5FF1F1305651B97E026
:1087A000FFFFE780205497D7FF1FA381071A97D7B1
:1087B000FF1F238D073237E700E0B7064000232074
:1087C000D71801000100378600408347660293F7FF
:1087D000370F2303F6022320D710B24041018280D5
:1087E00041C9D9C597D7FF1F83C78730D1C30111AE
:1087F00022CC4AC84EC656C25AC006CE26CA52C459
:108800002E89AA890144930A0004371B0300637769
:108810002403B3078940C207C183BE8463F4FA000E
:1088200093040004C204C180130A1BD497D7FF1F0E
:1088300083C7C7119DE37D1A631C0A00F24062449E
:10884000D2444249B249224A924A024B056182808F
:1088500097F0FFFFE78020B2D1BF338589002694CF
:10886000A685420497000000E78060E5418045B797
:10887000828097D7FF1F9387273F18429C4383D658
:1088800045000345070083C5C700035646006396AD
:10889000A50083D5E700638DD502011106CE23869E
:1088A000A7002397D700B705CF00DC4B9385757DD4
:1088B00005077D162EC2230001003AC42316C1000D
:1088C0002317D10099C30A858297F24005618280FF
:1088D0008280DC4DDC4B81CFB7E70400904503A3D9
:1088E0008705914517D5FF1F0345453802838280D0
:1088F0006D713C083EC6B707E500232291103EC8C3
:10890000AA843C083285232611103ECA23248110F4
:10891000232021112E8997300000E780C0642A842B
:10892000979501009385058E1775010013058578CD
:1089300097600100E780C018A28517950100130514
:10894000E59C97600100E780A0172945976001002A
:10895000E780E01BB705CB009385757D6800971015
:108960000000E780406AA285680097300000E78039
:10897000E051014781467000CA8526859720000096
:10898000E780C08D05CD2A84979501009385858762
:10899000177501001305057297600100E78040120A
:1089A000A285179501001305259797600100E780C0
:1089B0002011294597600100E78060158320C110D0
:1089C0000324811083244110032901105161828006
:1089D00097D7FF1F9387472918429C43797122D468
:1089E00006D60348070083C807012A8483D64500BA
:1089F000035546006396080183D82701638DD8028A
:108A00002388070105072399D7003708CC00DC4BE2
:108A10001308787D3ACC1307F5FF42CA23080100FA
:108A2000231EE100231FD10099C7080832C62EC4B7
:108A300082973246A245228597000000E78080EBAE
:108A4000B2502254456182806D713C083EC0B70728
:108A5000E5003EC23C083EC42326111023248110A9
:108A6000232291102317010023180100231901006C
:108A7000231A0100231B010097B7FF1F83D74798D4
:108A800099E3C167FD172316F10097B7FF1F83D73E
:108A9000479791EB97D7FF1F9387071D9C439C43F4
:108AA000DC4783D7070017B4FF1F13046495584CA5
:108AB0002317F10083574400484B2318F10031E19C
:108AC000978501009385057B177501001305855E69
:108AD00097600100E780C0FE178501001305C57A85
:108AE00097600100E780C0FD294597600100E7809D
:108AF00000028320C110032481108324411051619E
:108B0000828097B7FF1F83C7179089EBB7E70400F0
:108B1000BC5782975C4C23AA0700E1BFFD1797B6AC
:108B2000FF1FA382F68E03560701834704014C47BB
:108B30000A85230BF10097300000E780403297D779
:108B4000FF1F938767129C430147814688430A862B
:108B50006C0097100000E7806070AA8429C1978597
:108B6000010093852571177501001305A5549760C1
:108B70000100E780E0F4A6851785010013058571E3
:108B800097600100E780C0F3294597600100E78006
:108B900000F8584CB7E70400BC57484B9DBF97B747
:108BA000FF1F83C75786F5D7B7E70400BC4F1044B3
:108BB000854517D5FF1F0345650B82971DBF5C4E8A
:108BC000DC4BB9CFB1CD411122C41775010013059B
:108BD000654E2E84978501009385056806C69760CB
:108BE0000100E780E0EDA285178501001305456DC2
:108BF00097600100E780C0EC294597600100E7809D
:108C000000F1B7E704002244B24003A3870517D55B
:108C1000FF1F0345A5051306400691454101028348
:108C20008280411122C417A4FF1F1304247B1C4C13
:108C300006C689C7DC4399C34C488297584CB7E7AE
:108C40000400BC57484B82975C4CB240224423AA94
:108C500007004101828017A7FF1F1307277A834768
:108C600007009306F00B850793F7F70F63E9F6000B
:108C700097A6FF1F2384F678034507008280930799
:108C800000F8FDB7835745006386071001114AC8F5
:108C900017A9FF1F1309C97652C4032AC90106CEBA
:108CA00022CC03274A0126CA4EC656C2F15735E3E5
:108CB0001307D00DFD57636EC704B7E9040083A7FF
:108CC00009072A841305860042054181B284AE8AD1
:108CD0008297232AAA000325C9015C49A9E7978541
:108CE000010093856555177501001305A53C976034
:108CF0000100E780E0DC178501001305A56497609B
:108D00000100E780E0DB294597600100E78020E073
:108D1000DD57F2406244D2444249B249224A924A63
:108D20003E850561828093874400B705CF002319F3
:108D3000F5009385757D310597100000E780A02C24
:108D40000325C90183456400310597300000E780A1
:108D5000E0130325C9012686D6853105973000002A
:108D6000E780E00F7146A2854A8597600100E780A1
:108D7000C0C9504419CA83A78905854517D5FF1F67
:108D80000345C5EE8297814769B797000000E780E9
:108D9000E0CBD5BFFD573E858280411126C297A406
:108DA000FF1F9384E465D84C22C437E404003C548C
:108DB000484B06C68297DC4C0323C4052244B240CC
:108DC000924423AA070017D5FF1F034525EA8545CE
:108DD00041010283411126C297D4FF1F9384C4E846
:108DE0009C4006C622C44AC0D5C3DC43C5C35CC18F
:108DF0002300B5002A84978501009385253F1775C8
:108E000001001305252B97600100E78060CB294501
:108E100097600100E780A0CF9C4023A4070023A215
:108E2000070097A7FF1F9387675BDC4FDC4B91C759
:108E3000295597000000E78000DF97A7FF1F938761
:108E4000275CDC4FDC4B89C797000000E78020F5EA
:108E500037E904008327C905894517D5FF1F034556
:108E6000E5E082978327C905914517D5FF1F034584
:108E7000E5DF82979C4003A3470163090300228535
:108E80002244B2409244024941010283B24022444A
:108E900092440249410182800111328506CE22CCE2
:108EA00026CA2E8497300000E780E00BAA849785BD
:108EB00001009385E536177501001305A51F97601E
:108EC0000100E780E0BF0307840003566400835578
:108ED0004400A686178501001305854097600100B0
:108EE000E78000BE294597600100E78040C297A750
:108EF000FF1F83C7074F639D970001459700000040
:108F0000E78060D281450A8597000000E780C0ECC9
:108F1000F2406244D244056182806D712324811045
:108F2000232611102322911093F745002E84638786
:108F300007143C083EC0B707E5003EC23C083EC4EB
:108F4000231701002318010023190100231A01002F
:108F5000231B010097A7FF1F83D7474899E3C167E9
:108F6000FD172316F10097A7FF1F83D7474791EB03
:108F700097D7FF1F938747CF9C439C43DC4783D7FA
:108F8000070017A7FF1F130767452317F100544F6A
:108F9000835747002318F100DC4AA1E797850100B9
:108FA0009385452C177501001305C51097600100C6
:108FB000E78000B1178501001305052D97600100BA
:108FC000E78000B0294597600100E78040B4134571
:108FD00044008320C1100324811083244110516177
:108FE000828097A7FF1F83C7D73F2555D9C3FD1799
:108FF00017A6FF1FA307F63E03D606018347070106
:10900000CC460A85230BF10097300000E78020E56D
:1090100097D7FF1F938747C59C4317A7FF1F1307C9
:10902000E73B978601009386262988430A866C00D1
:1090300097100000E7808022AA8451D9978501000B
:1090400093854522177501001305C5069760010039
:10905000E78000A7A685178501001305A523976063
:109060000100E780E0A5294597600100E78020AA7C
:10907000268597000000E78000BB91BF93F725008D
:109080009DC7B7E70400BC47414681452808829741
:10909000255597000000E78000B928089305F00FD8
:1090A00097000000E78040D3134524001DB793F7D5
:1090B0001500014599DF97000000E78020991345CE
:1090C000140001BF5C4D411106C688C317D7FF1FAE
:1090D000232CF7B8B7E7040083A70708170500009B
:1090E0001305E5E38297B24097D7FF1F2380A7B807
:1090F00001454101828001113335A000A307A10081
:10910000B7E7040083A7471706CE1306F10085458D
:10911000130550308297F2400561828082804111B0
:1091200022C406C617D4FF1F0344C4B531E497B761
:10913000FF1F83C7770FB9E397C7FF1F83C7074F89
:1091400099E717B4FF1F0344240E1344140022852B
:1091500097000000E78060FA178501001305852954
:1091600009E4178501001305E5292244B2404101B5
:10917000176301006700C3940144D1BF0544C1BF18
:10918000797122D4A30F010037E4040083278417E8
:1091900026D24AD006D6AA842E89130550309305CC
:1091A000F10132C6829732468347F10193150601D9
:1091B000C18185CB01452EC697000000E780E0F312
:1091C00083274417B2454A8626858297054597002E
:1091D0000000E78080F2B250225492540259456157
:1091E0008280832744174A8626858297EDB74111EE
:1091F0009397050122C406C626C2C1872E8463D474
:109200000702B7E40400FC5417A5FF1F03454522DD
:10921000829719C1BC5482972165218DB2402244A6
:1092200092444101828093F715008DC7B7E704008F
:1092300083A7471A17A6FF1F1306861E97D5FF1F81
:10924000938585A317A5FF1F0345851E82971345A8
:109250001400E9B793F7250099CFB7E70400BC4F96
:1092600013060064894517A5FF1F0345651C8297F7
:109270001345240065B793F7850085CF97D7FF1F67
:1092800083C707A185E7B7E7040003A8871A130778
:10929000401F97A7FF1F83C7A719814613064006E3
:1092A000994517D5FF1F0355259E02981345840045
:1092B000B5B793F745000145B5D3B7E4040083A7DC
:1092C000041817D5FF1F0355259C8297BC4C130625
:1092D0000064914517A5FF1F034585158297134527
:1092E00044002DBF97D7FF1F83D7079A6398A70223
:1092F00017D7FF1F231BB79817D7FF1F2318C7982F
:1093000017D7FF1F2315D7982E8617850100130541
:10931000E515BE85175301006700837A17850100A4
:109320001305451617630100670063910357450055
:1093300097D7FF1F83D74795631EF704C167411175
:10934000F91722C417D7FF1F2320F79437E404002E
:1093500097D7FF1F23AC079297D7FF1FA3840792CD
:1093600097D7FF1F238607927C4C06C6894517A511
:10937000FF1F0345E50B82977C4C914517A5FF1F06
:109380000345050B82972244B240410117030000B8
:10939000670023D9178501001305C50E1763010067
:1093A0006700E3897D15954763E2A71C17870100D5
:1093B0001307C7020A053A951C41011122CC06CEBB
:1093C000BA972E848287178501001305250C9760B4
:1093D0000100E780C086A1A203C725009947631159
:1093E000F7022E8597000000E78080F48345640033
:1093F000178501001305850A97500100E780406C2E
:1094000097B7FF1F238207E2178501001305C50ADE
:109410007DBF03C7250095476319F702C16717D7BA
:10942000FF1F03576786F91703D5A5006309F702E5
:10943000B7E7040083A7C7178297178501001305B4
:10944000A50897500100E780807F854717B7FF1F69
:10945000230CF7DC17850100130585098DBF97D70D
:10946000FF1F2393A78283D7E50097D6FF1F239E74
:10947000F68083D7050197D6FF1F2399F68083D7FF
:10948000250197D6FF1F2394F68097C7FF1FA38B54
:10949000077E631BE502B7E70400BC4F09661306AD
:1094A0000690A14517A5FF1F034585F8829703562F
:1094B000E4008355A4001785010013052502975089
:1094C0000100E780E05F51B79307700F2316F100AA
:1094D000B7E7040083A7870D17A6FF1F034646F5CD
:1094E0006C0082974DF9854717C7FF1FA30CF778CB
:1094F0005DB71785010013056500D1BD83C5250043
:1095000091476392F502178501001305A500975056
:109510000100E780C07297000000E78080C0F24041
:1095200062440561828099476392F5022285970023
:109530000000E780E0DF8345640017850100130524
:10954000E5F597500100E780A057D1BF9547639A92
:10955000F50083471400E1F3178501001305C5FDED
:10956000BDB5178501001305A5FDE1BF8280375702
:10957000315F97A7FF1F9387E7EC130777D598C351
:109580009356C50017870100130707EBBA9683C5EA
:10959000060093568500BD8ABA9603C60600935608
:1095A0004500BD8A3D89BA962A9783C606000347BF
:1095B0000700238407002383D700A383E7002382C7
:1095C000B700A382C70097A7FF1F9387A7E823834D
:1095D000B700A383C7002384D700A384E700828059
:1095E000411106C697000000E780A0F8B7E7040025
:1095F00083A7871417A6FF1F1306C6E4D5450145A8
:109600008297B2404D4697A5FF1F9385A5E41305A9
:1096100070304101170300006700C3B66171232455
:10962000811A37E40400832704082326111A232211
:10963000911A2320211B232E311917050000130531
:1096400045BB829717A9FF1F130989DE99478544F7
:109650002300A900231CF100978501009385C5DC38
:1096600093074006177501001305C5A4231CF108D4
:109670002308910097C9FF1F9389A90B97500100F8
:10968000E780004483D50900178501001305C5D87C
:1096900097500100E780C042294597500100E780BC
:1096A000004703D5090097000000E78080EC83277E
:1096B00044171008854513055030829783274417B7
:1096C00017A6FF1F130606D9CD45130570308297E4
:1096D0008327441717A6FF1F1306C6D5B5451305E4
:1096E000603082978327441730088945130510316D
:1096F00082978327441730098945130520318297C3
:10970000832744159305000A0D4582978327441546
:109710009305000A11458297A30591002306910045
:1097200002CD23080100230C010083278416300991
:109730009145130570408297832784161306B10064
:109740008545130500408297832784167000854560
:10975000130510408297832784163008854513052A
:1097600020408297832784161008854513055040B2
:109770008297832704157D558297832744137D554F
:1097800082977D5597A0FFFFE78020F08327440C48
:10979000829797A0FFFFE78080CB8327841417A6CA
:1097A000FF1F130626CAD545014582978947130630
:1097B000700F814528092306F1009790FFFFE7808D
:1097C00000958D471306000881452808230CF108F1
:1097D0009790FFFFE780A0939147230CF1009767D4
:1097E00001009387A77E984383C747003AC8230A9E
:1097F000F10097D0FFFFE78020B770008545054551
:1098000097A0FFFFE78080EF30099305700F0945AF
:1098100097A0FFFFE78080EE3008930500080D4514
:1098200097A0FFFFE78080ED10089545114597A0B0
:10983000FFFFE780A0ECC16717C7FF1F1307C744EE
:10984000F9171CC32322070017A5FF1F130505BE28
:1098500097A0FFFFE78060E98327C41D17C5FF1F9E
:109860001305054182973C480345090085458297C9
:109870008320C11A0324811A8324411A0329011A5F
:109880008329C1195D618280C16717C8FF1F035812
:10989000A83FF9176301F8083DCDB5CD011126CADF
:1098A000B7E4040083A7841222CC2E862315B100CE
:1098B00006CE2A8401478146ED45428582972AC615
:1098C00011ED17850100130565B897500100E78079
:1098D0000037F2406244D24405618280FC44035662
:1098E000A100A28582972C0017C5FF1F0355C5391B
:1098F00097A0FFFFE78020EC69DD178501001305C5
:1099000025B697500100E780803383A7C412ED4548
:10991000280082977DBF82800DC5854717A7FF1F4E
:10992000A30FF7B097A7FF1F238C07B0354697A565
:10993000FF1F938525B013056030170300006700F3
:10994000638497A7FF1FA38C07AEE9BF97C7FF1FCC
:1099500083C70734A9EFC16717C7FF1F0357C73273
:10996000F9176306F7044111854722C417C7FF1F83
:109970002300F73237E404007C4C06C6A14517A546
:10998000FF1F0345E5AA82970323841A2244B240AD
:1099900097A7FF1F83C7C7A917C5FF1F0355C52E6C
:1099A0001307401F81463146994541010283828059
:1099B0006D712324811023261110232291103284EB
:1099C00001CD8947630AF5028320C1100324811069
:1099D000832441105161828017850100130505B76A
:1099E000AE8497500100E7808025A285268597C028
:1099F000FFFFE78060B2C9BFB7E70400FC4728005B
:109A0000829717850100130525B597500100E7805F
:109A100000238347810039C41307000B6380E702EA
:109A20001387A7051377F70F8D4663EDE602A2852E
:109A3000280097C0FFFFE780002979B78547E3F545
:109A400087F883459100177501001305E597B33535
:109A5000B00097A7FF1F2389B76497500100E780E4
:109A600020069DB703479100A207D98F35671307DA
:109A7000D7556385E7086368F7022D671307B75565
:109A80006387E70631671307C755638AE7042967C9
:109A90001307A7556394E702A285280097C0FFFF2C
:109AA000E780606115B739679306E7656381D7087A
:109AB00063E9F6001307E7556384E706A2852800EB
:109AC0003DB73D679306F755638AD7061307F766D8
:109AD000E396E7FE97C0FFFFE7804077F5B50146C4
:109AE000A285280097C0FFFFE7808049F1BDA285CD
:109AF000280097C0FFFFE780405AF9B58947E3F592
:109B000087EC97000000E780A0E49305E4FFC2051E
:109B1000C1811305A1009790FFFFE780606C6DB5D0
:109B2000A285280097C0FFFFE780E05971BDA2859C
:109B3000280097C0FFFFE780006279B597C0FFFF5C
:109B4000E780806A51B5C16717C5FF1F0355C5136C
:109B5000F9176307F500B7E7040003A3C7170283EB
:109B60008280854717C7FF1F230EF710014517F3A3
:109B7000FFFF6700835817F3FFFF6700835A1783BF
:109B8000FFFFE70223542A8408452E89B28919C9A8
:109B900000C1971500009385A586610597300100E7
:109BA000E780200581447D5A97100000E780E03966
:109BB00063C7A404814497100000E780003A63C89B
:109BC000A40497C7FF1F9387E70C9C43DC47B307A8
:109BD000F94091872302F400638309048327C900B5
:109BE000B307F4409587A302F4001C4C89C79C4737
:109BF00099C3228582971783FFFF6700E34F5C4478
:109C0000139714008504BA972390470171BF1C482D
:109C1000139714008504BA972390070069BF832720
:109C200089000547B307F4409587A302F4008357E2
:109C30000400638EE7028DC309476384E7040D4780
:109C4000E395E7FA978701009387C7E31CCC9787D2
:109C50000100938727E411A897870100938707AA3B
:109C60001CCC97870100938767AA5CC8BDBF978704
:109C700001009387A7951CCC9787010093870796CF
:109C8000EDB7978701009387A7E41CCC9787010065
:109C9000938707E5D9BF95E51783FFFFE7022344C4
:109CA000004618448347940075839D8B6317F70023
:109CB00097100000E78060B448C41783FFFF670077
:109CC000434482801783FFFFE702C33F13893500B7
:109CD000C16442094111AA890144F11413590901CF
:109CE000054A2EC697100000E7802026B24563483B
:109CF000A400014541011783FFFF6700E33F83A7ED
:109D0000090013171400BA9783D707006388B700B8
:109D10006394970063742A010504E1B70545D9BF30
:109D20001783FFFFE7022339AA892E89328BB68475
:109D30003A8ABE8A97A00000E780C0FE71C92685D6
:109D400097200000E780C00C8D4763E7A7007D5592
:109D50001783FFFF6700A33983DB440097100000DF
:109D6000E780A0242A8497100000E780402593070D
:109D7000740031443305850263CDA70297100000BB
:109D8000E780A02297100000E78020222A84971005
:109D90000000E780C0229307740031443305850238
:109DA00063C3A70497100000E780202093074500B5
:109DB00029A897100000E78080203305850213074B
:109DC000F0179307C017E35FA7FA2D55E3C277F9A1
:109DD00063040B02D6865286A6854A859720010029
:109DE000E780C0BDB5B797100000E780401D330580
:109DF00085029307C5FFD1BF832749001385C9009A
:109E000083D5270097000000E78000EC61F581B75B
:109E100069553DBF97C7FF1F2390A7E897C7FF1F4E
:109E2000938747E7904381470C463307F500420785
:109E300041836393B7008280544613984700850797
:109E4000C2962390E600D5B797C7FF1F938787E494
:109E50009C4303C58700828017C5FF1F0355C5E3D8
:109E600082801783FFFFE7028327C1671387D7FF2D
:109E7000630BE502636AA700F1176300F502014571
:109E80001783FFFF6700E3271387E7FF6302E502FD
:109E9000FD171D8D13351500E5B797500000E780BD
:109EA000602A7D15C5BF97500000E780E0FED5BF52
:109EB00097500000E78000FDEDB71783FFFFE70232
:109EC00003224111AA8401442EC697100000E780A6
:109ED000C008B2456348A400014541011783FFFF54
:109EE000670023229C48131514003E9583570500F4
:109EF000E385B7FE0504C9BF03485500814693F7C3
:109F0000F60F63E5070181473E85828058459397A8
:109F10005600BA9703D727006316B70003D7070088
:109F2000E304C7FE8506E1BF8346450001479377FA
:109F3000F70F63E4D700814711A81C45131657009B
:109F40000507B29703D60700E313B6FE3E8582806D
:109F50001783FFFFE702031793170501C18797CA0D
:109F6000FF1F938A2AD3635BF00883A70A00C047C8
:109F70009C4703570400198D420541816368F50031
:109F8000014422851783FFFF6700031712052A94F7
:109F9000CDBFDC4713944900014A3E9483474400F7
:109FA0006341FA02014A834754006349FA02850972
:109FB000C20993D9090183A70A009847E3EBE9FC9A
:109FC000C1B71C4413195A00A6853E994A859700CB
:109FD0000000E780C0EE05E1050AC9B75C4413192B
:109FE0005A00A6853E994A8597000000E78020ED3B
:109FF00019E1050A4DBFE30C09FA61B7AA8481494A
:10A000005DBF1783FFFFE702830D1C452A8481E7AC
:10A010009307C5001CC51C44231204001CC09307F1
:10A02000F00F63EDB70093F5F50F22859720000040
:10A03000E780C0E51783FFFF6700A30C9394050139
:10A04000C167C18063F9F500A685228597200000CD
:10A05000E780E0E8C5B7C18193F5F50F2285972029
:10A060000000E780A0E2A685228597200000E78017
:10A07000E0E3C9B797C7FF1F9387C7C188438280B2
:10A080001C4599C797C7FF1F23A6A7C0014582801B
:10A090007D55828097C7FF1F9387C7BF984383472B
:10A0A0004500484792073E9582801783FFFFE702ED
:10A0B0000303617100451C183EC6B70780013EC806
:10A0C0001C183ECA8357440002CE02D002CC231E85
:10A0D000F100834784002A8902D22301F1023C085F
:10A0E0003ED402D697000000E78000FB83570500AE
:10A0F0002316F10297500000E78000C82307A10251
:10A100005C4003556400F18313F717008347F102A5
:10A1100052055181F99BD98FA307F10297100100D5
:10A12000E780207939CDAA840355050097A0000067
:10A13000E78020C083D704002AD26800231CF100E6
:10A1400083D72400231DF1001C4803D647008C430D
:10A1500097200000E780A0D08347B400CA86177616
:10A160000100130626408117A305F4006C00481077
:10A1700097200100E78080845D611783FFFF6700FF
:10A1800043F82155D5BF1C45B1CF03C5A70089466B
:10A1900013576500630BD7028D46630ED7028546C1
:10A1A0006300D702130740063305E50203C7B70073
:10A1B000418B15CB83C7B700BD8B3355F5408280EB
:10A1C0001375F5031307803EC5B709671375F503CB
:10A1D00013070771D1BF372709001375F50313075C
:10A1E000077CD9B7014582801783FFFFE70223EF81
:10A1F00003A98500630C09048347B900AE8493F773
:10A20000070E85C303459900930520030D810505BD
:10A21000B305B5028844610597300100E78080AD41
:10A2200035A02E8597000000E78020F62A8419CDFE
:10A2300097000000E780605C8325C900B307B54044
:10A2400063FA87002E94B305A440E9F51783FFFF56
:10A25000670023EB85457DBF1783FFFFE70223E8F7
:10A260002A8403D50500011132C636C43AC22EC075
:10A2700002CA02CC02CE97A00000E78080AB8245E4
:10A280002ACA22852ECC97000000E780E0E0035721
:10A290000500231EE10097500000E780E0ADA246D4
:10A2A00032469247230FA10036874C08B28622859A
:10A2B000014697000000E780E0A605611783FFFFD5
:10A2C000670023E41783FFFFE70263E161711C1855
:10A2D0003EC6B70780013EC81C183ECA3C08004570
:10A2E0003ED4AA8402CC02CE02D002D202D697007B
:10A2F0000000E78060DA8357050035592316F10224
:10A3000097500000E78040A72307A10209C48357A4
:10A31000440081EB21594A855D611783FFFF670087
:10A3200043DE035564005205518197100100E78018
:10A3300040582A8965D18347B40093F7070E99C71F
:10A340001305840197300100E780009D8357440086
:10A35000231EF100834784002301F1025C40035572
:10A360000900D98313F7070883471102231CA100B2
:10A3700093F7F707D98FA300F10283572900231D14
:10A38000F1005C40F18313F717008347F102F99B5A
:10A39000D98FA307F10297A00000E78080992AD205
:10A3A00035D9834794006800139757008347B4005A
:10A3B000FD8BD98FA305F4001C4803D647008C43BE
:10A3C00097200000E780A0A9A68717770100130750
:10A3D0006719740005464C10268597000000E78039
:10A3E00060942A890DD98347B400A685FD8BA30507
:10A3F000F40097000000E78060DF31BF1783FFFFA4
:10A40000E702E3CD832485FE2A8441112685970047
:10A410000000E78080D7834734FF93F7070E8DCB8A
:10A420002AC6268597000000E78060C809CD8347CB
:10A4300034FFB245FD8BA309F4FE91C52285973008
:10A440000100E780208B41011783FFFF670063CB8A
:10A450007DD98327C4FF2685829775F5834734FF0E
:10A4600093F7070E91C7228597300100E780C08AD5
:10A47000032584FE97000000E78000E5E9B7178315
:10A48000FFFFE702C3C29C4141112A8903C70700AD
:10A4900089472E84935667006380F6040D466388CF
:10A4A000C6049307F0076304F7022E859720000087
:10A4B000E78060ABAA848149C16B130C490097B750
:10A4C000FF1F9387277D9C43984763E4E90441017C
:10A4D0001783FFFF670063C103D745008547E3F893
:10A4E000E7FE2E8597200000E78040ADE1B703D757
:10A4F0004500E3FEE7FC2E8597200000E780A0A63C
:10A50000AA84228597200000E78000A8C204C98C95
:10A510005DB7DC470355A900139A49003E9A93178B
:10A520000501C187635DF00083570A006397A702A6
:10A5300063E774038327CA00034D5A002DA0A16767
:10A540002167A98F1307F7EFE374F7FE63970900FC
:10A5500097000000E780209161FD85098DB7832772
:10A560008A00034D4A00835DA90003576900216AF0
:10A57000138BC7003AC6814A33CA4D01631E5D0181
:10A5800097B7FF1F938787719C43E1DBA2866286A2
:10A59000814526858297D1B7A1679387F7EF930C02
:10A5A0004BFF63F24703B2455A8597F0FFFFE78000
:10A5B000A0710DC103278B00104709CE10436382A1
:10A5C000C4023107D5BFEE85668597000000E7809D
:10A5D000008F71F993861A0093FAF60F130B0B0292
:10A5E00071BF835644005C43E3E9F6F622853AC620
:10A5F00097200000E7802081A1679387D7042A8AEB
:10A60000035D4400324763E897008347D90093E72E
:10A6100007F8A306F9001C4766852286E285829723
:10A62000C1670844FD17337AFA00529508C0231217
:10A63000A40125B797B7FF1F9387C7659843814744
:10A6400015C31447814763FFD500939745004C47D6
:10A65000BE9519C903C7550081476375E600DC45FF
:10A660001606B2973E85828003C745008147E37B8B
:10A67000E6FE16069C45F5B71783FFFFE70283A4A5
:10A68000AA892E8A814497BAFF1F938AAA6083A75A
:10A690000A00984763E6E4001783FFFF6700C3A53D
:10A6A000DC471394440001493E9413BB14008347D4
:10A6B0004400634BF900014913BB14008347540065
:10A6C000634FF9008504E1B7084493175900528796
:10A6D000DA860146A2853E9582990509C9BF48449C
:10A6E000931759005287DA860546A2853E958299CE
:10A6F0000509E9B71783FFFFE702639E814517F558
:10A70000FFFF1305054897B7FF1F239707589700CA
:10A710000000E780A0F61783FFFF6700839E97B7CE
:10A72000FF1F938727579C4395C31783FFFFE702BB
:10A73000039B814517F5FFFF1305A5449700000013
:10A74000E780C0F31783FFFF6700A39B8280178316
:10A75000FFFFE702239737E40400832784124111A7
:10A760002315E100AE893289368A3A86814601474F
:10A77000ED45AA8482972AC621C90356A100D28535
:10A7800097400100E78060288327C413CE85268583
:10A790008297058905C98327440D231421010146A9
:10A7A0002C00268582972A8401C9B7E7040083A775
:10A7B000C712ED4528008297228541011783FFFFCC
:10A7C000670083934944D5B76554FDB75C41FD17D5
:10A7D0005CC182801783FFFFE7026390B7E7040044
:10A7E000FC5F829795473305F50281450D811783FC
:10A7F000FFFF670003911783FFFFE702438EB7E770
:10A800000400FC5F829795473305F5020D8117839D
:10A81000FFFF6700038F1783FFFFE702438CB7E753
:10A82000040083A7870B0355050082971783FFFF5A
:10A830006700238D1783FFFFE702638A0355050036
:10A840003287AE861796FF1F0356E6C697B5FF1FE1
:10A850009385054597000000E780A0EF1783FFFF71
:10A860006700238A1783FFFFE7026387B7E70400C7
:10A8700083A7C71782971783FFFF67008388178313
:10A88000FFFFE702C385B7E7040083A7871397B5E7
:10A89000FF1F9385E540829701451783FFFF6700FF
:10A8A00043861783FFFFE7028383B7E7040083A78C
:10A8B000C71F81451795FF1F0355E5BB8297178377
:10A8C000FFFF670003841783FFFFE7024381B7E7B9
:10A8D000040083A7871397B5FF1F9385653D829773
:10A8E00001451783FFFF6700C3811773FFFFE7026E
:10A8F000037FB7E7040083A7C71F81451795FF1F94
:10A90000035565BD82971773FFFF6700837F177339
:10A91000FFFFE702C37C2E8597800000E78080B3AD
:10A9200097800000E78080F01773FFFF6700637D6A
:10A930001773FFFFE702A37A97800000E78080FA91
:10A940001773FFFF6700E37B5C49E1175CC95CC5D7
:10A9500083572501A1072319F50083570501A10796
:10A960002318F5008280F1473305F50297B7FF1FE2
:10A97000938707369C433E9582808D476315F60882
:10A9800003D74600854763F0E7081773FFFFE70228
:10A990000375368536842E8997100000E780A05C09
:10A9A00029C98357440093140501C18063E39704C8
:10A9B000228597100000E780005BFD1423129400AD
:10A9C0009307A0026300F5029307B0026307F50244
:10A9D00093079002631FF500228597000100E7802E
:10A9E000608901A80146CA85228597A00000E780FA
:10A9F00000B41773FFFF6700C37022859710000033
:10AA0000E7806007FDB7828097B6FF1F9386862C8C
:10AA10009C42014599CF9843D44217B6FF1F232B80
:10AA2000E62A6396D70097B6FF1F23A7E62A138569
:10AA3000C7FE82801773FFFFE702636A970000007A
:10AA4000E780A04B71443305850291459790000043
:10AA5000E780C0EC11E565551773FFFF6700636A77
:10AA600097B7FF1F23A4A72697000000E780E048C0
:10AA700033058502914597900000E78020EA61DD6B
:10AA800097B7FF1F23A6A72497000000E780E046A2
:10AA900097B7FF1F2396A72297000000E780E045A5
:10AAA00097B7FF1F239FA720977701009387C7B011
:10AAB00017B7FF1F232AF72097070000938707E99E
:10AAC00017B7FF1F2320F720014579B71773FFFF42
:10AAD000E702E360AA8517B5FF1F1305651E9710EF
:10AAE0000000E780605F1773FFFF670083611773E3
:10AAF000FFFFE702C35E97000000E78060FD97104C
:10AB00000000E780E05E97B7FF1F9387A71C9C4378
:10AB100091CF1387C7FE19CB83D5C7FF17B5FF1F8A
:10AB20001305C51B97200100E780C01C1773FFFFAA
:10AB30006700235D1773FFFFE702635A9700000069
:10AB4000E780C0EC09CD834785002A8493F707048A
:10AB500099EB0355E50097000000E78080F9177333
:10AB6000FFFF6700035A8347C5009304450117B9E7
:10AB7000FF1F1309291685E3832709005CC997B7CE
:10AB8000FF1F23A9971483274900F1FB97B7FF1FE5
:10AB900023A49714E9B7FD172306F50061059780F4
:10ABA0000000E78060DA8307840063CB07048347F3
:10ABB000840093E707F82304F400B7E704009C5FE0
:10ABC00082974205A94741813375F5028347840086
:10ABD00093F707FCC98F2304F4008347D4003E9504
:10ABE0001C402318A40089CF984319CB8347C40085
:10ABF0005040814585073305F502420541810297A2
:10AC0000832709005CC897B7FF1F23A5970C8327EC
:10AC1000490089E797B7FF1F23A0970C8347C4001B
:10AC20009DDF8355040117B5FF1F1305250B9720E2
:10AC30000100E780200C25B71773FFFFE702234AC6
:10AC400097B7FF1F9387C72E9C4701448583858B49
:10AC500085E3AE84B2853A8697100000E780204FE6
:10AC60002A8419C597100000E7806045829408CCBB
:10AC700022851773FFFF6700C3481773FFFFE702C2
:10AC8000634441112E8932C6AA8997000000E780EB
:10AC9000C031324713060502CA8697050000938526
:10ACA000C5CC17B5FF1F1305A50197000000E7806D
:10ACB000E0F82A8425C99304C50097000000E780C6
:10ACC000E0411946AA85268597100000E7802019E3
:10ACD0008545268597100000E7800015177501004F
:10ACE0001305458B4E95834505002685971000007A
:10ACF000E780C0195C4831468145A1075CC85CC447
:10AD000083572401E1172319F40083570401E11745
:10AD10002318F4001C4C3E859770FFFFE780203F0E
:10AD2000A3042501228541011773FFFF6700C33C7F
:10AD30001773FFFFE702A33A4111AA842EC632C45B
:10AD400097100000E780003A004DB2452246834745
:10AD500084000CC050C093F7F70393E70704230463
:10AD6000F40023180400268597100000E7802035A2
:10AD700083479400A9462317A40013D7370005077B
:10AD80003307D7029D8B85072306F400A306E40052
:10AD900083C70401D8488507230FF7FE17B7FF1FA5
:10ADA000130747F35843232A04009307440129E378
:10ADB00017B7FF1F2322F7F217B7FF1F232CF7F057
:10ADC00017B4FF1F130484F1228597200100E78048
:10ADD000A0E41C44858B5D8D19E581452285972073
:10ADE0000100E78020F141011773FFFF6700633125
:10ADF0001CC317B7FF1F2321F7EED9B71773FFFF47
:10AE0000E702E32D97050000938565B7014597009C
:10AE10000000E78000B001451773FFFF6700632E55
:10AE20001773FFFFE702A32B97000000E78080B0B5
:10AE30001773FFFF6700E32C8347C500A5E3177373
:10AE4000FFFFE702C3292A840355E50097000000AD
:10AE5000E78000C821C18347840093F7F7FB2304F0
:10AE6000F4001C4091C7DC4381C74C4001458297E8
:10AE700097000000E78080B917B5FF1F130505E6AE
:10AE800097200100E78040E90355E40097000000A7
:10AE9000E78020C61773FFFF6700A3268280177321
:10AEA000FFFFE702C32397B7FF1F9387A7E297052A
:10AEB0000000938565C817B5FF1F130525E223A081
:10AEC000070023A2070097200100E78080D21773B4
:10AED000FFFF670003231C4D91CFDC4381CF177325
:10AEE000FFFFE702C31F8345070082971773FFFF29
:10AEF00067002321828097B7FF1F938767E09C43F9
:10AF000003C50700828097B7FF1F938767DF9C43C5
:10AF100003C51700828097B7FF1F938767DE9C43A6
:10AF200003C52700828097B7FF1F938767DD9C4387
:10AF300003C54700828097B7FF1F938767DC9C4358
:10AF400003C53700828097B7FF1F938767DB9C4359
:10AF500003C55700828097B7FF1F938767DA9C432A
:10AF600003C56700828097B7FF1F938767D99C430B
:10AF700003C57700828097B7FF1F938767D89C43EC
:10AF800003C58700828097B7FF1F938767D79C43CD
:10AF900003C59700828097B7FF1F938767D69C43AE
:10AFA00003C5A700828097B7FF1F938767D59C438F
:10AFB00003C5B70011E11D45828097B7FF1F938736
:10AFC00027D49C4303C5C700828097B7FF1F938790
:10AFD00027D39C4303C5D700828097B7FF1F938771
:10AFE00027D29C4303C5E700828097B7FF1F938752
:10AFF00027D19C4303D50701828097B7FF1F938712
:10B0000027D09C4303C52701828097B7FF1F9387F2
:10B0100027CF9C4303D54701828097B7FF1F9387B3
:10B0200027CE9C4303D56701828097B7FF1F938784
:10B0300027CD9C4303D58701828097B7FF1F938755
:10B0400027CC9C4303C5A701828097B7FF1F938736
:10B0500027CB9C4303C5B701828097B7FF1F938717
:10B0600027CA9C4303C5C701828097B7FF1F9387F8
:10B0700027C99C4303C5D701828097B7FF1F9387D9
:10B0800027C89C438857828097B7FF1F938747C77D
:10B090009C4303D5C702828097B7FF1F938747C69B
:10B0A0009C4303D5E70219E11305800C828097B712
:10B0B000FF1F9387E7C49C4303C50703828097B7AC
:10B0C000FF1F9387E7C39C43C85B828097B7FF1F2E
:10B0D000938787C28843828097B7FF1F938707C2F1
:10B0E0008843828019E17D558280F5DE984265DFD4
:10B0F000FDD917B7FF1F1307A7E31847AA87715594
:10B10000058B631D072403C507001547E37DA7FCD6
:10B1100003C737001305F0057D171377F70FE364B6
:10B12000E5FC03C35700E30003FC83C86700E38C1E
:10B1300008FA03C77700494579171377F70FE364D7
:10B14000E5FA03C7A70011481305F7FF1375F50FBC
:10B15000E36BA8F803CE97000D481305FEFF1375A7
:10B16000F50FE362A8F803C8B70063090800651883
:10B170001378F80F1305600DE36705F703C5C700E3
:10B18000794879151375F50FE36FA8F403C8D70054
:10B190000D457D181378F80FE36705F503D807010F
:10B1A000930E40175118420813580801E3ED0EF3AF
:10B1B00003C8E7007D181378F80FE36605F303C8AA
:10B1C00027017D181378F80FE36F05F103C8870096
:10B1D000C54E75181378F80FE3E70EF103D8670131
:10B1E000856E938EBEE06D18420813580801E3EC9B
:10B1F0000EEF03D847016D18420813580801E3E425
:10B200000EEF03D887017918420813580801E36C40
:10B2100005ED03C8A7017D181378F80FE36505ED68
:10B2200003C5B7011D487D151375F50FE36DA8EA39
:10B2300003C5D701714879151375F50FE365A8EAC1
:10B2400003D5E7011308E00F7D1542054181E36C4A
:10B25000A8E803C50702494879151375F50FE3649B
:10B26000A8E8C85301C937C834005915130858BF96
:10B27000E36BA8E603A8870237C53400130555BF62
:10B280005918E36205E717B5FF1F2329C5A603C6B2
:10B29000050117B5FF1F2325F5A60545E375C5E490
:10B2A00003D82501D04933760603E31E06E203C620
:10B2B0001501E30A06E217B6FF1F232FB6A283C5C6
:10B2C000270001466387A50003C61700F145330632
:10B2D000B60283C707039305C00272971A071307C4
:10B2E000C70516031A9796084697B387B7024155C4
:10B2F0003E973297420741836362E8061773FFFF68
:10B30000E702E3DD368597800000E780406C970018
:10B310000100E780C04B2A8497A00000E780205EF0
:10B320002A9497F00000E780002A2A949790000062
:10B33000E78040852A9497F0FFFFE780E06F2A942A
:10B3400097400000E78000972A9497700000E780FC
:10B3500040A022951773FFFF6700A3DA828017735E
:10B36000FFFFE702C3D74111A307A10097A0000088
:10B37000E78040C99305F100170500001305E5B506
:10B3800097F0FFFFE780802F014541011773FFFF12
:10B39000670023D71773FFFFE702E3D117B4FF1F3E
:10B3A000130404B90328840079599368180097B4EA
:10B3B000FF1F23A314B91378180063100802BA847E
:10B3C000BE89368B328A2E89AA8A97F0FFFFE780E2
:10B3D000E0A77D15269519E531594A851773FFFFBA
:10B3E0006700E3D097F0FFFFE78040A67D15269524
:10B3F000A167E353F5FE97B7FF1F938727EA9843AA
:10B400003E8C814B01CB014597F00000E780C0479F
:10B41000933B15004A85DA865686D28597900000C0
:10B42000E78060512A8911CD1C44F99B17B7FF1F93
:10B430002324F7B083270C00CDD3E3800BFA829747
:10B4400069BF268597B7FF1F23A607AE97F0FFFFBA
:10B45000E780809C4146CE8517B5FF1F1305C5B612
:10B4600097300100E780605A97D00000E780E09CA9
:10B470000325040B97D00000E780A0A0054597D0D6
:10B480000000E780A0A7054597000000E78060ED79
:10B49000A9B797B7FF1F9387A7A99C47858BEDC7CF
:10B4A0001773FFFFE702A3C317B5FF1F130505B00E
:10B4B00097B7FF1F23AE07A697B7FF1F23AC07A6BA
:10B4C00097B7FF1F23AA07A697200100E780C08433
:10B4D00097500000E78080F997100100E780405006
:10B4E00097100100E780405697B7FF1F9387C7A2C8
:10B4F0009C4391C7054597800000E780E02397B7FC
:10B50000FF1F9387278B9C4399C741657D159770D3
:10B510000000E780E0A597F00000E780804197D029
:10B520000000E780209397B7FF1F938727B59C43C0
:10B53000139717016356070097F00000E780A0B04B
:10B5400097B7FF1F23A207A897B7FF1F23A007A83D
:10B5500097B7FF1F23AE07A697B7FF1F23AC07A619
:10B5600097000000E780008C97000000E780A0753E
:10B5700097F0FFFFE780401897F00000E780E0D9E0
:10B580001773FFFF6700E3B7828097B7FF1F9387AA
:10B59000279A8843828097B7FF1F93876799C8438C
:10B5A0008280B7E7B0009387075063E1A70297B79F
:10B5B000FF1F9387E797D843FD576367E50097B769
:10B5C000FF1F23A9A79681473E858280B957EDBF0B
:10B5D0001773FFFFE702A3B097800000E780607554
:10B5E00097800000E780C0771773FFFF670063B1A3
:10B5F0001773FFFFE70203AD2A84930414020111BD
:10B600002E85B289A685214636C63A899730010033
:10B61000E780403D0DE9B24638082686CE85130501
:10B62000940497500000E780604121462C084A8529
:10B6300097300100E780003B133515000561177353
:10B64000FFFF670063AB0145D5BF1773FFFFE7023C
:10B6500003A99305450617A5FF1F1305A56A9710B3
:10B660000100E78020691773FFFF670083A9177344
:10B67000FFFFE702C3A641112EC697F0FFFFE78048
:10B68000C017B24588C141011773FFFF670063A768
:10B690001773FFFFE70203A3AA842E84978000009C
:10B6A000E780006CAA898545228597000000E78025
:10B6B000E07D83C7E4011389940899E313890403A7
:10B6C000CE85228597000000E780407C21469305C7
:10B6D0001902228597000000E780607897B7FF1F66
:10B6E000938707858C43228597100000E780C082EE
:10B6F000214693858402228597000000E78020760A
:10B700001773FFFF6700439F1773FFFFE702A39ABA
:10B71000397197F00000E780E0B49305400661E9D5
:10B7200097800000E78000606302051497A7FF1F61
:10B7300083C7075F13B7170097A6FF1F2382E65E34
:10B74000014499CFC16417A9FF1F1309697E9309AA
:10B75000400EFD1497000000E78020836342A40A96
:10B7600097F0FFFFE78060094169B7290900096A7E
:10B77000FD7A2A8B81447D199389F97B130A0A711A
:10B78000938A8AC797000000E780208063D7A404CB
:10B790001304400EB387840217A7FF1F13074779CE
:10B7A0000324070B3E948357C4016382270B184080
:10B7B0003307EB4063EAE900834744008507B3871A
:10B7C0004703D6976365F70801468145094597F019
:10B7D000FFFFE780C04AAA8B29E597400000E78079
:10B7E000808385476317F50689659385057117A5DD
:10B7F000FF1F1305255197100100E780A04F95A06A
:10B80000B30734030327090BBA9703D7C7016308AB
:10B81000970003C75700A38207002382E7000504AF
:10B8200015BF9305C500228597000000E78080E6DC
:10B830005E85228697650100938505D797F0FFFF07
:10B84000E780404F5E8597100000E780608A85049E
:10B8500015BF97A7FF1F9387A76D9C478D83858B87
:10B86000C1F721611773FFFF6700638801468545B3
:10B87000094502D002D202D402D697F0FFFFE7803A
:10B880000040AA8479DD97F00000E780E09C1389EE
:10B89000C4002A8481454A8597000000E780005F44
:10B8A0000C4041464A8597000000E780405B8329B1
:10B8B00044006385090C4E8502D802DA02DC02DE00
:10B8C00097300100E780E0382ACE141005462C0896
:10B8D00008184ECC97500000E780E00A1375F50F6A
:10B8E00051ED8355840093E525004A8597000000BB
:10B8F000E780E05E11460C104A8597000000E78063
:10B900000056014697650100938585CA268597F004
:10B91000FFFFE7802042268597000000E780407DFA
:10B920005C40A1D3014685450D4597F0FFFFE780B8
:10B930000035AA841DD548401389C4009730010002
:10B94000E78020312AC64A8597000000E780404CF6
:10B950003246636FC5004C404A8597000000E7807F
:10B96000005001468145268597F0FFFFE780803C27
:10B97000268597000000E780A077E5B58355840011
:10B98000ADB71763FFFFE702837597A7FF1F938784
:10B99000275A9C471DC193E7870017A5FF1F130572
:10B9A000653617A7FF1F2329F75897100100E78076
:10B9B00040321763FFFF6700C374DD9B17A7FF1FAB
:10B9C000232CF75697300000E780E0647DF117A53F
:10B9D000FF1F1305253397100100E780E033D1BF27
:10B9E0001763FFFFE702236D4169AA892E8AB28A95
:10B9F000368BBA8B814417ACFF1F130C6C53930C1E
:10BA0000400E7D1997F0FFFFE780205863C4A40023
:10BA100001443DA03384940383270C0B3E94835749
:10BA2000C401638627055A87D6865286CE851305BC
:10BA3000040397000000E780E0BB01C923800B00EE
:10BA400022851763FFFF6700836A8347F40185C37C
:10BA50005A87D6865286CE85130594089700000033
:10BA6000E78040B909C585472380FB00D1BF850425
:10BA700051BF835745006380071E1763FFFFE7022E
:10BA8000636401112A8497000000E780C04D09C952
:10BA900085476309F50605611763FFFF6700C36506
:10BAA00097E00000E780007C7DF58357440049471C
:10BAB000ED9BE392E7FEC145228597000000E780F9
:10BAC0004033AA84228597000000E780204F035767
:10BAD000440002CE91472A89631AF7002285970015
:10BAE0000000E780A0513C082ACC3ECE97E0000041
:10BAF000E78080765C55C5D374084A86A6850545DF
:10BB0000829751BF03574400D147E3F6E7F8032A71
:10BB10000400C169014997AAFF1F938A6A41130B68
:10BB2000400EFD1997F0FFFFE7802046634FA90EF6
:10BB30002285032A040097000000E780C042A14547
:10BB40002A89228597000000E780A02AAA842285FE
:10BB500097000000E780804A14402A86AA89780866
:10BB60002685CA8597000000E780C0E7AA8405D52E
:10BB700003C7F40189476315F7008347C10181DFDB
:10BB80005546D2851385640097300100E780E0E7D1
:10BB9000014597800000E780C01901C583D7C40123
:10BBA000A5E797A7FF1F9387A7389C4793551900D0
:10BBB000858913D73700058B01CF8983858B6399DE
:10BBC000B70001452EC697000000E780C0DBB245F4
:10BBD0004E8597800000E780601F0346C1012A84DC
:10BBE00093751900268597900000E780E03935C1EC
:10BBF000268597800000E780E018268511C0014562
:10BC000097800000E780004C97300000E780A0405C
:10BC10008547E312F5E883C754001307F00FE38C60
:10BC2000E7E68507A382F400BDB5B304690383A7E3
:10BC30000A0BBE9483D7C401638B37015546D28566
:10BC40001385640097300100E780C0D955DD0509F0
:10BC5000D1BD5DD86DB782801763FFFFE7028346D1
:10BC600097800000E780000C05C1C164014417A95A
:10BC7000FF1F1309E92B9309400EFD1497F0FFFFF6
:10BC8000E780A030634EA40017A5FF1F13058507AA
:10BC900097100100E780E0031763FFFF6700C345CB
:10BCA000330534038327090B3E958357C501638809
:10BCB00097002312050097800000E780A00C050480
:10BCC00075BF97A7FF1F9387A7269C478D83858BFA
:10BCD0008DE31763FFFFE702834017A5FF1F1305DE
:10BCE000650297100100E78020031763FFFF6700DC
:10BCF000434182801763FFFFE702633E9705000020
:10BD00009385C5A017A5FF1F1305C5FF9710010058
:10BD1000E78020EE1763FFFF6700A33E1763FFFF76
:10BD2000E702E33B8841B7E70400BC5B0505420539
:10BD30004181829709C585472300F50005051763F2
:10BD4000FFFF6700033C83C7F5FF2E858507A38FA0
:10BD5000F5FE828083C7F5FFFD1793F7F70FA38FDA
:10BD6000F5FE99EF1763FFFFE7026337B7E70400BB
:10BD7000BC571385F5FF82971763FFFF6700633891
:10BD800082801C41035745008D8FBA951CC1231238
:10BD9000B5003E85828093D78500A2051441DD8DD4
:10BDA000835745001387E6FF18C189072312F50062
:10BDB00013D685004111238FB6FEA38FC6FE410125
:10BDC000828018419307F7FF1CC183574500850700
:10BDD0002312F500A30FB7FE8280835745008D8F95
:10BDE0002312F5001C41BE950CC12E858280AA87C6
:10BDF00003D7470008410D8FAA952392E7008CC313
:10BE00008280184108453305A7408280835745004A
:10BE1000035765001D8F1C4108453385A740330536
:10BE2000A74082801763FFFFE702632B41112EC6F4
:10BE30002A8497000000E780A0FDB2456373B50037
:10BE400001A0835744000840BE952312B4003E95DC
:10BE500041011763FFFF6700C32A1763FFFFE70273
:10BE6000032841112E84B28532C697000000E78076
:10BE7000A0FB3246A28597300100E78000B941015E
:10BE80001763FFFF6700E3271763FFFFE702232520
:10BE90002E84854597000000E78000F92300850087
:10BEA0001763FFFF6700E3251763FFFFE702232304
:10BEB00041112317B100894597000000E780C0F6C3
:10BEC0008347E1002300F5008347F100A300F5005C
:10BED00041011763FFFF6700C3221763FFFFE702FB
:10BEE000032093D78500A2054111DD8D2317B100F2
:10BEF000894597000000E78020F38347E100230095
:10BF0000F5008347F100A300F50041011763FFFF2F
:10BF10006700231F1763FFFFE702631C1397850168
:10BF200093D78501C166938606F0D98F13D7850014
:10BF3000758FD98FA2053707FF00F98D4111DD8D6F
:10BF40002EC6914597000000E78000EE6C00114678
:10BF500097300100E78060AB41011763FFFF670086
:10BF6000431A1763FFFFE70283171C41854503C48B
:10BF7000070097000000E78080E622851763FFFF37
:10BF8000670023181763FFFFE70263151C41411187
:10BF9000894503C7070083C717002307E100A307EC
:10BFA000F10097000000E78080E30355E1004101C4
:10BFB0001763FFFF6700E3141763FFFFE702231215
:10BFC0001C414111894503C7070083C71700230798
:10BFD000E100A307F10097000000E78040E08357ED
:10BFE000E100410113D58700A2075D8D4205418123
:10BFF0001763FFFF6700E3101763FFFFE702230EDD
:10C000000C4141112A841146680097300100E780F5
:10C01000C09F9145228597000000E78040DCB24731
:10C02000C166938606F01397870113D58701598D52
:10C0300013D78700758F598DA2073707FF00F98F37
:10C040005D8D41011763FFFF6700A30B1C45BE9583
:10C050000CC18280AE87944391E6584101EF0CC138
:10C060005CC1828003C7570013671700A382E700F3
:10C07000B687D5B70CC3EDB7AA87084119CD1841CB
:10C08000D44398C36313D500D8C32A870346570007
:10C090009376160081E6232007008280944381CAAC
:10C0A0008C4203A847008CC363930601CCC3799AE2
:10C0B00014C3A302C7003687D1BF1C45DC471D8DC2
:10C0C000B777DBB6938777DB09853305F502420541
:10C0D00041818280F147B385F50248452E958280E3
:10C0E0008347450085072302F50082801763FFFF21
:10C0F000E702E3FE2A8409E41763FFFF6700630099
:10C1000083474400F5DBFD1793F7F70F2302F40094
:10C11000E5F71C4403D7270005072391E700DC431C
:10C1200099C3228582974C4889CD83475400898BD7
:10C1300099E71C4422859C479C439C478297232A6D
:10C1400004000040232004007DB71763FFFFE702CF
:10C1500003F98357250041112EC681EB0144228546
:10C1600041011763FFFF6700C3F9035705008147CB
:10C17000F146E305F7FEB385D702404585072E94C7
:10C180008345440008C4F5F5B247AA8481E7232A11
:10C19000040009A81C456C0022859C439C4382979F
:10C1A00048C84DDD85472312F400B2472320040020
:10C1B000231804002319F4005C485CC483D72400CE
:10C1C000FD172391F40061BF1763FFFFE70223F11E
:10C1D00097A7FF1F938707B58843232605002324CD
:10C1E0000500410597100100E78000B31763FFFFCA
:10C1F000670023F11763FFFFE70263EE17A4FF1F39
:10C20000130444B21C40411199CF9C472300B50050
:10C210002AC65CC197000000E78040FB1C40DC435D
:10C2200099C33245829741011763FFFF670063EDB1
:10C230000347450029E3584DAA877D551DCF176355
:10C24000FFFFE702C3E91CC3DC4797A6FF1F23AB30
:10C25000E6ACF156130507012390D70097050000BF
:10C260009385050297100100E780A09801451763A8
:10C27000FFFF670003E97D55828082801763FFFF1F
:10C28000E702E3E501116146814528009760FFFF61
:10C29000E780E0E797A7FF1F9387C7A89C43280084
:10C2A0009305F00FDC473EC697000000E780C0F41E
:10C2B00005611763FFFF6700C3E497A7FF1F93871C
:10C2C00067A69C43D847A1679387C702631EF70AF6
:10C2D000397106DE22DC26DA80004AD84ED652D4E6
:10C2E00056D23285B28497000000E780C0C7AA8981
:10C2F000268597000000E78020C92318A4FC268526
:10C3000097000000E78040C82319A4FC2685970009
:10C310000000E78060C783D744000A8A231AA4FC80
:10C32000858393F7F70F230EF4FC8607BD0793F779
:10C33000073F3301F1408A8A01498347C4FD63679F
:10C34000F902CE85130584FC232C54FD97000000D0
:10C35000E78080EA5281130104FCF2506254D25407
:10C360004259B259225A925A2161828026859700F9
:10C370000000E78060C193171900D6970509239044
:10C38000A7001379F90F55BF828097A7FF1F9387E6
:10C3900067999C43D847A1679387A702631AF70A56
:10C3A000397106DE22DC26DA80004AD84ED652D415
:10C3B00056D23285B28497000000E780C0BAAA89BD
:10C3C000268597000000E78020BCFD572318A4FCB9
:10C3D00026852319F4FC97000000E780E0BA83D794
:10C3E00044000A8A231AA4FC858393F7F70F230ECF
:10C3F000F4FC8607BD0793F7073F3301F1408A8AB3
:10C4000001498347C4FD6367F902CE85130584FCA7
:10C41000232C54FD97000000E78000DE52811301B9
:10C4200004FCF2506254D2544259B259225A925AE0
:10C4300021618280268597000000E780E0B4931791
:10C440001900D69705092390A7001379F90F55BF56
:10C45000828097A7FF1F9387E78C9C43D847A167EB
:10C4600089076310F70A397106DE22DC26DA8000BC
:10C470004AD84ED652D456D232853289970000001F
:10C48000E78060AEAA894A8597000000E780C0AFC8
:10C49000835749000A8A2318A4FC858393F7F70F72
:10C4A000230CF4FC8607BD0793F7073F3301F140E7
:10C4B0008A8A8144834784FD63E7F402CE851305AD
:10C4C00084FC232A54FD97000000E780E0D25281CB
:10C4D000130104FCF2506254D2544259B259225A08
:10C4E000925A216182804A8597000000E780C0A9A6
:10C4F00093971400D69785042390A70093F4F40F24
:10C5000055BF828097A7FF1F9387C7819C43D84759
:10C51000A1679387E704631EF70A397106DE22DC00
:10C5200026DA80004AD84ED652D456D23285B2840A
:10C5300097000000E78020A3AA89268597000000C5
:10C54000E78080A42318A4FC268597000000E780DC
:10C55000A0A3231AA4FC268597000000E780C0A2B0
:10C5600083D744000A8A2319A4FC858393F7F70F25
:10C57000230EF4FC8607BD0793F7073F3301F14014
:10C580008A8A01498347C4FD6367F902CE85130592
:10C5900084FC232C54FD97000000E780E0C5528105
:10C5A000130104FCF2506254D2544259B259225A37
:10C5B000925A21618280268597000000E780C09C06
:10C5C00093171900D69705092390A7001379F90F3F
:10C5D00055BF82809797FF1F9387C7749C43D847A6
:10C5E000A1679387C704631AF70A397106DE22DC54
:10C5F00026DA80004AD84ED652D456D23285B2843A
:10C6000097000000E7802096AA8926859700000001
:10C61000E7808097FD572318A4FC2685231AF4FC95
:10C6200097000000E780409683D744000A8A2319C8
:10C63000A4FC858393F7F70F230EF4FC8607BD0750
:10C6400093F7073F3301F1408A8A01498347C4FDCC
:10C650006367F902CE85130584FC232C54FD9700F3
:10C660000000E78060B95281130104FCF25062546B
:10C67000D2544259B259225A925A21618280268557
:10C6800097000000E780409093171900D69705099E
:10C690002390A7001379F90F55BF82809797FF1F4A
:10C6A000938747689C43D847A167DD076317F70462
:10C6B0001763FFFFE702A3A27971328532849700E6
:10C6C0000000E780408A2AC6228597000000E780A4
:10C6D000A08B2311A102228597000000E780A0888B
:10C6E000B2452300A102280897000000E780C0B0EF
:10C6F00045611763FFFF6700C3A082809797FF1F04
:10C70000938747629C43D847A16793878704631741
:10C71000F7041763FFFFE702839C79713285328447
:10C7200097000000E78020842AC622859700000039
:10C73000E78080852311A102228597000000E78011
:10C740008082B2452300A102280897000000E780FC
:10C75000A0AA45611763FFFF6700A39A828097979D
:10C76000FF1F9387275C9C43D847A1679387A70443
:10C770006312F7021763FFFFE702639601112800B7
:10C78000814597000000E78020A705611763FFFF40
:10C790006700239782809797FF1F9387A7589C4332
:10C7A000D847A167938757026319F7021763FFFF02
:10C7B000E702E3920111328597F0FFFFE780A07A4C
:10C7C0002308A1008145280097000000E780C0A24F
:10C7D00005611763FFFF6700C39282809797FF1F71
:10C7E000938747549C43D847A1679387E702631B0D
:10C7F000F7041763FFFFE702838E0111328532844D
:10C8000097F0FFFFE7804078AA84228597F0FFFF2A
:10C81000E7808077854709E9228597F0FFFFE78069
:10C8200080744205B337A000280081452318910089
:10C830003ECA97000000E780209C05611763FFFF58
:10C840006700238C82809797FF1F9387A74D9C4397
:10C85000D84799476313F7081763FFFFE702238858
:10C8600079713285328497F0FFFFE780C06F2AC666
:10C87000228597F0FFFFE78020712310A102228517
:10C8800097F0FFFFE780206E2301A102228597F039
:10C89000FFFFE780406DA301A102228597F0FFFF13
:10C8A000E780606C2302A102228597F0FFFFE780FA
:10C8B000806B2313A102228597F0FFFFE780A06A17
:10C8C000B2452314A102280897000000E780C09217
:10C8D00045611763FFFF6700C38282809797FF1F40
:10C8E000938747449C43D847A1679387C703631343
:10C8F000F7081753FFFFE702837E79713285328490
:10C9000097F0FFFFE78020662AC6228597F0FFFF99
:10C91000E78080672310A102228597F0FFFFE78060
:10C92000A0662311A102228597F0FFFFE780A06394
:10C930002302A102228597F0FFFFE780C062A302D5
:10C94000A102228597F0FFFFE780E0612303A102A7
:10C95000228597F0FFFFE7800061B245A303A102A3
:10C96000280897000000E780208945611753FFFFE2
:10C970006700237982801753FFFFE7024376011196
:10C980002A8497F0FFFFE780005EAA84228597F053
:10C99000FFFFE780605F228597F0FFFFE780C05EC2
:10C9A000035744008D4763F7E700228597F0FFFFA8
:10C9B000E780805D228597F0FFFFE780E05C28003C
:10C9C000A68597000000E780208305611753FFFFCD
:10C9D000670023739797FF1F9387C7349C43D847FB
:10C9E000A167FD07631FF7001753FFFFE702236FDF
:10C9F000328597000000E78040F81753FFFF67007B
:10CA0000437082809797FF1F9387C7319C43D84715
:10CA1000A167E5076315F7081753FFFFE702236CCB
:10CA200079713285328497F0FFFFE780C0532AC6C0
:10CA3000228597F0FFFFE7802055228597F0FFFFC2
:10CA4000E78080542310A102228597F0FFFFE78042
:10CA5000A053520551812311A10222852302010214
:10CA600097F0FFFFE7802050A302A102228597F0F4
:10CA7000FFFFE780404F2303A102228597F0FFFFCD
:10CA8000E780604EB245A303A102280897F0FFFF9C
:10CA9000E780807645611753FFFF670083668280D9
:10CAA0009797FF1F938707289C43D847A1679387D1
:10CAB000E703631FF7001753FFFFE7024362328566
:10CAC00097000000E78060EB1753FFFF6700636388
:10CAD00082809797FF1F9387E7249C43D847A167DD
:10CAE00093874704631EF7021753FFFFE702235F94
:10CAF00079713285328497F0FFFFE780C0462AC6FD
:10CB0000228597F0FFFFE7802048B245280897F07C
:10CB1000FFFFE780606E45611753FFFF6700635EAC
:10CB200082809797FF1F9387E71F9C43D847A16791
:10CB3000938787026310F7041753FFFFE702235A16
:10CB400079713285328497F0FFFFE780C0412AC6B1
:10CB5000228597F0FFFFE7800041B2452300A10244
:10CB6000280897F0FFFFE780206945611753FFFF12
:10CB70006700235982801753FFFFE70243560111D4
:10CB800097F0FFFFE780203EAA85280097F0FFFF7F
:10CB9000E780806605611753FFFF6700835697970C
:10CBA000FF1F938727189C43D847A167D107631FAE
:10CBB000F7001753FFFFE70283523285970000000A
:10CBC000E780A0FB1753FFFF6700A353828097976E
:10CBD000FF1F938727159C43D847A167C507631F8D
:10CBE000F7001753FFFFE702834F328597000000DD
:10CBF000E780A0F81753FFFF6700A3508280979744
:10CC0000FF1F938727129C43D847A167B907631F6B
:10CC1000F7001753FFFFE702834C328597000000AF
:10CC2000E780A0F51753FFFF6700A34D8280979719
:10CC3000FF1F9387270F9C43D847A167AD07631F4A
:10CC4000F7001753FFFFE702834932859700000082
:10CC5000E780A0F21753FFFF6700A34A82809797EF
:10CC6000FF1F9387270C9C43D84789476318F70217
:10CC70001753FFFFE702A3460111328532C897F030
:10CC8000FFFFE780402EAA85280097F0FFFFE7808E
:10CC9000A05605611753FFFF6700A3468280979750
:10CCA000FF1F938727089C43D847A1678D0763110F
:10CCB000F7041753FFFFE7028342011132853284E4
:10CCC00097F0FFFFE780202A13066100AA844C003A
:10CCD000228597300000E780C0232800A68597F0C2
:10CCE000FFFFE780605105611753FFFF6700634155
:10CCF00082809797FF1F938727039C4381CFDC4354
:10CD000091CB1753FFFFE702833D82971753FFFF35
:10CD10006700233F82801753FFFFE702433C79718E
:10CD20003C08AE843ED2A165B7070A002A843ED4EF
:10CD300048103C08DD053ED636C432C63AC297D00C
:10CD4000FFFFE780402C12474810BA8597F0FFFF9D
:10CD5000E780C01332464810B28597F0FFFFE780A6
:10CD6000E014A2464810B68597F0FFFFE780001256
:10CD7000501001478146A685228597D0FFFFE780A6
:10CD8000E04D45611753FFFF6700A3371753FFFFBF
:10CD9000E702E33401117C000329C501AE843ECAD9
:10CDA000A165B70707002A843ECC48087C00C5056A
:10CDB0003ECE97D0FFFFE78000258345D900480885
:10CDC00097F0FFFFE780800C500801478146A68559
:10CDD000228597D0FFFFE780604805611753FFFF6A
:10CDE000670023321753FFFFE702632F83C79500C5
:10CDF00093F7F707A384F50097000000E78040F958
:10CE00001753FFFF6700E32F1753FFFFE702232DA0
:10CE100079713C08AE843ED2A165B70709002A8427
:10CE20003ED448103C08938545043ED632C636C4ED
:10CE300097D0FFFFE780201DA2464810B68597F0E7
:10CE4000FFFFE780A00432464810B28597F0FFFF4D
:10CE5000E780C005501001478146A685228597D0FE
:10CE6000FFFFE780A03F45611753FFFF670063297D
:10CE70001753FFFFE702A32683C7950041112A84B9
:10CE800093F7F707A384F50032852EC697F0FFFFCE
:10CE9000E780800F85672AC46370F50297700000F1
:10CEA000E78020E92246B24509ED114781462285F7
:10CEB00097000000E78060E641011753FFFF67001D
:10CEC000432401478346F501DDB71753FFFFE7020F
:10CED000631F01113C003ECAB7070A003ECC3C006C
:10CEE0003ECE83C79500AA89328593F7F707A384BE
:10CEF000F5002E8497F0FFFFE78000098567637DCA
:10CF0000F504A165AA8493858504480897D0FFFF9E
:10CF1000E780600F268597700000E78080E12A890E
:10CF200029E19145480897F0FFFFE78020F6A685A4
:10CF3000480897F0FFFFE78060F7CA85480897F038
:10CF4000FFFFE780A0F4014781465008A2854E8587
:10CF500097D0FFFFE780803005611753FFFF670020
:10CF6000A3198145480897F0FFFFE78020F20349A5
:10CF7000090275BF1753FFFFE702C31479711C1034
:10CF80003ECAB7070F003ECC404D1C10AA84AE89A4
:10CF90004808994532C636893ECE97D0FFFFE780D4
:10CFA000800632464808B28597F0FFFFE78000EE22
:10CFB000630C0902A545480897F0FFFFE780C0E62B
:10CFC0002546CA8597200100E78020A45008014724
:10CFD0008146CE85268597D0FFFFE78020284561D2
:10CFE0001753FFFF670043118355C402480897F0A9
:10CFF000FFFFE780A0EB0355E402814505C58547A7
:10D0000085456301F502C167FD179305F00F630BBA
:10D01000F5007D1597700000E780208E93051500C0
:10D0200093F5F50F480897F0FFFFE78020E683456A
:10D030000403480897F0FFFFE78040E583451403A9
:10D04000480897F0FFFFE78060E483552403480811
:10D0500097F0FFFFE78080E583554403480897F089
:10D06000FFFFE780A0E49DB71753FFFFE702230708
:10D0700083C795008146014693F7F707A384F5001F
:10D0800097000000E78040EF1753FFFF670063073A
:10D090001753FFFFE702A30479713E841C103ECAB8
:10D0A0002E89B7070F00A1653ECCFD051C10AA8490
:10D0B000480842C03AC23ECE36C432C697D0FFFFBF
:10D0C000E78060F432464808B28597F0FFFFE780BA
:10D0D000E0DBA2464808B68597F0FFFFE78000DD59
:10D0E00012474808BA8597F0FFFFE78020DC024826
:10D0F000630C08029145480897F0FFFFE780C0D213
:10D100001146A28597200100E78020905008014732
:10D110008146CA85268597D0FFFFE78020144561A8
:10D120001753FFFF6700E3FD8945480897F0FFFFAD
:10D13000E78080CF834704002300F5008347140075
:10D14000A300F500E1B71753FFFFE702A3F783C77A
:10D15000950001112A8A93F7F707A384F500328519
:10D16000AE8432C697F0FFFFE78000E232462A899C
:10D17000328597F0FFFFE78000DF85676373F90270
:10D18000AA894A8597700000E780A0BA2A8419ED21
:10D19000114781464A86A685528597000000E780A0
:10D1A000C0B705611753FFFF670003F59387E9FFD9
:10D1B00093F7F70F0547E366F7FE8347F50195EB15
:10D1C0008947E380F9FE8346F401528501474A8688
:10D1D000A68597000000E78040B4A167D9074808FA
:10D1E0003ECC230A010002CE97000000E780A0B0E9
:10D1F0004DBF639EE7008947639EF90093071020A7
:10D20000231FF50097700000E780C0B76DBF094786
:10D21000E39BE7FA8D47E398F9FA228597700000BF
:10D22000E78080DF9797FF1F938707CF9C4399E79D
:10D230009797FF1F938707B89C4399C703D50400AE
:10D2400097800000E780A0CE231F040022855DBFE9
:10D250001753FFFFE702A3E801113C003ECAB707DE
:10D260000B003ECC3C003ECE83C795002A89328518
:10D2700093F7F707A384F500AE8497F0FFFFE780EC
:10D28000A0D093170501C187635AF006A1652A84CF
:10D290009385E502480897D0FFFFE780C0D6A285B6
:10D2A000480897F0FFFFE78060C09797FF1F9387BC
:10D2B00067B09C43A9EB01449375F40F480897F0BD
:10D2C000FFFFE780A0BC9355844093F5F50F480815
:10D2D00097F0FFFFE78080BB9355044193F5F50F6E
:10D2E000480897F0FFFFE78060BA01478146500881
:10D2F000A6854A8597D0FFFFE78040F60561175362
:10D30000FFFF670003E0416585460546A2857D1560
:10D3100097500000E78060BD59DD5105970001007E
:10D32000E780808F130440063344850271B717539A
:10D33000FFFFE702C3DA0111B70706003EC683C745
:10D34000950021642A8993F7F707A384F500AE843A
:10D3500028009305A4040AC40AC897D0FFFFE780F9
:10D3600080CA300001478146A6854A8597D0FFFFD5
:10D37000E780C0EE97E0FFFFE780E011130494041C
:10D38000480822CC230A010002CE97000000E78063
:10D39000809605611753FFFF6700A3D61753FFFF61
:10D3A000E70243D2C1642A8901449799FF1F9389F8
:10D3B00029B8130A8002FD1497E0FFFFE780E0BD63
:10D3C0006347A40001451753FFFF6700E3D2B3078B
:10D3D000440303A7C90ABA9703D707006306970057
:10D3E00083D72700638427010504F9B70545E1BF0A
:10D3F0001753FFFFE70203CD2A8A2E8999C123A084
:10D40000050081498144979AFF1F938A2A92614BB4
:10D4100097E0FFFFE780A0BE63C7A4004E851753C7
:10D42000FFFF670063CD3384640383A70A003E9443
:10D430008357040099E763040900232089008504C9
:10D44000C1BF4146D2851305440097100100E78013
:10D45000605975F5A289E5B71753FFFFE70283C648
:10D4600039717C083ED4B7070A003ED67C083ED806
:10D4700083C795002A8A328593F7F707A384F500BE
:10D480002E8932C697F0FFFFE78000B0856763738F
:10D49000F5083246AA84328597F0FFFFE780A0ACFA
:10D4A0008547AA8963E8A706A165938585042810A6
:10D4B00097D0FFFFE78020B5268597700000E780B2
:10D4C00040872A8429ED9145281097F0FFFFE780D7
:10D4D000E09BA685281097F0FFFFE780209DCE8572
:10D4E000281097F0FFFFE780609A014781463010CF
:10D4F000CA85528597D0FFFFE78040D6A167938702
:10D50000770448183EDC230A010202DE97F0FFFF91
:10D51000E780607E21611753FFFF6700E3BD81450F
:10D52000281097F0FFFFE7806096A685281097F0F7
:10D53000FFFFE780A0979797FF1F9387E7D59C434E
:10D5400081CB22856389090097D00000E7804024C1
:10D550008345040271B797D00000E780C022CDBF99
:10D560001753FFFFE70203B683C795004111AA894D
:10D5700093F7F707A384F5003285AE84328A97F0DB
:10D58000FFFFE78060A08567637FF5022A899760C7
:10D590000000E780007A2A84914631C58347F5016F
:10D5A00005476387E70291C70D476366F704AD46F9
:10D5B0001DA89305050303250A00414697100100A5
:10D5C000E78040420DE941011753FFFF6700C3B2F6
:10D5D0009305950803250A00414697100100E7804E
:10D5E0006040814669F54A86A6854E859700000011
:10D5F000E780C081C9BF83250A001305940897708E
:10D600000000E780A02919C1C146F1BF9797FF1F0D
:10D61000938787909C4399E79787FF1F9387877924
:10D620009C4399C7228597800000E780208A69FD86
:10D630008547A30FF400228597B00000E78060843F
:10D64000228597600000E780E0734E8581464A8618
:10D65000A68597F0FFFFE780607BA167938757045B
:10D6600048003EC42302010002C697F0FFFFE78096
:10D67000806891BF1753FFFFE702E3A383C79500BC
:10D680004111AA8993F7F707A384F50032852E8903
:10D69000B28A97F0FFFFE780208F85676374F50EED
:10D6A000AA8497600000E780C0682A840DED416B72
:10D6B000014A979BFF1F938BAB87130C400E7D1B7A
:10D6C00019A833048A0383A70B0B3E948357C40124
:10D6D00063836705050A97E0FFFFE780008BE3425D
:10D6E000AAFE95460DA08357C50163969702930540
:10D6F000050303A50A00414697100100E780802E2C
:10D70000994611E181462686CA854E8597F0FFFF2E
:10D71000E780C06F85A883A50A00130504039770EE
:10D720000000E780A017C14679FD2285231E9400E2
:10D7300097A00000E780E074228597600000E780F2
:10D7400060649797FF1F938727B59C43A9C3230065
:10D750000402228597D00000E78040F04E85814684
:10D760002686CA8597F0FFFFE780406AA167938706
:10D77000070448003EC42302010002C697F0FFFFE1
:10D78000E780605741011753FFFF670043968947C1
:10D790002300F402E1B7397106DE22DC4AD88000AA
:10D7A00052D456D25AD026DA4ED65ECE2E8A32893E
:10D7B0002A8B97D0FFFFE780407A060571054199D3
:10D7C0008A8A3301A140232224FC231404FC97D02D
:10D7D000FFFFE780807883479A000605350593F7B9
:10D7E000F7072315A4FCA304FA004A85232624FC8A
:10D7F00097E0FFFFE780407993170501C1876340F9
:10D80000F0025681130104FCF2506254D254425982
:10D81000B259225A925A025BF24B21618280AA8449
:10D820004A8597E0FFFFE7802076AA894A8597E03E
:10D83000FFFFE7806075A1659385C5022A891305FE
:10D8400044FC97C0FFFFE780007C268597C0FFFF60
:10D85000E7804070854511C94A86CE8597C0FFFF95
:10D86000E780C069AA8B21E98945130544FC97E04C
:10D87000FFFFE780A061A685130544FC97E0FFFF4A
:10D88000E780C062CE85130544FC97E0FFFFE78088
:10D89000E061CA85130544FC97E0FFFFE780006163
:10D8A00001478146130644FCD2855A8597D0FFFF75
:10D8B000E780C09AB9B78145130544FC97E0FFFFA4
:10D8C000E780C05CA685130544FC97E0FFFFE78076
:10D8D000E05DCE85130544FC97E0FFFFE780005D27
:10D8E000CA85130544FC97E0FFFFE780205C814474
:10D8F00097D0FFFFE7806066E3D4A4FA83A70B010B
:10D9000013971400BA9783D5070099C5130544FCF3
:10D9100097E0FFFFE78080598504D9BF797106D66B
:10D9200022D44AD000184ECE52CC56CA26D25AC85B
:10D93000AE893289AA8A97D0FFFFE7800062060588
:10D94000690541990A8A3301A140232A24FC231C3A
:10D9500004FC97D0FFFFE780406083C7990006056D
:10D960002D0593F7F707231DA4FCA384F9004A852E
:10D97000232E24FC97E0FFFFE78000619317050149
:10D98000C187634FF0005281130104FDB25022544D
:10D9900092540259F249624AD24A424B456182800E
:10D9A000AA844A8597E0FFFFE780005EA165938522
:10D9B000A5022A89130544FD97C0FFFFE780A064F4
:10D9C000268597C0FFFFE780E058854509C9CA85CD
:10D9D00097C0FFFFE78080552A8B29E18945130511
:10D9E00044FD97E0FFFFE780604AA685130544FDEC
:10D9F00097E0FFFFE780804BCA85130544FD97E061
:10DA0000FFFFE780A04A01478146130644FDCE850B
:10DA1000568597D0FFFFE7806084B5B78145130531
:10DA200044FD97E0FFFFE7806046A685130544FDAF
:10DA300097E0FFFFE7808047CA85130544FD97E024
:10DA4000FFFFE780A046814497D0FFFFE780E050CA
:10DA5000E3DBA4FA83270B0113971400BA9783D54D
:10DA6000070099C5130544FD97E0FFFFE7800044D8
:10DA70008504D9BF1743FFFFE7026366834745006C
:10DA8000404DD5EFFD575DC483469400094763635D
:10DA9000D70A0346B400854663EEC6088306E40051
:10DAA00063CA06085C45F9562390D7009787FF1F85
:10DAB00083C7072899E3A304E4009787FF1F938790
:10DAC000672F9C4381E78947A306F4009787FF1FD0
:10DAD0009387877C9C4381E789472306F400970559
:10DAE000000093854506AA841305040197F0000001
:10DAF000E7802010FD57231AF40281471CDC0148FF
:10DB00009787FF1F23A287229787FF1F93870722EC
:10DB1000232E040304C0804397D0FFFFE780204EEC
:10DB200061463306C502814522859740FFFFE780A5
:10DB3000005E81473E851743FFFF6700835CFD570A
:10DB4000D5BF1743FFFFE70283592A8403554502D7
:10DB500097600000E780E01D19E5231E04001743CD
:10DB6000FFFF6700035A8357E401F5DB930504FFC9
:10DB700017450100130585DD97E00000E780E014FC
:10DB8000F9BF1743FFFFE70283552E89A1654111B5
:10DB90009385E5032A8436C432C6BE843AC297C050
:10DBA000FFFFE780404612472285BA8597E0FFFFD6
:10DBB000E780C02D32462285B28597E0FFFFE780DF
:10DBC000E02EA2462285B68597E0FFFFE780002E73
:10DBD000630309029145228597E0FFFFE780C02497
:10DBE0001146A68597100100E78020E24101174306
:10DBF000FFFF670003518945228597E0FFFFE7801B
:10DC0000A02283C704002300F50083C71400A300EB
:10DC1000F500E9BF1743FFFFE702634C83C7950098
:10DC2000444D054793F7F707A384F5001C424111C3
:10DC300083C707006367F7062E842A89B1C003C72C
:10DC4000D400630FF7021787FF1F1307A7161843A7
:10DC500005C3A386F40097A00000E780404A83C76D
:10DC6000D40099E741657D1597400000E78040307A
:10DC700083D72403918B89C797E00000E780C01306
:10DC80004A85A28597F0FFFFE7808010A167C10752
:10DC900048003EC42302010002C697F0FFFFE78060
:10DCA000800541011743FFFF6700A3451743FFFFAE
:10DCB000E702E34203D745008D47AA8441112E8431
:10DCC00032892E8563E3E70297E0FFFFE780C02BF0
:10DCD000AA8523000900268597C0FFFFE78000255D
:10DCE00041011743FFFF6700C34197E0FFFFE78053
:10DCF000A0292AC6228597E0FFFFE780E028B245E9
:10DD000085472A862300F900268597C0FFFFE78014
:10DD1000E01EF9B7397106DE22DC26DA80004ED625
:10DD200052D456D24AD85AD05ECEAE89B284AA8A8C
:10DD300097D0FFFFE7806021060513052502419972
:10DD40000A8A3301A140232224FC231404FC97D027
:10DD5000FFFFE780801F83C7990006054D0593F7F5
:10DD6000F7072315A4FCA384F9002685232624FCA9
:10DD700097E0FFFFE780402193170501C1876340CB
:10DD8000F0025281130104FCF2506254D254425901
:10DD9000B259225A925A025BF24B21618280AA8BBD
:10DDA00003AB040097C0FFFFE780C01A51E583D79B
:10DDB000440001498544F11793B71700A301F4FC0F
:10DDC000834734FCA165C9C79385E504130544FC6A
:10DDD00097C0FFFFE7802023A685130544FC97E04A
:10DDE000FFFFE780A00ADE85130544FC97E0FFFFF4
:10DDF000E780C00B834734FC114691E30946DA857E
:10DE0000130544FC97E0FFFFE78060058144630A47
:10DE10000900416B7D1B97D0FFFFE780001363CCA7
:10DE2000A40201478146130644FCCE85568597C05F
:10DE3000FFFFE780A042B1B7A685130634FC970028
:10DE40000000E780E0E6933415002A8986048DBF40
:10DE50009385C504A5BF8327C90013971400BA97FB
:10DE600083D5070063886501130544FC97E0FFFF35
:10DE7000E780C003850445B71743FFFFE702A323EC
:10DE800079711C103EC4B7070F003EC61C103EC877
:10DE900083C79500AA8A328593F7F707A384F50014
:10DEA000AE89328497E0FFFFE780000E93170501EB
:10DEB000C187635AF0062A8A228597E0FFFFE78030
:10DEC000A00C2A895285032B040097C0FFFFE7802E
:10DED000600839ED8357440081440544F11793B736
:10DEE0001700A303F10083457100DA872287CA86F1
:10DEF0005286280097000000E780E0C8014781466D
:10DF00003000CE85568597C0FFFFE7802035A1679A
:10DF10009387D70348083ECC230A810026CE97F08A
:10DF2000FFFFE78040DD45611743FFFF6700231CCB
:10DF3000A2851306710097000000E78060D7AA84CD
:10DF4000094455D13544E30055FB4A8597F0FFFF5E
:10DF5000E78000450D4441D9014497D0FFFFE78099
:10DF6000C0FE634DA400C16B0144FD1B97D0FFFFB1
:10DF7000E780A0FD634EA4001544B5B7DC44131739
:10DF80001400BA9783D70700638327030504F1B70A
:10DF9000D84493171400BA9703D70700631B77017F
:10DFA00023902701268597A00000E78080DB0144AD
:10DFB0001DBF050465BF1743FFFFE702A31083C71A
:10DFC000950041112A8A93F7F707A384F50032855B
:10DFD0002E89328497E0FFFFE78000FB931705014D
:10DFE000C1876353F006AA89228597E0FFFFE78087
:10DFF000A0F92311A1004E85832A040097C0FFFFDA
:10E00000E78040F539E58357440085440144F11722
:10E0100093B71700A300F100034811000357210034
:10E02000D6875285CE862686CA8597F0FFFFE78081
:10E030006006A167F10748003EC42302910022C692
:10E0400097F0FFFFE78020CB41011743FFFF6700F8
:10E05000A30AA2851306110097000000E78040C5BF
:10E060002A84894455D98357210011678544BA977A
:10E07000C2071167C1831307F7EFE36FF7F89787BC
:10E08000FF1F938767E99C4381CB854513052100DA
:10E0900097500000E7802075835521002285814438
:10E0A00097C0FFFFE780A0E125D923100500228556
:10E0B00097A00000E78040CD85B71743FFFFE70238
:10E0C00083FF83C7950041112A8B93F7F707A38439
:10E0D000F50032852E8A328497E0FFFFE780C0EAA0
:10E0E00093170501C1876351F006AA8A228597E03C
:10E0F000FFFFE78060E92A895685832B040097C0DB
:10E10000FFFFE78020E531E5835744008144054463
:10E11000F11793B71700A301F10003483100DE8720
:10E120005A854A87D6862286D28597F0FFFFE780F8
:10E1300060F6A167ED0748003EC42302810026C6B1
:10E1400097F0FFFFE78020BB41011743FFFF670007
:10E1500003FAA2851306310097000000E78040B55E
:10E16000AA8409445DD99167CA97C2071167C18320
:10E170001307F7EF0544E362F7FACA8597C0FFFF7C
:10E18000E780E0D3014451F9814997D0FFFFE78050
:10E19000C0DC63DBA900984893971900BA9703D7AE
:10E1A000070005EF2390270197D0FFFFE780E0DA13
:10E1B0001544E384A9F6268597A00000E780C0BC3B
:10E1C0009787FF1F938747D59C430144B9D74A855A
:10E1D00097500000E780C05889B785097DB717437D
:10E1E000FFFFE70223EE79713E847C083EC82E8A49
:10E1F000B7071400A1653ECAE5057C08AA8908088E
:10E2000036C4428932C6BA8AC6843ECC97C0FFFF64
:10E21000E78060DFCA85080897E0FFFFE78000C756
:10E2200032460808B28597E0FFFFE78020C8A24683
:10E23000630A09049D45080897E0FFFFE780C0BE18
:10E240001D4681459740FFFFE78060EC63890A081F
:10E250009145080897E0FFFFE78000BD1146A685BD
:10E2600097000100E780607A100801478146D28557
:10E270004E8597C0FFFFE78060FE45611743FFFFB3
:10E28000670083E7B685080897E0FFFFE78000C2D4
:10E290001C400808D8439355C7018589120751834C
:10E2A000B205D98D97E0FFFFE78040C01C40080809
:10E2B00083C5870097E0FFFFE78040BD1C4008084A
:10E2C00083C5A70097E0FFFFE78040BC1C4008081B
:10E2D00083C5970097E0FFFFE78040BB85BF894576
:10E2E000080897E0FFFFE78020B483C704002300FD
:10E2F000F50083C71400A300F500BDB71743FFFF67
:10E30000E70243DC83C795004111AA8993F7F70719
:10E31000A384F5003285AE84328497E0FFFFE78066
:10E32000A0C693170501C187635DF0042A89032AFB
:10E33000040097C0FFFFE780E0C119E9835744005C
:10E340000548F11793B71700A307F100814631A8DC
:10E350001306F100A28597000000E78060951DC5B7
:10E360001C459DC783D6470001480347F10093072A
:10E370008500D2884A86A6854E8597000000E780F2
:10E3800040E641011743FFFF670003D709487DBFFF
:10E390001D486DBF1743FFFFE702C3D265715C08DC
:10E3A0003EC4B7077B013EC65C083EC883C79500E4
:10E3B0002A8A328593F7F707A384F500AE8997E0A0
:10E3C000FFFFE78040BA8357E100E1C78945280095
:10E3D00097C0FFFFE78020C38145280097E0FFFF3B
:10E3E000E780C0AA97C0FFFFE78000C99787FF1F9B
:10E3F000938787EA9C431784FF1F03446493AA848E
:10E400003334800099C3136424009787FF1F9387D8
:10E41000679A9C4399C3136444009787FF1F9387AF
:10E42000A7AF9C4399C31364840083D504002800DC
:10E43000014997E0FFFFE78060A783D5240028000B
:10E4400097E0FFFFE78080A683D54400280097E08F
:10E45000FFFFE780A0A597D0FFFFE78000AB9315F3
:10E460000501C181280097E0FFFFE78020A4A28575
:10E47000280097E0FFFFE78060A39C446360F902F7
:10E48000014781463000CE85528597C0FFFFE78067
:10E49000E0DC59611743FFFF670003C6DC44131437
:10E4A000490028003E9497E0FFFFE780609683478D
:10E4B00044000347540089070607BA978607E36AB2
:10E4C000F5FC835524002800814A97E0FFFFE78090
:10E4D000E09D83454400280097E0FFFFE780009B14
:10E4E00083455400280097E0FFFFE780209A834788
:10E4F000440063C9FA00814A8347540063C1FA02A9
:10E500000509A5BF1C4413975A002800BA9783D564
:10E510000700850A97E0FFFFE7804099C9BF032BFA
:10E52000C40093975A0028003E9B83552B00850A10
:10E5300097E0FFFFE780809783550B00280097E066
:10E54000FFFFE780A0964DBF1743FFFFE70223B907
:10E550005C4993E717005CC997A00000E78020B6EC
:10E560001743FFFF6700E3B91743FFFFE70223B735
:10E570002E84814597F0FFFFE780C0E705C58357EC
:10E580000500FD172310F50009C48357250023104B
:10E59000F40097000000E78060FB01451743FFFF90
:10E5A000670023B631457DD823100400C5BF17434B
:10E5B000FFFFE70223B183C7950041112A8A93F731
:10E5C000F707A384F50032852E89328497E0FFFF98
:10E5D000E780809B93170501C1876356F006AA89DF
:10E5E000C145228597E0FFFFE780A0802A8B4E85FA
:10E5F000832A040097C0FFFFE780C09531E9835765
:10E600004400231101000544F11793B71700A3003C
:10E61000F10081440348110003572100D687528539
:10E62000CE862286CA8597F0FFFFE780A0A6A16765
:10E630009387170248003EC42302810026C697E054
:10E64000FFFFE780406B41011743FFFF6700C3AA4C
:10E6500013061100A28597F0FFFFE7806065AA848A
:10E6600009E523110100094475B7930521005A8576
:10E6700097000000E78080EF835721002A84D9DBD0
:10E680009787FF1F938747899C4381CB8545130557
:10E69000210097500000E780001583552100268552
:10E6A000314497C0FFFFE78080812DD523100500FE
:10E6B000268597900000E780206D0144A1BF174395
:10E6C000FFFFE702C3A141112E896C00AA8402C694
:10E6D00097F0FFFFE78000D20DC103570500050743
:10E6E0002310E50097000000E78040E681473E8563
:10E6F00041011743FFFF6700C3A03247954765DB21
:10E70000CA85268597300000E780400DC147E34069
:10E7100005FE3244854741462310F4008357090023
:10E72000A685130544002311F40097000100E7803B
:10E73000C02D228545BF1743FFFFE702A39883C77B
:10E7400095004111AA8A93F7F707A384F500328553
:10E75000AE89328497E0FFFFE780008393170501BD
:10E76000C1876356F0062A8AC145228597D0FFFFEC
:10E77000E7802068AA845285032B040097B0FFFF2E
:10E78000E780407D31E9835744002311010085442F
:10E79000F11793B71700A300F100014403481100DB
:10E7A00003572100DA875685D2862686CE8597F0D4
:10E7B000FFFFE780208EA1679387070248003EC4D1
:10E7C0002302910022C697E0FFFFE780C05241017B
:10E7D0001743FFFF67004392A2851306110097F0CD
:10E7E000FFFFE780E04C2A8409E5231101008944FA
:10E7F00075B726859305210097000000E78060EC3F
:10E80000AA8449FD83552100228597B0FFFFE78048
:10E81000006B49F5014997C0FFFFE7800074635D15
:10E82000A900184893171900BA9703D707000DEFEE
:10E83000035721002390E70097C0FFFFE780E071B6
:10E84000630625039777FF1F9387076D9C4399C73E
:10E850000355210097500000E78080F022859790B3
:10E860000000E78060521DBF050975B795443DB7AC
:10E8700005C19307F00F630FF500C547630CF50062
:10E880009307F5FF05453315F50042054181828068
:10E890000145828041657D158280B9E91743FFFFFC
:10E8A000E702E38303450603328497000000E78014
:10E8B00060FC9305803EB305B502C205C18181CDE0
:10E8C0000357E402854763F8E7001305040197E066
:10E8D0000000E78020428357E40241677D1763858B
:10E8E000E700FD172317F4021743FFFF670063815A
:10E8F00082801733FFFFE702037C004283C7950045
:10E90000444D0349140093F7F707A384F5008347A8
:10E910000400220911673369F900A167B347F900C0
:10E9200041112A8BAE8A63ECE70E8347240013075C
:10E93000C00EB91793F7F70F6373F710034734004E
:10E94000C14763EEE70E834744001307E00793C710
:10E9500007086371F70C8349840083477400A20998
:10E96000B3E9F900856763F7F90A034A640083474E
:10E9700054004E85220A336AFA0097500000E7805F
:10E98000403B61C123962403834B3400137AFA0081
:10E99000239A34032388740323994403938904013D
:10E9A000631C090023A60402239804024E8597E005
:10E9B0000000E78060363DA0034924004A859700A7
:10E9C0000000E78020EB2397A402834744004E8594
:10E9D000A388F402E38D0BFCE30B09FC97E0000035
:10E9E000E780202F97900000E78000738146014662
:10E9F000D6855A8597E0FFFFE7800058A167938787
:10EA000097033EC423020100480002C697E0FFFFBF
:10EA1000E780602E41011733FFFF6700436D854497
:10EA2000A2862686D6855A8597E0FFFFE780C054E8
:10EA3000A167938797033EC423029100F1B7BD44B9
:10EA4000C5B79144F1BF1733FFFFE702A367011178
:10EA50001C08404D3EC2B7070F003EC41C083EC60E
:10EA60002A89AE8997C0FFFFE78000D7585C1C5CFD
:10EA70006346B70E6394E50063E2A70E3385A740B3
:10EA8000B3B7A700B305B7401306803E81469D8DFE
:10EA900097000100E78080B793140501C180A1654C
:10EAA0009385C503480097B0FFFFE780C0558145B7
:10EAB000480097D0FFFFE780603D8355040448007D
:10EAC00097D0FFFFE780803E83552404480097D00D
:10EAD000FFFFE780A03D814589CCC167FD17930505
:10EAE000F00F6388F400268597500000E780E0E08F
:10EAF000AA85480097D0FFFFE780403903554404BA
:10EB0000814501CDC167FD179305F00F6307F5003F
:10EB100097500000E78060DEAA85480097D0FFFF8D
:10EB2000E780C03683456404480097D0FFFFE78044
:10EB3000E03583457404480097D0FFFFE780003537
:10EB4000500001478146CE854A8597B0FFFFE78098
:10EB5000E07005611733FFFF6700035A814481B7F6
:10EB60001733FFFFE702A35783C7950093F7F70713
:10EB7000A384F50097000000E78020ED1733FFFF26
:10EB8000670023581733FFFFE702C35383C795007D
:10EB90004111404D93F7F707A384F5002A8A328587
:10EBA000B284AE8997D0FFFFE780003E2A8B26858E
:10EBB00097D0FFFFE780403D2A89268597D0FFFF49
:10EBC000E780603A93170B0163CA0702E177CA979F
:10EBD000C207C183116763E3E70293070910C20705
:10EBE000C1831307B00F637BF70093170901C18737
:10EBF000AA8A634AF000C54763FE570141011733F3
:10EC0000FFFF6700634F97B0FFFFE7802025E31702
:10EC100025FFD5B763080B026306090281446389A7
:10EC20000A02B7077F0023106405231124057CC066
:10EC3000568597000000E780E0C39304803EB3044C
:10EC4000950239A0B7077F00232004047CC08144CB
:10EC50000355240497E00000E780A0A3A1C497C057
:10EC6000FFFFE78060B7269593D7F44133379500CF
:10EC7000AE97BA9708DC5CDCCE8552859700000021
:10EC8000E780A0DC99E023220404A1679387B703FF
:10EC900048003EC42302010002C697E0FFFFE78060
:10ECA0008005A9BF814701481CDC232E0403E9B776
:10ECB0001733FFFFE702A34297C0FFFFE78020342E
:10ECC000E1473305F502914597500000E78000C504
:10ECD000E55711C59777FF1F23AAA70481473E85F3
:10ECE0001733FFFF6700E34185471777FF1F2301B5
:10ECF000F70482801733FFFFE702633E9777FF1F19
:10ED00009387870280433DC0835704046390A7061E
:10ED100083572404639CB7043689B28497C0FFFFED
:10ED2000E78080AB5C5C63C3B7046395B7001C5C91
:10ED300063EEA7028347640463F3F400A68723030A
:10ED4000F4048347740463F39700A687A303F404D1
:10ED50008357440441677D176385E70085072312C5
:10ED6000F4043C4481C7CA85268582971733FFFF88
:10ED7000670023399777FF1F938707FB9C43014563
:10ED800099C303C5870082801733FFFFE70223354D
:10ED90000111B70707003EC683C79500584D0AC446
:10EDA00093F7F7070AC8A384F5002A89AE8411CB2C
:10EDB0001C4283C707002304F70097900000E780F8
:10EDC0000034216493055402280097B0FFFFE780C8
:10EDD000802397000000E78020FAAA85280097D0BA
:10EDE000FFFFE780A00A300001478146A6854A85DB
:10EDF00097B0FFFFE780804613044402480822CC06
:10EE0000230A010002CE97E0FFFFE780C0EE056114
:10EE10001733FFFF6700E32E1733FFFFE702232CB2
:10EE200001117C003ECAB70707003ECC7C003ECEF5
:10EE300083C795002E84AA8493F7F707A384F5006F
:10EE4000A16593855502480897B0FFFFE780A01B96
:10EE500097000000E78040F2AA85480897D0FFFF9E
:10EE6000E780C002500801478146A285268597B0F9
:10EE7000FFFFE780A03E05611733FFFF67006328AF
:10EE80009777FF1F938747EA9C43094599C303C5BA
:10EE9000970082809777FF1F938707E99C43094576
:10EEA00099C303C5D70082809777FF1F9387C7E771
:10EEB0009C43014599C303C5A70082801733FFFF18
:10EEC000E70243200111B70708003EC683C795003B
:10EED000404D0AC493F7F7070AC8A384F5002A89AE
:10EEE000AE8429C41442854703C7060063E0E70ADD
:10EEF00083479400094681496380C702B307F740FE
:10EF0000A304E400B339F00083C716002305F4001E
:10EF100097900000E780A01E03572403058B19C7B4
:10EF20006386090097D00000E78000E9216493051B
:10EF30008402280097B0FFFFE780E00C97000000F4
:10EF4000E78040F4AA85280097D0FFFFE78000F40F
:10EF500097000000E78080F5AA85280097D0FFFF82
:10EF6000E780C0F2014781463000A6854A8597B008
:10EF7000FFFFE780A02E13047402480822CC230A66
:10EF8000010002CE97E0FFFFE780E0D6056117336E
:10EF9000FFFF670063161733FFFFE70243140111F9
:10EFA0007C003ECAB70708003ECC7C003ECE83C73B
:10EFB00095002E84AA8493F7F707A384F500A16532
:10EFC00093858502480897B0FFFFE780C00397004C
:10EFD0000000E78020EBAA85480897D0FFFFE78074
:10EFE000E0EA97000000E78060ECAA85480897D027
:10EFF000FFFFE780A0E9500801478146A2852685EA
:10F0000097B0FFFFE780802505611733FFFF67009A
:10F01000430F9777FF1F938727D19C43014599C3DF
:10F0200003C5B70082801733FFFFE702430B0111CE
:10F03000B70707003EC683C79500404D0AC493F743
:10F04000F7070AC8A384F5002A89AE8405C81C42C4
:10F05000054783C707006368F7060347B400630FDB
:10F06000F700A305F40097900000E780400983476C
:10F07000B400B9CF97D0FFFFE78040BE216493056D
:10F08000B400280097B0FFFFE780E0F7970000008A
:10F09000E78060F8AA85280097D0FFFFE78000DFAF
:10F0A000014781463000A6854A8597B0FFFFE7807B
:10F0B000E01A2904480822CC230A010002CE97E076
:10F0C000FFFFE78040C305611733FFFF670063035D
:10F0D00097D0FFFFE78020BF55B71733FFFFE70248
:10F0E000030001117C003ECAB70707003ECC7C003C
:10F0F0003ECE83C795002E84AA8493F7F707A38496
:10F10000F500A165AD05480897B0FFFFE780A0EFC7
:10F1100097000000E78020F0AA85480897D0FFFFFD
:10F12000E780C0D6500801478146A285268597B062
:10F13000FFFFE780A01205611733FFFF670063FC44
:10F140009777FF1F938747BE9C43094599C303C523
:10F15000C70082801733FFFFE70263F801117C00CC
:10F16000AE843ECAA165B70707002A843ECCD1050C
:10F170007C0048083ECE97B0FFFFE780C0E89700CC
:10F180000000E78020FCAA85480897D0FFFFE780B1
:10F19000E0CF500801478146A685228597B0FFFF42
:10F1A000E780C00B05611733FFFF670083F5173356
:10F1B000FFFFE702C3F283C7950093F7F707A38425
:10F1C000F50097000000E78020F91733FFFF670084
:10F1D00043F31733FFFFE702E3EE83C795000329EC
:10F1E000C501411193F7F707A384F5001C4283C9B9
:10F1F0000700854763E637079777FF1F9387C7099F
:10F200009C432E84AA8485CF97000000E78080F37A
:10F2100089476306F502630409028347C9006380D6
:10F2200037032306390197900000E78040ED8357AC
:10F230002903898B89C797D00000E780E0B726852E
:10F24000A28597000000E78020F1A167CD07480064
:10F250003EC42302010002C697E0FFFFE780A0A999
:10F2600041011733FFFF670023E99777FF1F93875B
:10F27000A7AB9C431D4599C303C5E70082801733A4
:10F28000FFFFE702C3E50111B70707003EC683C7CA
:10F290009500584D0AC493F7F7070AC8A384F500F0
:10F2A0002A89AE8415C71C4283C70700939687013D
:10F2B000E18663C4060685466381D7068346E70078
:10F2C0006388F6002307F70097900000E78020E3AB
:10F2D00021649305E400280097B0FFFFE780A0D2E7
:10F2E00097000000E780A0F8AA85280097D0FFFFCC
:10F2F000E780C0B9014781463000A6854A8597B0AE
:10F30000FFFFE780A0F53504480822CC230A01005E
:10F3100002CE97E0FFFFE780009E05611733FFFFF5
:10F32000670023DE1733FFFFE70263DB01117C0078
:10F330003ECAB70707003ECC7C003ECE83C795008F
:10F340002E84AA8493F7F707A384F500A165B90575
:10F35000480897B0FFFFE78000CB97000000E780E8
:10F3600000F1AA85480897D0FFFFE78020B2500837
:10F3700001478146A285268597B0FFFFE78000EE12
:10F3800005611733FFFF6700C3D71733FFFFE7029D
:10F3900063D3AA8401441779FF1F13092999E1490E
:10F3A00097C0FFFFE780A0C56344A400014519A8EA
:10F3B00033053403832709003E958357250063975F
:10F3C000970011051733FFFF670003D30504C9BF7A
:10F3D000032E8500630A0E121773FF1F1303C3B3B6
:10F3E00003230300631503002943639006120323DC
:10F3F0004E01631503001D43639907101733FFFF88
:10F40000E70263CBC689428A3E89BA8AB684328BC8
:10F41000AE8B2A84B5E103554E0019E501431A85E8
:10F420001733FFFF6700A3CCA167A98F116763FBA8
:10F43000E70097000000E78080F5814597F0FFFF27
:10F44000E780C0120844B70700E05841F98F18451B
:10F450005CC1B707001FF98F1CC55C4991C76105E6
:10F4600097E00000E780408BE38A09FA22859790B5
:10F470000000E78060C65DB7328597C00000E78076
:10F4800040430D4349DD1C44116703D54700A16784
:10F49000A98F63FBE70097000000E78040EF8145FC
:10F4A00097F0FFFFE780800C0323840093164B0145
:10F4B000D1828347B300035663008588FD8BA30583
:10F4C000F300FD777D8E558EFD76FD16B204F18E2C
:10F4D00083274301C58E231273012313D300230412
:10F4E000530123052301A3044301BDDF228597B007
:10F4F000FFFFE78080C9AA850844B5D1610597D090
:10F500000000E780207F8DB71D431A858280173366
:10F51000FFFFE70223BB0569AA84AE89328A014452
:10F52000FD5A7D1997C0FFFFE78020A26347A40022
:10F5300001451733FFFF670023BCD844931714001D
:10F54000BA9703D70700631F370323905701630758
:10F550000A00268597900000E780A0809C449DC308
:10F5600083D76700B3F72701639E3701D28801482C
:10F570008147014781460146814526859700000065
:10F58000E78040E5050479BF1733FFFFE70283B347
:10F5900079711C103EC4B7070F003EC61C103EC850
:10F5A00083C79500AA8A328593F7F707A384F500ED
:10F5B0002E89328497D0FFFFE780009D93170501C5
:10F5C000C187635AF006AA89228597D0FFFFE7809A
:10F5D000A09B2A8A4E85032B040097B0FFFFE7808B
:10F5E000609739ED8357440081440544F11793B780
:10F5F0001700A303F10083457100DA872287D286C2
:10F600004E86280097E0FFFFE780E05701478146DC
:10F610003000CA85568597B0FFFFE78020C4A167F8
:10F620009387F70348083ECC230A810026CE97D063
:10F63000FFFFE780406C45611733FFFF6700C3ABF6
:10F64000A2851306710097E0FFFFE7806066AA8439
:10F65000094455D1528597E0FFFFE78060D40D44FF
:10F6600059D90546D285268597000000E78060EAD3
:10F670002A8451B71733FFFFE70263A683550700BB
:10F680000346270041112A842E8532C62EC497E0F6
:10F69000FFFFE780E0D001C93246A24522859700EE
:10F6A0000000E78000E741011733FFFF670063A513
:10F6B0001733FFFFE70223A083C795004111AA8AF1
:10F6C00093F7F707A384F5003285AE89328497D08B
:10F6D000FFFFE780608B93170501C1876357F00A2E
:10F6E000C1452A8A228597C0FFFFE78080702A8D56
:10F6F000228597D0FFFFE78020892A89228597D02D
:10F70000FFFFE7804086930705F893F7F70F13078D
:10F71000E007AA8B637BF706228597D0FFFFE7807F
:10F7200080842A8C228597D0FFFFE780C083AA8C33
:10F730005285032B040097B0FFFFE780A08139E9D1
:10F7400083574400231101008144F11793B7170038
:10F75000A300F1000544034711008356210093875D
:10F7600084005685DA8822885286CE8597F0FFFF7E
:10F77000E78020A7A167E90748003EC42302810073
:10F7800026C697D0FFFFE780005741011733FFFFE0
:10F790006700E39513061100A28597E0FFFFE7805D
:10F7A0002051AA8409E52311010009446DB793058E
:10F7B00021006A8597F0FFFFE780A0F02A8441FDD1
:10F7C000835521009356C900131649018548668860
:10F7D000E2875E87858A5182268597000000E78050
:10F7E00060BF2A848DBF1733FFFFE702C38C83C736
:10F7F000950041112A8B93F7F707A384F500328512
:10F80000AE89328497C0FFFFE78000789317050127
:10F81000C1876352F00A2A8A228597C0FFFFE780DA
:10F82000A076AA8A228597C0FFFFE780E0752A8923
:10F83000228597C0FFFFE7800073930705F893F7D1
:10F84000F70F1307E0072A8C6377F706228597C026
:10F85000FFFFE7804071AA8C228597C0FFFFE780F9
:10F8600080702A8D5285832B040097A0FFFFE780CC
:10F87000606E39E58357440085440144F11793B71E
:10F880001700A301F10003473100930784005A8554
:10F89000DE882688D6865286CE8597F0FFFFE780E1
:10F8A00040948D4748003EC42302910022C697D061
:10F8B000FFFFE780404441011733FFFF67002383C8
:10F8C000A2851306310097E0FFFFE780603E2A849F
:10F8D000894455D99356C9001316490185486A8849
:10F8E000E6876287858A5182D68597000000E78087
:10F8F00060AEAA8449BF1723FFFFE702A37C2A89D1
:10F9000081440144617A916A176BFF1F130BCB602E
:10F9100097B0FFFFE780606463C7A40022851723C8
:10F92000FFFF6700637D8327090093991400CE973A
:10F9300003D507003307450142074183636457033A
:10F9400005C103270B0019C785453E859740000078
:10F95000E78060E9832709000504CE97239007001C
:10F9600085047DB797000000E78060A28327090027
:10F970000504CE972390070065D5814597F0FFFFDA
:10F98000E780C0BEF1BF1723FFFFE702A37383C761
:10F99000950041112A8A93F7F707A384F500328571
:10F9A0002E89328497C0FFFFE780005E9317050120
:10F9B000C187635AF004AA89832A040097A0FFFF35
:10F9C000E780405931E58357440085440144F117ED
:10F9D00093B71700A301F10003483100D687528581
:10F9E0000147CE862686CA8597D0FFFFE780806ACA
:10F9F000A167F50748003EC42302910022C697D0B4
:10FA0000FFFFE780402F41011723FFFF6700C36E10
:10FA1000A2851306310097E0FFFFE78060292A8462
:10FA200089445DD99767FF1F9387074F9C4381CF18
:10FA3000044997B0FFFFE7804052AA85268597408A
:10FA40000000E78040DA1305040197000000E7801A
:10FA5000C0EA228597800000E78000338144ADBF73
:10FA60001723FFFFE702236583C795004111AA8A88
:10FA700093F7F707A384F5003285AE89328423110A
:10FA8000010097C0FFFFE780205093170501C18751
:10FA90006354F0062A8AC145228597C0FFFFE7809C
:10FAA0004035AA8B5285032B040097A0FFFFE78007
:10FAB000604A21E98357440085440144F11793B714
:10FAC0001700A300F1000348110003572100DA8753
:10FAD0005685D2862686CE8597D0FFFFE780805B4D
:10FAE000A1679387270248003EC42302910022C6E3
:10FAF00097D0FFFFE780202041011723FFFF670019
:10FB0000035FA2851306110097E0FFFFE780401A0C
:10FB10002A8489444DD99767FF1F9387E73F98430D
:10FB20003E8901CF044997B0FFFFE7800043AA85D3
:10FB3000268597400000E78000CB1305040197005D
:10FB40000000E78080DB97B0FFFFE780004195442D
:10FB50003DD9930521005E8597F0FFFFE78060B6F1
:10FB6000AA8435F11C480357210022852390E70021
:10FB700097800000E780402183270900A9D703551B
:10FB8000210097400000E780A0BD35BF1723FFFF8D
:10FB9000E702635283C795004111AA8A93F7F707DA
:10FBA000A384F5003285AE89328497C0FFFFE780D9
:10FBB000A03D93170501C1876351F0062A8A22856B
:10FBC00097C0FFFFE780403C2A895285032B040041
:10FBD00097A0FFFFE780003831E583574400854454
:10FBE0000144F11793B71700A301F1000348310056
:10FBF000DA8756854A87D2862686CE8597D0FFFF3C
:10FC0000E7804049A167F90748003EC423029100FC
:10FC100022C697D0FFFFE780000E41011723FFFFA8
:10FC20006700E34CA2851306310097E0FFFFE780F1
:10FC300020082A8489445DD99167CA97C207116751
:10FC4000C1831307F7EF8544E362F7FA9767FF1F55
:10FC50009387872C9843BE8B01CF044997B0FFFF51
:10FC6000E780A02FAA85268597400000E780A0B7EF
:10FC70001305040197000000E78020C897B0FFFF3C
:10FC8000E780A02D95443DD11C48228581442390D6
:10FC9000270197800000E780200F83A70B00B9D7CA
:10FCA0004A8597400000E780A0AB89B71723FFFF84
:10FCB000E702E3422A844105B28497000000E7800E
:10FCC000C0C311C5228597800000E780E00B814604
:10FCD0000146A685228597800000E780C04E1C4C17
:10FCE00089C7DC4799C3228582971723FFFF6700E6
:10FCF00043419767FF1F938727039C43014599C39F
:10FD00001385070182809767FF1F9387E701884368
:10FD100082801723FFFFE702833C9317C600DD8D27
:10FD2000C2054111C1812A8432C697C0FFFFE78016
:10FD3000E0173246228511829375F60F97C0FFFFB8
:10FD4000E780C01441011723FFFF6700833B17239F
:10FD5000FFFFE702233779713C083ED2B7070C005A
:10FD60003ED43C083ED683C79500AE842A8993F7DB
:10FD7000F707A384F500A16593853504481097A083
:10FD8000FFFFE7804028C165FD150144176AFF1F8A
:10FD9000130A0A1A930A400EAE892E8B2EC697B00C
:10FDA000FFFFE780801E4205931704014181C18354
:10FDB000B24563E9A702C167FD176387F5004810E4
:10FDC00097C0FFFFE780800E501001478146A6854F
:10FDD0004A8597A0FFFFE780604845611723FFFF32
:10FDE000670083313307540383270A0BBA9703D67E
:10FDF000C701630A3601638A350148109700000085
:10FE0000E78060F1DA85050451BFB285EDBF1723A5
:10FE1000FFFFE702432A79717C083EC8B70711004B
:10FE20003ECA7C083ECC83C79500AA89328593F7E9
:10FE3000F707A384F5002E8997C0FFFFE780C01461
:10FE400085676378F504A165AA848905080897A0E9
:10FE5000FFFFE780401B268597400000E78060EDAC
:10FE6000133415000A04A285080897C0FFFFE78035
:10FE7000E001A685080897C0FFFFE780200325CC96
:10FE8000014781461008CA854E8597A0FFFFE7808D
:10FE9000E03C45611723FFFF67006325B307540368
:10FEA0000327CA0ABA9703D70700631C970003D633
:10FEB000270063806505080897000000E780A0E53B
:10FEC000DE8505042EC697B0FFFFE780000D4205D2
:10FED000931704014181C183B245E3E1A7FCC167E7
:10FEE000FD17E38FF5F8080897C0FFFFE78000FCD7
:10FEF00041BFB285F9B7C165FD150144176AFF1FFF
:10FF0000130A0A03930A80022E8BAE8B65BF172358
:10FF1000FFFFE702C31C1841834717008346070011
:10FF2000A207D58FD207D1832390F50083472700FE
:10FF3000034717008D45A207D98F91832310F60040
:10FF400097C0FFFFE780A0E91723FFFF6700631B4F
:10FF50001723FFFFE7020317C16401441769FF1F5E
:10FF6000130909FD93098002FD1497B0FFFFE78094
:10FF7000C0026347A40001451723FFFF6700C317B2
:10FF8000330534038327C90A3E9583570500E3856B
:10FF900097FE0504D9BF1723FFFFE702A3122A8AA1
:10FFA000AE89B284B68A97400000E78080D819E510
:10FFB00091473E851723FFFF670003142A894E856A
:10FFC00097C00000E780E08E2A84638E0A048D4784
:10FFD0006DD103570500C547E31D47FD0347F901F0
:10FFE0008546AD47E317D7FC8347450081CF41469F
:10FFF000A6855D0597F00000E780C09E814755D932
:020000040001F9
:10000000AD4745BF130965012302E500CA85268572
:1000100097100000E780606231C1A547E38B0AF8C2
:100020002302040079B705C183570500E39247F91D
:100030004146A685190597F00000E780A09A814700
:100040002DD99947BDB74E8597000000E78080F015
:100050002A84954739DD130955004DBF4146A685D1
:1000600023104401231134011305190097F00000F7
:10007000E780A099228597800000E780A0EA814769
:100080000DBF1723FFFFE702830579717C003ECC8B
:10009000B7070A003ECE7C003ED083C79500B284ED
:1000A0002E8493F7F707A384F5001306A1002A898D
:1000B0002C00268597000000E780A0E5A1652808B0
:1000C0008D0597A0FFFFE78000F490408355A100C5
:1000D00003558100854697000000E78000ECAA8464
:1000E000AA85280897C0FFFFE78040DA0356A100E1
:1000F00083558100280897000000E780C0C13008C0
:1001000001478146A2854A8597A0FFFFE780001539
:10011000854748103ED42302910202D697D0FFFFB4
:10012000E78060BD45611723FFFF670083FD17234C
:10013000FFFFE702C3FA79717C003ECCB7070A00E3
:100140003ECE7C003ED083C79500B2842E8493F7C8
:10015000F707A384F5001306A1002A892C00268541
:1001600097000000E780E0DAA16528088D0597A0D8
:10017000FFFFE78040E990408355A10003558100CF
:10018000814697000000E78040E1AA84AA852808FC
:1001900097C0FFFFE78080CF0356A1008355810001
:1001A000280897000000E78000B730080147814623
:1001B000A2854A8597A0FFFFE780400A48102302E6
:1001C000910202D402D697D0FFFFE780C0B245610A
:1001D0001723FFFF6700E3F21723FFFFE70223F077
:1001E00097000000E78060DB1723FFFF670063F1E3
:1001F0009767FF1F938787B3884382801723FFFF8A
:10020000E702E3ED835725004111AE842A842307DA
:10021000B10017F5FFFF130525466C002316F1000A
:1002200097A0FFFFE780804591C42285978000005A
:10023000E780E0D6FD572310F40013062002814525
:10024000130554009720FFFFE78060EC410117235E
:10025000FFFF670003EB1723FFFFE702A3E67971B7
:100260007C003ECCB7070A003ECE7C003ED083C760
:100270009500AA89AE8493F7F7073285A384F50029
:100280001306A1002C0097000000E78080C80355EA
:100290008100114497400000E780A0A915C50355CF
:1002A000A100014497B00000E780A06011CD035782
:1002B00005008357810045446318F7008545970082
:1002C0000000E780E0F30144216993053900280824
:1002D00097A0FFFFE78020D3A285280897C0FFFFE3
:1002E000E780C0BA0356A100835581002808970013
:1002F0000000E78040A2300801478146A6854E8570
:1003000097A0FFFFE78080F548104AD423028102BE
:1003100002D697D0FFFFE780009E45611723FFFFBD
:10032000670083DD1723FFFFE702C3D99767FF1F2D
:100330009387879F2A8488432E8915C503574503D1
:100340008357C4016311F70223260502231805020F
:10035000410597D00000E780209C63060900978044
:100360000000E78060DB81449769FF1F938949BCE7
:10037000130A800297B0FFFFE78020C263C4A40481
:100380009767FF1F938707A39C4399C70355C40131
:1003900097200000E780C0BD630709002285978091
:1003A0000000E780C0A01306400E814522859720FB
:1003B000FFFFE780C0D5FD57231EF4001723FFFF82
:1003C000670083D33385440383A7C90A3E95035747
:1003D00005008357C4016317F700CA859700000022
:1003E000E78000E2850479B71723FFFFE70283CD9A
:1003F00083C795004111AA8993F7F707A384F500F5
:100400003285AE8497C0FFFFE78000B885676378C8
:10041000F5042A8997400000E780A091014401CDAE
:1004200083D7040031446388270185459700000085
:10043000E78080EF01444E85A2864A86A68597D044
:10044000FFFFE780A09CA1679387170448003EC484
:100450002302810002C697D0FFFFE780C0894101D7
:100460001723FFFF670043C91723FFFFE70283C578
:100470009767FF1F9387478B804329C4014597C027
:100480000000E780002181470148C1641CDC232E65
:100490000403232004041769FF1F130969A90144F9
:1004A0009309400EFD1497B0FFFFE78000AE634F45
:1004B000A400814517F5FFFF1305857F97A0FFFF77
:1004C000E780C01B1723FFFF670003C33305340316
:1004D0008327090B3E958357C501638797008545A0
:1004E00097000000E78040E4050475BF93570501BD
:1004F00013D78700A380F50093170501C183A1835B
:100500002380E5002381F500A381A50082801723C5
:10051000FFFFE702C3BC2300050083C71500A3004B
:10052000F50083C725002301F50083C73500A3012B
:10053000F50083C745002302F50083C75500A302D9
:10054000F50083C7650093059500A3030500230309
:10055000F50023040500328597000000E78040F98C
:100560001723FFFF6700E3B91723FFFFE70283B5F7
:100570004111E9540DCD85CD93F9C5FF2E842A890B
:10058000AA84338AA900B7EA040063189A020D8886
:10059000854411CCB7E704009C5F82972AC6228667
:1005A0006C003305390197E00000E780004626859E
:1005B00041011723FFFF670023B483A78A03910437
:1005C000829793170501C183A183A38EF4FE9357ED
:1005D0000501238FF4FEA183238EA4FEA38FF4FED6
:1005E0006DB763E6D5021723FFFFE70243AFB2877B
:1005F00041113686BE8536C697E00000E780E040B0
:10060000B246410136851723FFFF670083AF81465D
:1006100036858280838705001387F5003D05FD87B9
:1006200093F77708834607007D158606B58FA300EC
:10063000F5006307B7007D17834717009D83DDB77B
:1006400082801723FFFFE70283A9B7E7040083A78F
:10065000070932872A863A858297133515001723B2
:10066000FFFF670003AA15C181478DC11723FFFF54
:10067000E702E3A6414697E00000E780003985479E
:100680003E851723FFFF6700C3A781473E85828011
:100690001DCD1723FFFFE70283A4414681452A842D
:1006A0009720FFFFE780A0A641468145130504037C
:1006B0009720FFFFE780A0A50147C167232204041C
:1006C00038C87CC805451723FFFF670083A3014591
:1006D000828081473DCDB5CD1723FFFFE70223A0E0
:1006E000B2842E891306800581452A849720FFFF56
:1006F000E780E0A1CA8524C4268597000000E78032
:10070000C0F64146814522859720FFFFE78020A063
:100710003044A285228597000000E780C0F2930450
:100720000401A285268597000000E780E0EEA685FB
:100730001305040297000000E78000EE2285970071
:100740000000E78020F585473E851723FFFF6700FF
:10075000439B3E8582801723FFFFE702A39641114A
:10076000E9540DCD85CD93F9C5FF2E842A89AA843D
:10077000338AA900B7EA0400639844030D888144D2
:1007800011CCB7E704009C5F82972AC622866C00D2
:100790003305390197E00000E780202726854101D5
:1007A0001723FFFF6700439583A78A03910482976D
:1007B00093170501C183A183A38EF4FE935705010E
:1007C000238FF4FEA183238EA4FEA38FF4FE6DB7C6
:1007D00065CD1723FFFFE702E38EB28411E60545DE
:1007E0001723FFFF670043912A842E890145EDD925
:1007F0003C487848B3E6E700E5D69386F7FFB3B701
:10080000F6007D17032A4404BA9734C87CC86305F0
:100810000A06C14913050A03B38949412295637D3C
:100820003601B2862E86A68597000000E780A0DB01
:100830007C40BE9464C065B7CE862E86CE85970078
:100840000000E78040DAC114D2944E9923220404B8
:10085000A2879306040103C7070003C607038507A1
:10086000318FA38FE7FEE398F6FE3044A285228500
:1008700097000000E78020DD2699C14933069940A2
:1008800063EC9900A9DCA686A685130504039700EE
:100890000000E78040D579BF8147B306F4003307F5
:1008A000F6000347070083C5060085072D8F2380C8
:1008B000E600E39437FF3044A285228597000000CC
:1008C000E78060D8C1145DBF014582800DC1172348
:1008D000FFFFE702C3801306800581459720FFFFD5
:1008E000E780E08205451723FFFF6700838101450C
:1008F0008280814749C5C1C51713FFFFE702237EE8
:10090000FC4141462E84AA846399C70413860501DD
:10091000A2878146C14503C7070003C507038507B2
:10092000298F3305D600034505008506298FA38F3F
:10093000E7FEE392B6FE3044A285268597000000CC
:10094000E78060D0228597000000E78060F8854747
:100950003E851713FFFF6700C37A138507031D8EBB
:10096000814522959710FFFFE780607A7C4013074E
:1009700000F813060402A2972388E70251BF3E85C0
:1009800082801713FFFFE70283756D712E84B28496
:10099000AA8590102800368997000000E780A0D330
:1009A00009EDD55725A050400C40280097000000C5
:1009B000E78040E27DD5FD142104F5F42C004A8542
:1009C00097000000E78020F3814761DD3E8551619B
:1009D0001713FFFF6700E3721713FFFFE70223708F
:1009E00041112EC432C62C00054697000000E78056
:1009F00080F941011713FFFF6700A3701713FFFF72
:100A0000E702E36D01112A842EC602C802CA02CC95
:100A100002CE97E00000E780C023B2462A86A28576
:100A2000080897000000E78060FB1375F50F05616B
:100A30001713FFFF6700E36C1713FFFFE702236A3A
:100A40007971B2872A8421462308B1001305110168
:100A5000BE853AC436C697E00000E78000FBB24688
:100A600093059101368597000000E78060A82285F4
:100A7000141035460C0897000000E78020F62A8401
:100A8000224701E921460C103A8597E00000E780F3
:100A9000C0F7228545611713FFFF670083661713B0
:100AA000FFFFE702C3637171AE84AA850A853284B1
:100AB00097000000E78060BB11C90A86A6852285E1
:100AC00097000000E78020B8814711E1C5473E85C7
:100AD0004D611713FFFF6700C3621713FFFFE702A3
:100AE000035D1D712A8AB289BE8435468547130588
:100AF00011012E8CB68A3A8BC28C468D2308F100E8
:100B000097E00000E78060F010100C085285231F6A
:100B1000010097000000E780C0F82A843DEDA1475E
:100B20006313FD089307900591E0E5473546E2859C
:100B30001305110113990A012308F1001359090142
:100B400097E00000E78060EC1357890093978A00D4
:100B5000D98F90080C085285231FF10097000000E0
:100B6000E78020F42A8415E9A1E49387FA009183B1
:100B70001379F9003EC6631309004149668B81442D
:100B8000C14B854DB247639F970C6A868C003385B5
:100B90005C0197E00000E78040E72285256117139C
:100BA000FFFF6700835493079004C9F0A547BDBFBA
:100BB000834701050947C14B2308F100834711050D
:100BC000A58FA308F10093872400814463E1FB040F
:100BD000014714083386E6008C08B386E400BA9512
:100BE000DA9683C6060083C505000507AD8E23008F
:100BF000D600E390E7FE4147639CE70490080C08A9
:100C0000528597000000E780C0E925D181A0B30696
:100C10009B00BA871008B305F60090083E9603C5FE
:100C200006000346060085078506298E2380C50039
:100C3000E39277FF998F90080C085285BE94970035
:100C40000000E78000E68947014749D12A84B1B70F
:100C500090083E96034606001408BE962380C60000
:100C6000850759BFB24785046387971481471808E1
:100C7000B306F70098083E973386F900034707004C
:100C8000034606008507318F2380E600E39177FF56
:100C900090080C08528597000000E78080E05DF521
:100CA0003546E285130511012308B10197E00000E4
:100CB000E780A0D513970401418393978400218393
:100CC000D98F10180C085285231FF10097000000DF
:100CD000E78020DD25FD814710183387F9003E9617
:100CE0000347070003460600B306FB008507318F64
:100CF0002380E600E39277FF65A81808B306F700A3
:100D000098083E973386F90003470700034606001C
:100D10008507318F2380E600E3E127FFCA87639EC2
:100D2000770990080C08528597000000E78060D78B
:100D300011FD81479800B306F700900818103E9700
:100D40003E9603470700034606008507318F238040
:100D5000E600E39177FF3546E2851305110123088C
:100D6000B10197E00000E78040CA13970401418376
:100D7000939784002183D98F10180C085285231F64
:100D8000F10097000000E780C0D1E31105EC814736
:100D900010183387F9003E96034707000346060004
:100DA000B306FB008507318F2380E600E3E227FFCF
:100DB000C109410BC1BB814785B79408BE9683C664
:100DC000060018083E972300D700850789BF638077
:100DD00006321713FFFFE702832D59712A84BE895B
:100DE000B28B85473546130511022E8B468C4289FE
:100DF000BA8A368A2300F10297E00000E780E0C05B
:100E000010180C1022852317010297000000E780BC
:100E100040C963180512A147631FFC06930790059C
:100E200063930900E5473546DA85130511029314EB
:100E30000A012300F102C18097E00000E780E0BCD6
:100E400093178A0013D78400D98F90080C1022853D
:100E50002317F10297000000E780A0C47DE16392B0
:100E600009049307FA00BD88918391E0C144C20749
:100E7000C183DE8C814A3EC6414DB24763E2FA0E21
:100E80006286B3854B01881097E00000E78080B54B
:100E90004DC93D557DA093079004E39609F8A547F9
:100EA00059B7834701050947C14C2300F102834725
:100EB0001105B3C7F900A300F10293872900814906
:100EC00063E1FC04814618103306D7008C08338791
:100ED000D900B69556970347070083C505008506D8
:100EE0002D8F2300E600E390D7FE41476390E7068D
:100EF00090080C10228597000000E78080BA35D159
:100F000089A0B3863A01BA871010B305F60090089D
:100F10003E9603C506000346060085078506298E12
:100F20002380C500E39297FF3387EC4090080C10B4
:100F30002285BA9997000000E780A0B6894701474B
:100F400041D165611713FFFF6700231A90083E9691
:100F5000034606001410BE962380C600850779B7A5
:100F6000B247850A93990A01939D8A0093D9090192
:100F70006391570F85473546DA8513051102230023
:100F8000F10293D9890097E00000E78000A8B3ED53
:100F90003D0190000C1022852317B103970000003B
:100FA000E78020B059FD8147A68963EA9706268627
:100FB0000C084A8597E00000E78020A581471810BB
:100FC000B306F700100898083E973E9603470700BF
:100FD000034606008507318F2380E600E3E197FE94
:100FE000639FA90590080C10228597000000E780F8
:100FF00040AB21F981479810B306F7009008181804
:101000003E973E9603470700034606008507318F4B
:101010002380E600E391A7FF4109C10CB9BD180880
:101020009000B306F7003E963387FC0003470700A5
:10103000034606008507318F2380E600B5B7980880
:101040004E97034707001C10CE972380E7008509C1
:1010500041BF85473546DA85130511022300F102A9
:1010600093D9890097E00000E780209AB3ED3D0115
:1010700090000C1022852317B10397000000E78031
:1010800040A2E31005EC814718089000B306F70072
:101090003E963387FC00034707000346060085079A
:1010A000318F2380E600E391A7FF41460C084A8573
:1010B00097E00000E780609581471810B306F700BD
:1010C000100898083E973E9603470700034606001F
:1010D0008507318F2380E600E391A7FF90080C106D
:1010E000228597000000E780C09B1DD599BD7D55E6
:1010F00082801713FFFFE70283FE01112A842E85E9
:1011000093055100328902C002C202C402C6930490
:10111000740097F0FFFFE780A03D1D46A6851305EC
:10112000910097E00000E780408E10088A854A858C
:1011300097000000E780E09619ED93071400180867
:1011400083C607000346070085070507B18EA38FF6
:10115000D7FEE397F4FE05611713FFFF670063FAFC
:101160001713FFFFE70203F62E848C414111AA8971
:10117000838715003289914463D30700A1449757B0
:10118000FF1F938767119C43A1C7C1CA8D472310D6
:10119000F10083C725004A852301F10083C735008C
:1011A000A301F10083C745002302F10083C7550066
:1011B000A302F10083C7650093059100A30301001A
:1011C0002303F1002304010097F0FFFFE780403282
:1011D0000C404A860A8597F0FFFFE780803303289A
:1011E000040083564400A6881D0881470147E51680
:1011F00042868A854E8597000000E780408E2A89C6
:1012000019E5A685228597B0FFFFE780E0C14A85F2
:1012100041011713FFFF670023EE4A860A8597F006
:10122000FFFFE780002F6DB71713FFFFE70283E989
:101230002E848C414111AA898387150032899144FB
:1012400063D30700A1449757FF1F9387E7049C438C
:10125000A1C7C1C68D472310F10083C725004A8569
:101260002301F10083C73500A301F10083C74500C6
:101270002302F10083C75500A302F10083C7650074
:1012800093059100A30301002303F100230401004F
:1012900097F0FFFFE780C0250C404A860A8597F04B
:1012A000FFFFE780002783564400032804008A8557
:1012B000858EC2061D08C1822312D400A6888147EC
:1012C0000147E51642864E8597000000E78060B032
:1012D00041011713FFFF670023E24A860A8597F052
:1012E000FFFFE78000234DBF1713FFFFE70223DF57
:1012F000B335B000011185052A891315F601336550
:1013000015012308B1009305110136843AC632C095
:101310003EC442C297F0FFFFE780801DA2471248FB
:10132000425593D68700230BF10093059101935703
:101330008800A30AD100A30BF100230C010197F050
:10134000FFFFE780E01A3247024603280400B33764
:10135000E000835644009207914411C2A1444A859B
:10136000A68842860C0897F0FFFFE78040772A891D
:1013700019E5A685228597B0FFFFE780E0AA4A8598
:1013800005611713FFFF6700C3D71713FFFFE702BD
:1013900063D301113EC68647B335B0008505AA89DF
:1013A0001315F6015D8D2308B100930511013684F4
:1013B0003A89B28442C446C297F0FFFFE7804013E7
:1013C00022489248164593578800A30AF1009305D6
:1013D000910193D78800230B0101A30BF100230C8B
:1013E000110197F0FFFFE780A010324710408356AD
:1013F0004400B337E000920703280900914891C0E8
:10140000A1480C084E8597000000E780809CAA84C4
:1014100001E9835544004A8597B0FFFFE780C0A0EB
:10142000268505611713FFFF670003CDAA95930773
:10143000F00F170701001307E7546317B50013C532
:10144000F7FF1375F50F828005058346F5FFB58F0D
:10145000BA9783C70700D5B70357450014419307D0
:10146000F00F170601001306E65136974207418335
:10147000139506014181631BE500AD8FB29703C54B
:101480000700130515F3133515008280850603C583
:10149000F6FFA98FB29783C70700D9BF1713FFFFC5
:1014A000E702E3C3B28736842E86BA86AA853E85D4
:1014B000BA8497F0FFFFE7806052634F05002285F2
:1014C00097D00000E780E0782A86A686A285268548
:1014D00097F0FFFFE78080501713FFFF670063C29C
:1014E0001713FFFFE70203BE5D712A8BAE8A170553
:1014F00001001305A5462C00B284368ABA893E89BC
:1015000097F0FFFFE780C04F2A845DE13410414629
:10151000DA85280097F0FFFFE780404C2A8449E9EC
:101520008547A303F100A6C2930771002408BEC437
:10153000A68685470D462C18281002DC02DED6C090
:10154000BEC697F0FFFFE78000442A8435E1834759
:101550007102A6860D4693F7F7072300FA00C147EC
:101560003EDE2C188947281026DCA303F10097F0F3
:10157000FFFFE78040412A8405ED4146A6854E8560
:1015800097D00000E78060488D47A6860D462C184E
:101590002810A303F10097F0FFFFE780C03E2A84E4
:1015A00001E94146A6854A8597D00000E780E045DD
:1015B000228561611713FFFF670003B41713FFFF54
:1015C000E702E3B197F700009387C7A0984383C76A
:1015D000470079712A89AE84170501001305853803
:1015E0000C083AC42306F10097F0FFFFE780404162
:1015F0002A8405ED14104146CA85080897F0FFFFBC
:10160000E780C03D2A8415E1140815462C00081017
:1016100097F0FFFFE780803C2A8401E921462C08EF
:10162000268597D00000E780403E2285456117134C
:10163000FFFF670003AD1713FFFFE70243AA97F709
:101640000000938727999C477971AA842E841705F7
:1016500001001305A5310C083EC697F0FFFFE78097
:10166000203A0DE914104146A685080897F0FFFFBF
:10167000E780C03605E1140811466C00081097F0A9
:10168000FFFFE780A03519E58347F10193F7F703E2
:101690002300F40045611713FFFF670083A61713AB
:1016A000FFFFE702C3A33688A14881470147E5460B
:1016B00097F0FFFFE780A0421713FFFF670063A4C6
:1016C0001713FFFFE702A3A13688A148814701470E
:1016D000E54697F0FFFFE780C06F1713FFFF670035
:1016E00043A21713FFFFE702839F01112A842E856F
:1016F0000C0832C697F0FFFFE780803009ED3247D3
:1017000097060100938606251008C145228597009B
:101710000000E780E0D805611713FFFF6700639EB4
:101720001713FFFFE702A39B4111C1472EC032C42C
:101730008A8509463EC23EC697F0FFFFE780A02497
:1017400041011713FFFF6700C39B1713FFFFE70259
:1017500003994111AE8613061009AA850A8502C0B5
:1017600002C202C402C697F0FFFFE78020274101B2
:101770001713FFFF6700E3981713FFFFE702239695
:101780003287970601009386E61E2E869305000297
:1017900097000000E780C0D01713FFFF6700639633
:1017A0001713FFFFE702A3937971C1472ACC2ED00C
:1017B00032D42C080D4628003ECE3ED23ED602C47E
:1017C00002C602C802CA97F0FFFFE780C01B45614E
:1017D0001713FFFF6700E3921713FFFFE702239041
:1017E0000111AA842E8417050100130525198A8585
:1017F00097F0FFFFE780C02015E514084146A68555
:101800000A8597F0FFFFE780601D09ED8347E1013E
:101810000347F101A207D98FCA07C9836177D98F1E
:101820002310F40005611713FFFF6700838D15CDAA
:101830001713FFFFE702A38A9747FF1F938787537A
:1018400090439745FF1F938525531745FF1F1305A9
:10185000654E97D00000E78000C51745FF1F1305B0
:10186000654D1713FFFF6700C3891745FF1F130559
:10187000654C82808DCD1713FFFFE70243869747A3
:10188000FF1F9387274F944301112E840A869745A3
:10189000FF1F9385654E97D00000E78040C60A85FC
:1018A0000294014505611713FFFF670083857D558D
:1018B00082801713FFFFE702838297D00000E78042
:1018C00080D19747FF1F23A7A74A17F5FFFF1305EE
:1018D000E5C997B00000E780C0741713FFFF6700E9
:1018E00043821747FF1F1307274B93171500084321
:1018F0003E95FD572310F50082801703FFFFE70296
:10190000037E2A84084009E51703FFFF6700637F11
:101910001C4158401CC06313E5005CC08347550060
:1019200023200500F99BA302F50097A0FFFFE780A5
:10193000207CC9BF1703FFFFE702C3789747FF1F4B
:101940009387874798432A8411CB8347350093F7C1
:10195000070289C70355050089450297130544010D
:1019600097B00000E780403B835504000355E40036
:1019700097300000E780A00C485819C597A0FFFFDA
:10198000E7800077232A04021305840397000000F0
:10199000E780E0F68144B1499790FFFFE780206A35
:1019A00063CBA402834734002320040493F727FC6D
:1019B000A301F40000489790FFFFE78040691316E9
:1019C0001500814522859700FFFFE78040741703CB
:1019D000FFFF67006372B3873403032904038504A0
:1019E0003E994A8597000000E78060F123040900D2
:1019F00065B78347350093F7070299E30145828075
:101A00008357E500E39CB7FEC167FD176316F60038
:101A100005458280054599A81703FFFFE702236C5F
:101A200093170601C187B2842A8401496359F002E1
:101A3000835705009DCB01456367F600034584008D
:101A40003E953325A6001375F50F0DA01C481317FE
:101A50001900BA9783D70700E38E97FA0509979084
:101A6000FFFFE780C05EE343A9FE01451703FFFFC8
:101A7000670023691703FFFFE702C364AE89AA84E6
:101A80009790FFFFE78060522A8497D0FFFFE7809E
:101A9000A02EAA86014713068401970500009385AE
:101AA00085E41745FF1F1305652F9790FFFFE7801B
:101AB000E0182A8925C98C441304C50022859E0597
:101AC00093F5050897A0FFFFE780403CCC40838753
:101AD0007400E18163DD070493E50508228597A082
:101AE000FFFFE780A03A0D4693854400228597A02A
:101AF000FFFFE780C03683D50400228597A0FFFF53
:101B0000E780E03D83D52400228597A0FFFFE78092
:101B1000003D03D6490083A50900228597A0FFFF59
:101B2000E780E0334A851703FFFF6700E35C93F526
:101B3000F5076DB71703FFFFE702635A01112A8407
:101B4000328532C697A0FFFFE780E0279780FFFF2E
:101B5000E780C030835704001747FF1F1307473D36
:101B60003246231BF100930700F8A30DF1001C4738
:101B70001843231AA1008983858BB307F740B285E8
:101B800048083ECE231C0100230D010097000000F1
:101B9000E78080EE05611703FFFF67008356170398
:101BA000FFFFE7022352004101453DC49304C400F6
:101BB00026853289AE8997A0FFFFE780C02495452E
:101BC0002A8A2685035B040197A0FFFFE780202176
:101BD000268597A0FFFFE780603E8D45AA8A26856F
:101BE00097A0FFFFE780A01F268597A0FFFFE78053
:101BF000E03C5C48420A135A0A01D2975CC423189D
:101C00006401814763983A0146054D8133062541B9
:101C10009337160013F5F70F1703FFFF6700C34D47
:101C20001703FFFFE702234989692A8BAE8B328AAB
:101C3000B68A81440144314CFD199790FFFFE7803B
:101C4000004063CDA4009790FFFFE7804042018DE4
:101C500033B5AA001703FFFF670063493389840384
:101C600083270B003E9963170A0083478900850488
:101C70003E94E1B703560A00DE854A8533F6C90073
:101C800097000000E780E0F16DD10545E1B717034B
:101C9000FFFFE702C34401112A847C000355E500DD
:101CA0003ECAB70707003ECC7C003ECE972000001E
:101CB000E78020082A898545480897A0FFFFE7802C
:101CC00020399945480897A0FFFFE780E015AA84CE
:101CD0004A8597200000E780A0082380A40097474A
:101CE000FF1F9387E7249C434166130606F09396F3
:101CF000870113D78701558F93D68700F18E558FB3
:101D0000A207B706FF00F58FD98F11462C00138567
:101D100014003EC497D00000E78020CF5008A38273
:101D200004008945228597000000E780E0E019C99A
:101D3000AA851305840397A0FFFFE780E0313C40AC
:101D400085073CC005611703FFFF6700833B17034E
:101D5000FFFFE702C3389790FFFFE78040312A84F6
:101D600005049790FFFFE780802F3305A402F14719
:101D700091453305F50297200000E78020BA11E570
:101D800065551703FFFF6700C3379747FF1F23AD54
:101D9000A7009790FFFFE780802D2A840504979085
:101DA000FFFFE780C02B3305A40289450605972075
:101DB0000000E780A0B669D59747FF1F23AEA7FCB8
:101DC0009790FFFFE780A02A2A8405049790FFFFE1
:101DD000E780E0283304A4029747FF1F239087FC85
:101DE0009790FFFFE780A0282A849790FFFFE78065
:101DF0000027930714003385A7029747FF1F2390FE
:101E0000A7FA97F700009387277B1747FF1F232B1D
:101E1000F7F80145BDB71703FFFFE702A32AAA841D
:101E20002E8901449749FF1F93898910130A800660
:101E30009790FFFFE780A0226347A40001451703A6
:101E4000FFFF6700632B3305440383A709024A861B
:101E5000A6853E9597000000E780E0B919E10504EA
:101E6000C1BF0545E9BF1703FFFFE702C324AA8AE4
:101E70002E8BB28B368C3A8A814401448149974C2F
:101E8000FF1F938CEC0A130D80069790FFFFE780ED
:101E9000001D63C9A40011E085494E851703FFFFAB
:101EA0006700E3243389A40383A70C025E86D685EA
:101EB0003E994A8597000000E780E0B31DC19790E6
:101EC000FFFFE780C01A0544636D4501D286628634
:101ED000DA851305090397000000E780A0D411C13B
:101EE000854985045DB71703FFFFE702A31DC164A1
:101EF00041112A8901449749FF1F93896903130AF5
:101F00008006FD1436C632C42EC29790FFFFE780CC
:101F1000001592452246B2466348A400014541019E
:101F20001703FFFF6700431D3305440383A709021E
:101F30003E9509C683473500C18B9DC791C683472F
:101F4000350093F707028DC3630699008357E500B8
:101F5000639C27010357050001CB63E7E500834736
:101F60008500BA97E3CDF5FA050469BF1703FFFFB3
:101F7000E7024315C1642A8901449749FF1F9389E9
:101F800029FB130A8006FD149790FFFFE780200DC0
:101F90006346A4001703FFFF6700031633054403DD
:101FA00083A709023E958357E500638A970063047F
:101FB00099006396270197000000E780E0970504E9
:101FC000E1B71703FFFFE702830E89692A8AAE8A09
:101FD000328BB68B8144174CFF1F130C6CF5930C9E
:101FE0008006314DFD199790FFFFE780400763C6DB
:101FF000A4001703FFFF6700430F3389940383276F
:102000000C028355CA015A863E994A859700000002
:10201000E780609E31C1814D15A03384AD038327D5
:10202000090303D60B00D68533F6C9003E942285FA
:1020300097000000E780E0B609E9850D9790FFFF63
:10204000E780E0FFE3CBADFC01A82285970000000C
:10205000E780E08A23040400850471B71703FFFFBB
:10206000E70263054169AA8A014A174BFF1F130B58
:102070002BEC7D19C14B054C9790FFFFE78020FEAC
:102080006346AA001703FFFF6700630693098006F3
:10209000B3073A0383290B02BE9983D7E900638E05
:1020A000270163842A01639A570103A4890301E885
:1020B0004E8597000000E780C0BD050A75BF8357B5
:1020C0000401639977099304C400268597A0FFFF54
:1020D000E78060D385452A8D2685835C040197A01F
:1020E000FFFFE780C0CF268597A0FFFFE780A0E72E
:1020F00062056185635905048D45268597A0FFFF1C
:10210000E780E0CD8945268597A0FFFFE78020CDB9
:102110008945268597A0FFFFE78060CC8545268509
:1021200097A0FFFFE780E0CC83470500094793F7BE
:10213000F707639AE7009945268597A0FFFFE78098
:1021400040CBA30285014848337D2D01231894011B
:102150006A9548C40040A1BF1703FFFFE70223F8B8
:1021600037E404008327041D82979747FF1F83C726
:1021700027C91715FF1F1305653BA300F50083272B
:10218000441C82978327841C81461306F00F8145E7
:10219000014582971703FFFF6700A3F61747FF1F4C
:1021A000130707B618439745FF1F83C565C59747B3
:1021B000FF1F938767C3834687030346970363978D
:1021C000D5009747FF1F238DC7C2828083C5870133
:1021D0000347A7036317B6009747FF1F2382E7C291
:1021E000828003C687016317C7009747FF1F2389B3
:1021F000D7C0828083C68701130750026319D700B6
:10220000930760021747FF1F230CF7BE828083C627
:102210008701130660026315D60093077002DDB7CD
:1022200083C7870155BF9747FF1F9387E7BBD44BF1
:102230000947638DE6081703FFFFE70243EA1749E2
:10224000FF1F1309A9B73E8483470900918B9DCFD7
:10225000B7E4040083A7041D829783A7441C174595
:10226000FF1F130525B6829783A7841C8146174656
:10227000FF1F034626B781450145829721C5834745
:102280000900ED9B1747FF1F230AF7B2834704009D
:1022900093F7F70F85CB91471747FF1F2320F7B61A
:1022A00097000000E78080EB97000000E78040EF98
:1022B000B7E70400BC4F414691451745FF1F034552
:1022C00025B382971703FFFF6700A3E382801703FC
:1022D000FFFFE702C3E08D4741116306F504C547E0
:1022E0006308F50285476310F5029747FF1F238BAC
:1022F000A7B0B7E70400BC4B930500101745FF1FBC
:10230000034505AF829741011703FFFF670063DFB5
:1023100085471747FF1F2307F7AEB7E70400BC4BFD
:1023200093050020E1BF9747FF1F9387E7ABD44B8E
:102330001147638DE600B7E7040083A7071D829766
:10234000B7E70400BC4B930500044DBF0549174790
:10235000FF1F232527AB83C7070032C62E8493F7C0
:10236000F70FD5D3B7E4040083A7041D7D141374BD
:10237000F40F8297E37689FCB245994703C61500AE
:10238000E3F0C7FCFC4409061745FF1F1305C5A76A
:102390008297BC48930500081745FF1F034545A5D4
:1023A000829779BF1703FFFFE70263D31747FF1F29
:1023B000130787A34047184B1C409746FF1F23ABCA
:1023C000F6A26316E4001747FF1F2327F7A21305A1
:1023D00084FE9790FFFFE78060A6035564FF978017
:1023E000FFFFE780E06E97A0FFFFE78060D0170354
:1023F000FFFF670003D11703FFFFE70243CE9747B4
:10240000FF1F9387679ED84BDC4789C79700000062
:10241000E78080F985471747FF1F2321F79E9747DD
:10242000FF1F9387E78D9C43930500021745FF1F0D
:102430000345059C83C787031747FF1F2302F79CAB
:10244000B7E70400BC4B82971703FFFF670063CB1D
:102450009747FF1F23ACA79882801703FFFFE7026F
:1024600063C637E404007C4CA1451745FF1F0345B4
:10247000259882977C48A1451745FF1F034545973E
:102480009744FF1F938444968297DC4489EB97001E
:102490000000E78080D91703FFFF6700E3C503D57D
:1024A00067FF9780FFFFE780A062AA896DD1D848B7
:1024B00091476310F7027C4C91451745FF1F034578
:1024C000259382977C4891451745FF1F0345459208
:1024D000829703A9490103D409018947B7E9040098
:1024E0001747FF1F232CF79083A7091D21044204DF
:1024F000829783C784011715FF1F130525036119F0
:102500001717FF1FA304F70283A7491C4180829776
:102510009747FF1F2388078E83A7C91C814609465A
:102520009375F40F4A85829711E99747FF1F83C778
:10253000A79D89C79700FF1FE780C06BB7E704001E
:10254000BC4F2146A1451745FF1F0345658A829769
:1025500099B71703FFFFE70283B893F7052001112E
:102560002E8481CF97000000E78020E913450420E6
:1025700005611703FFFF6700C3B893F70510A9CFE4
:102580009744FF1F93844486DC4897000000E7804F
:1025900020C11737FF1F1307A776184383C784018D
:1025A000034787036318F700DC4489C797000000DE
:1025B000E78080DF85471747FF1F2321F784B7E7B0
:1025C0000400BC4B930500021745FF1F03454582DD
:1025D00082971345041069BF93F70508BDC7974755
:1025E000FF1F83C77782E91719469745FF1F938519
:1025F000C5811305D10093F4F70F1749FF1F034955
:10260000A98097C00000E780404093970401C183F0
:102610001737FF1F1307C77F231DF100231CF1008D
:102620009737FF1F9387477C3ACE3ACAD843230691
:10263000010009CBDC439315890154080D46E1855F
:10264000680082971345040825B793F72500A5C3B2
:102650009737FF1F93874779D84B89476306F7025F
:102660009737FF1F83C7877513F7270011EF918BEB
:1026700099CFB7E70400BC4F1306000A8945173508
:10268000FF1F0345E576829713452400D5B597379C
:10269000FF1F9387E7669C4383C787031737FF1F96
:1026A0002300F77697000000E78060DBF1BF93F727
:1026B000050281CB97000000E78060DA1345040231
:1026C00045BD93F7850081CB97000000E780E0D2FD
:1026D0001345840071BD93F7150081CB970000006E
:1026E000E780A0B41345140061B593F7450081CB92
:1026F00097000000E78060B31345440095BD93F751
:10270000050495C39737FF1F83C7076E91CB9700CA
:102710000000E780A0A491471737FF1F2320F76E22
:1027200013450404B1B593F705010145E38207E4BD
:102730009737FF1F9387476BD84B91476310F70478
:102740009737FF1F938787679C4313D7270085839D
:10275000D98F858B91E7B7E7040083A7071D829780
:10276000B7E70400FC4F91451735FF1F0345456847
:10277000829785471737FF1F2322F7681345040107
:10278000C5BB9737FF1F2381A77882801703FFFF00
:10279000E702E3949737FF1F23AE07649737FF1FC5
:1027A00023AC076485471734FF1F1304645517379C
:1027B000FF1F2325F7641C4083C787031737FF1FBC
:1027C0002300F7649790FFFFE780A08F29C5971734
:1027D000FF1F23A1A7D61C40170500001305A5D78E
:1027E00083C787031737FF1F230CF7601717FF1FD7
:1027F000A30EF7D29737FF1FA388075EB7E7040041
:1028000083A7070882979737FF1F2383A75E1703C5
:10281000FFFF6700038FB7C7898E938767ED171790
:10282000FF1F2329F7D045BF1737FF1F0347C75B9B
:10283000795555E79737FF1F9387075B03C7170045
:1028400005079736FF1FA381E65A03C717008D4679
:102850003377D7029736FF1FA388E65883C6170041
:102860001737FF1F1307C749184393F6F60FA9EE52
:10287000834787031737FF1F2304F7588547173708
:10288000FF1F2303F7569737FF1F938727539C4358
:102890000145998BA9E71703FFFFE702438437E45B
:1028A00004007C48C1451735FF1F034565548297D6
:1028B0003C4885451735FF1F0345855382970145E1
:1028C0001703FFFF6700E38383C7170085466395FF
:1028D000F6008347970379BF8347A70361BF8280D0
:1028E0009737FF1F83C74750A1CF17F3FEFFE702BB
:1028F000037F37E404009737FF1F2387074E7C4888
:1029000085451735FF1F0345A54E82977C4C9145A1
:102910001735FF1F0345C54D82977C4891451735F4
:10292000FF1F0345E54C82973C48C1451735FF1F03
:102930000345054C8297014517F3FEFF6700637C52
:102940007955828017F3FEFFE70263792A840355E5
:1029500065FF9780FFFFE780A0179737FF1F9387DA
:10296000A748D847BE841DEF9790FFFFE780807788
:102970009C48232004009DEB9737FF1F23AE87461A
:102980009737FF1F23A88746B7E70400BC4B89454C
:102990001735FF1F0345C5458297014517F3FEFF15
:1029A00067002376630A8700184375BF80C3973793
:1029B000FF1F23A38744C9BF7955CDB717F3FEFF87
:1029C000E702E3719737FF1F938747548843232615
:1029D000050023240500510597A00000E780C033BF
:1029E00017F3FEFF6700E37117F3FEFFE702236FA3
:1029F0001734FF1F130484511C40411199CF9C4789
:102A00002302B5002AC61CC197000000E78040FBE6
:102A10001C409C4B99C332458297410117F3FEFF3E
:102A20006700236E17F3FEFFE702636B4111444D0D
:102A3000328532842EC69790FFFFE780C0522AC4A9
:102A400022859790FFFFE780205403A84400630C81
:102A50000800B245835744001840224683D54500FC
:102A6000AA8626850298410117F3FEFF6700636975
:102A700017F3FEFFE702A366404D1DC808C0970587
:102A80000000938565031305440197A00000E780CB
:102A900040169737FF1F938767479C43014589E797
:102AA0009737FF1F23A4874617F3FEFF6700636570
:102AB0007D55DDBF17F3FEFFE70263620111680079
:102AC0009305F00F02C602C802CA02CC02CE9700DC
:102AD0000000E780A0F1056117F3FEFF6700636265
:102AE0009737FF1F938787429C43D847A1679D076D
:102AF0006319F70217F3FEFFE702635E01113285E7
:102B00009790FFFFE7802046230AA10081456800D7
:102B100097000000E78080ED056117F3FEFF670076
:102B2000435E82809737FF1F9387473E9C43D84779
:102B3000A167938777036319F70217F3FEFFE70294
:102B4000035A011132859790FFFFE780C041230AA5
:102B5000A1008145680097000000E78020E9056139
:102B600017F3FEFF6700E35982809737FF1F9387B3
:102B7000E7399C43D84795476316F70417F3FEFFE0
:102B8000E702E3550111328532849790FFFFE78019
:102B9000803D230AA10022859790FFFFE780C03E79
:102BA00083574400231BA10081453ECC1C40680094
:102BB0003ECE97000000E78060E3056117F3FEFF5B
:102BC000670023548280930785FF8DC38327C5FF49
:102BD00091CFDC4B81CF17F3FEFFE7024350032573
:102BE00085FF829717F3FEFF6700A351828017F3DA
:102BF000FEFFE702C34E2A8432859790FFFFE780ED
